:100000000C943B050C9456050C9456050C9456051F
:100010000C9456050C9456050C9456050C945605F4
:100020000C9456050C9479180C9456050C945605AE
:100030000C945D2C0C9456050C9456050C945605A6
:100040000C9456050C9456050C940D170C945605FB
:100050000C94110C0C9456050C94D80B0C9456056A
:100060000C948D1D0C9456050C94182B0C9456056D
:100070000C94A3660C9456050C9456053B1E2E1E3C
:10008000221E081EEE1DCA1DDC1D3F21732070209C
:10009000CA1D5D20432023200320B11F5F1F471E80
:1000A0008D2B802BCD2BB12BA52B3E2B4F2B4F2BEC
:1000B000562B722B6D2B522B5A2B562B692B762BD2
:1000C000522B5A2B562B652B7B2B522BDF2B0A0DD9
:1000D000426174743A0020332043656C6C732020B5
:1000E0000020342043656C6C73202000204C6F7717
:1000F000207761726E696E67206C6576656C3A2058
:1001000025642E2564000A0D3D3D3D3D3D3D3D3DB0
:100110003D3D3D3D3D3D3D3D3D3D3D3D3D3D3D3D0F
:100120003D3D3D3D3D3D3D3D3D3D3D000A0D466C67
:1001300069676874436F6E74726F6C0A0D48617200
:1001400064776172653A25642E25640A0D536F66E3
:1001500074776172653A5625642E25642563200004
:100160000A0D74686520757365206F662074686970
:100170007320736F667477617265206973206F6E88
:100180006C79207065726D6974746564200A0D6FF6
:100190006E206F726967696E616C204D696B726F5A
:1001A0004B6F707465722D4861726477617265007F
:1001B0000A0D7777772E4D696B726F4B6F70746590
:1001C000722E646520286329204869537973746509
:1001D0006D7320476D6248000A0D3D3D3D3D3D3D3C
:1001E0003D3D3D3D3D3D3D3D3D3D3D3D3D3D3D3D3F
:1001F0003D3D3D3D3D3D3D3D3D3D3D3D3D000A0DCF
:1002000047656E65726174696E67206465666175C5
:100210006C74204D69786572205461626C65000AC7
:100220000D4D697865722D436F6E6669673A2027B8
:1002300025732720282575204D6F746F7273290050
:100240000A0D466F756E6420424C2D4374726C3AF1
:100250002000256420000A0D0A0D2121204D49535C
:1002600053494E4720424C2D4354524C3A2025646A
:10027000202121000A0D3D3D3D3D3D3D3D3D3D3DA3
:100280003D3D3D3D3D3D3D3D3D3D3D3D3D3D3D3D9E
:100290003D3D3D3D3D3D3D3D3D000A0D496E69748E
:1002A0002E20454550524F4D003A2047656E6572ED
:1002B0006174696E672044656661756C742D506168
:1002C00072616D65746572207573696E67206F6CFD
:1002D0006420537469636B2053657474696E67732B
:1002E000000A0D466C696768742D74696D65202578
:1002F00075206D696E2020546F74616C3A257520ED
:100300006D696E000A0D414343206E6F7420636176
:100310006C696272617465642021000A0D5573690D
:100320006E6720706172616D6574657273657420AB
:100330002564000A0D43616C6962726174696E67BD
:100340002070726573737572652073656E736F725A
:100350002E2E004F4B0A0D000A0D436F6E74726F04
:100360006C3A200048656164696E67486F6C640090
:100370004E6F726D616C20284143432D4D6F646553
:1003800029000A0D3D3D3D3D3D3D3D3D3D3D3D3D51
:100390003D3D3D3D3D3D3D3D3D3D3D3D3D3D3D3D8D
:1003A0003D3D3D3D3D3D3D0A0D002E000A0D2044E2
:1003B0004143206F7220493243204552524F52210F
:1003C00020436865636B204932432C2033567265A5
:1003D000662C2044414320616E6420424C2D4374BE
:1003E000726C005B25695D005B25695D002B204D0B
:1003F000696B726F4B6F70746572202B0048573AAF
:100400005625642E25642053573A25642E256425ED
:10041000630053657474696E673A25642025730020
:10042000493243204552524F52212121004D6973D8
:1004300073696E6720424C2D4374726C3A256421B7
:10044000210028632920486F6C676572204275730C
:100450007300486F6568653A2020202020253569A3
:1004600000536F6C6C486F6568653A2025356900EC
:100470004C756674647275636B3A20253569004F5C
:1004800066662020202020203A20253569004B6513
:10049000696E65200048F668656E726567656C7503
:1004A0006E6700616B742E204C616765004E696356
:1004B0006B3A20202020202025356900526F6C6C7B
:1004C0003A202020202020253569004B6F6D706177
:1004D00073733A202020253569004B313A25346961
:1004E00020204B323A25346920004B333A253469B9
:1004F00020204B343A25346920004B353A253469A5
:1005000020204B363A25346920004B373A25346990
:1005100020204B383A25346920004E693A25346949
:100520002020526F3A253469200047733A253469F8
:10053000202047693A253469200050313A25346932
:10054000202050323A253469200050333A2534694E
:10055000202050343A25346920004779726F202DCD
:100560002053656E736F72004E69636B202534698A
:1005700020282533692E25692900526F6C6C2025AF
:10058000346920282533692E256929004769657259
:1005900020253469202825336929004E69636B20A2
:1005A00025346920282533692E25782900526F6C5F
:1005B0006C2025346920282533692E2578290047A9
:1005C00069657220253469202825336929004E6920
:1005D000636B202534692028253369292825336950
:1005E0002900526F6C6C2025346920282533692935
:1005F0002825336929004769657220253469202838
:1006000025336929282533692900414343202D20BA
:1006100053656E736F72004E69636B2025346920D9
:10062000282533692900526F6C6C202534692028F5
:100630002533692900486F636820253469202825FF
:1006400033692900566F6C746167653A2020202554
:1006500035690052432D4C6576656C3A202025356E
:10066000690052432D4368616E6E656C733A2534A0
:1006700069004B6F6D706173732020202020202053
:10068000005269636874756E673A202025356900E9
:100690004D657373776572743A2020253569005370
:1006A000746172743A202020202025356900506F33
:1006B0007469313A202025336900506F7469323AE9
:1006C000202025336900506F7469333A2020253388
:1006D0006900506F7469343A2020253369005365EE
:1006E00072766F202000536574706F696E742020DD
:1006F000253369005374656C6C756E673A20253339
:10070000690052616E67653A2533692D25336900AA
:1007100045787465726E436F6E74726F6C20200042
:100720004E693A2534692020526F3A2534692000F9
:1007300047733A253469202047693A2534692000F7
:1007400048693A253469202043663A2534692000F7
:10075000424C2D4374726C204572726F727320008C
:100760002025336420202533642020253364202075
:100770002533642000202533642020253364202085
:100780002533642020253364200020253364202075
:100790002533642020253364202025336420004243
:1007A0004C2D4374726C20666F756E64200020259A
:1007B000632020202563202020256320202025631E
:1007C0002000202563202020256320202025632071
:1007D0002020256320002025632020202D2020209C
:1007E0002D2020202D0031300031310031320046E3
:1007F0006C696768742D54696D6520200020202085
:100800002020202535756D696E00546F74616C3A37
:100810002535756D696E0028726573657429000A47
:100820000D506C6561736520636F6E6E6563742037
:100830005370656B7472756D20726563656976655A
:100840007220666F722062696E64696E67204E4F17
:10085000572E2E2E006F6B2E0A0D0054696D656F9A
:1008600075742E0A0D000001020304040506070832
:10087000090A0B0B0C0D0E0F101111121314151584
:1008800016171818191A1B1B1C1D1D1E1F1F2021AF
:100890002122232324242525262727282829292AFD
:1008A0002A2B2B2C2C2D2D2D2E2E2F2F303030316E
:1008B00031323232333333343434353535363636FB
:1008C00037373737383838393939393A3A3A3A3B9D
:1008D0003B3B3B3C3C3C3C3C3D3D3D3D3E3E3E3E4F
:1008E0003E3F3F3F3F3F3F4040404040404141410D
:1008F00041414142424242424242434343434343D5
:1009000043444444444444444445454545454545A1
:100910004545464646464646464646474747474774
:10092000474747474747484848484848484848484D
:100930004849494949494949494949494949494A27
:100940004A4A4A4A4A4A4A4A4A4A4A4A4A4B4B4B04
:100950004B4B4B4B4B4B4B4B4B4B4B4B4B4B4C4CE5
:100960004C4C4C4C4C4C4C4C4C4C4C4C4C4C4C4CC7
:100970004C4D4D4D4D4D4D4D4D4D4D4D4D4D4D4DA8
:100980004D4D4D4D4D4D4D4E4E4E4E4E4E4E4E4E8E
:100990004E4E4E4E4E4E4E4E4E4E4E4E4E4E4E4E77
:1009A0004E4F4F4F4F4F4F4F4F4F4F4F4F4F4F4F58
:1009B0004F4F4F4F4F4F4F4F4F4F4F4F4F4F4F4F47
:1009C00000008F001E01AD013B02CA025803E6037E
:1009D000740402058F051B06A7063307BE074808E7
:1009E000D2085B09E3096B0AF20A780BFD0B810C54
:1009F000040D860D070E870E060F840F00107B1066
:100A0000F5106E11E5115B12CF124213B3132314CC
:100A10009214FE146A15D3153B16A1160517671715
:100A2000C81727188318DE1837198E19E319361AD4
:100A3000871AD61A231B6E1BB61BFD1B411C831C79
:100A4000C31C001D3C1D751DAB1DE01D121E421E6A
:100A50006F1E9A1EC31EE91E0D1F2E1F4D1F691FFC
:100A6000841F9B1FB01FC31FD31FE11FEC1FF51F67
:100A7000FB1FFF1F002011241FBECFEFD0E1DEBF00
:100A8000CDBF13E0A0E0B1E0EAECF8ED02C00590C4
:100A90000D92A63DB107D9F71AE0A6EDB3E001C06B
:100AA0001D92A633B107E1F70C948E060C9400005A
:100AB000282FFB018150853008F023E0842F9927EF
:100AC000332721503040829FD001839FB00D929FE9
:100AD000B00D1124AC59BF4F019724F00E94476C10
:100AE0000192FACF0E94A5650895863038F085E01E
:100AF000A2E0B0E0082E0E94546C08958823C1F74C
:100B00000895582F863048F155E0842F9927252FD6
:100B1000332721503040829FD001839FB00D929F98
:100B2000B00D1124AC59BF4FFB01019724F0019087
:100B30000E94546CFACFA2E6B0E0042E0E94546CDE
:100B4000A0E5B0E088E0FB01182E0E94606C852FC4
:100B50000E9475050E94A56508958823B1F6089541
:100B6000CF93A2E0B0E00E94476C802DC82F815047
:100B7000853020F0C3E08C2F0E9475058C2F9927BB
:100B8000CF9108958091DE08E82FFF27EE0FFF1F19
:100B9000E455F74F808191818D5E9F4F14F0109244
:100BA0000301808191818A5B9F4F24F4809103012E
:100BB000882319F020917B0717C081E080930301FF
:100BC00020917B07280F20937B07253038F088EE93
:100BD00093E09093FC038093FB0306C066E970E00A
:100BE000822F0E946231E6CF822F99279093490885
:100BF0008093480808951F93CF93DF93182F88237D
:100C000089F48091FC088233D8F0809300018091B0
:100C100000018D3518F48DE580930001112309F44E
:100C200079C038C08EEC90E09F938F931F920E9402
:100C300078140F900F900F908091FC08823328F762
:100C400084EF91E00E94F717EC01112309F042C0F4
:100C50008091270390912803823891050CF046C0BB
:100C60008091FC0823E0829FC00111248093000141
:100C7000112369F268EC70E0822F0E94623186EDE8
:100C800090E09F938F931F920E9478140F900F9083
:100C90000F90BDCF809100016AE00E94D76B892F31
:100CA00099279F938F93809100010E94D76B99277A
:100CB0009F938F938CEE90E09F938F931F920E944F
:100CC00078148DB79EB707960FB6F8949EBF0FBEE7
:100CD0008DBF20C0CE010E940018882309F0B8CF34
:100CE000CE010E9400188823A9F3B2CF8091FC089E
:100CF0009927880F991F880F991F8093000111234E
:100D000009F485CF68EC70E084E00E94623181EEE6
:100D100090E0B7CFDF91CF911F910895CFEFD0E151
:100D2000DEBFCDBFEE24FF2414B815B8C7EED3E064
:100D3000E297D7FFFDCF189B6FC1199B78C12DE0BB
:100D40002093020181E887B93E9A8FEF88B98BE141
:100D500084B981E085B98EE38AB987E48BB9469A74
:100D600084B7877F84BF8091600088618093600032
:100D70001092600080ED97E09093FC038093FB035A
:100D80001092D8041092D7041092B1081092B008B3
:100D90001092DA041092D9041092DC041092DB0451
:100DA000243108F43FC188E894E0A0E0B0E08093EB
:100DB000860390938703A0938803B09389032A3016
:100DC00009F465C1243109F462C1289A0E946218AD
:100DD0000E9433180E944D110E94482C0E945B1CF7
:100DE0000E94D72A0E94DA61789486E091E09F936E
:100DF0008F931F920E9478140F900F900F9085E6AA
:100E000090E09F938F938CE490E09F938F931F9239
:100E10001F92809102016AE00E94D76B892F992767
:100E20009F938F93809102010E94D76B99279F9384
:100E30008F938CE291E09F938F931F920E9478147E
:100E40008DB79EB70D960FB6F8949EBF0FBE8DBF9F
:100E500080E691E09F938F931F920E9478140F90E9
:100E60000F900F9080EB91E09F938F931F920E94C1
:100E700078140F900F900F9088ED91E09F938F93CF
:100E80001F920E9478148091C8000F900F900F90CD
:100E9000803209F4F4C0809102018C3008F0C0C0A7
:100EA000299A49E06EED78E083E00E945805C8EE8B
:100EB000D3E0DE010E94476C802D813009F4B9C077
:100EC0008EEF91E09F938F931F920E9478140F9062
:100ED0000F900F9020ED35E0F9018FE01586168612
:100EE0001786108A8150349687FFF8CF80E480936C
:100EF000DD058093DE051092DF058093E005809389
:100F0000E10590EC9093E2051092E3058093E405EF
:100F10008093E5051092E6059093E7059093E80528
:100F20008093E9051092EA058093EB059093EC0518
:100F300081E08093D00541ED55E08BE0E4E0F1E005
:100F4000DA0101900D928A95E1F78DE4DE01F90155
:100F5000182E0E94606C8091850399279F938F9330
:100F60005F934F938FE192E09F938F931F920E9424
:100F700078148DB79EB707960FB6F8949EBF0FBE34
:100F80008DBF80E492E09F938F931F920E9478140C
:100F9000109247041092FF030E944F3F0F900F9052
:100FA0000F908091FF038823E1F31092470480EDB6
:100FB00097E00E94F717EC01CC24DD2472E5A72E00
:100FC00072E0B72E1092FF030E944F3F8091FF0303
:100FD0008823E1F3F601EE0FFF1FEE0FFF1FE05332
:100FE000FA4F858518160CF054C086010156174F2C
:100FF000CE010E940018882309F04EC0D8018C91C0
:10100000882309F049C08093FF030E944F3F8091DD
:10101000FF038823E1F3ECCF199B2FC024E190CE8E
:1010200029983FCF8BE095E0A0E0B0E0C0CE2BE068
:1010300087CEA1E0B0E00E94476C802D8F3F09F47D
:101040003FCF1092850320ED35E08DE4DE01F901FC
:10105000182E0E944F6C90918503F9013D962FE068
:101060008081349618160CF49F5F215027FFF8CF2B
:101070009093850341ED55E06ECF2AE061CE8091DB
:10108000CA00863009F007CF0E94AA6504CF2898CD
:101090009DCE86010156174FF8018081882309F003
:1010A0003FC086010F5F1F4F68010C30110508F427
:1010B00089CFCC24DD2456E5A52E52E0B52EC1E023
:1010C00025C0F601EE0FFF1FEE0FFF1FE053FA4F92
:1010D000858518160CF586010F5F1F4F1F930F9320
:1010E000BF92AF929F930E947814C093F9030F9020
:1010F0000F900F900F900F9083E898E0C80ED91EC4
:10110000D6011C9268010C301105D0F4F601E156AD
:10111000F74F90819923A9F286010F5F1F4FECCF03
:1011200086010F5F1F4F1F930F93BF92AF921F92C5
:101130000E9478140F900F900F900F900F90B4CFE3
:1011400084E792E09F938F931F920E9478140E94ED
:101150004F3F0F900F900F90A1E0B0E00E94476CBE
:10116000802D803509F029C20EE010E0D8010E94E0
:10117000476C802D9927582F442748010894811CDB
:10118000911CD4010E94476C802D480F511DECEF3B
:10119000AE2EEFEFBE2EA00EB11ED5010E94476C01
:1011A000802D9927382F22276DEFC62E6FEFD62E70
:1011B000C00ED11ED6010E94476C802D280F311D14
:1011C000EFEF2F3F3E0709F4B9C2FFEF4F3F5F0734
:1011D00009F4B4C23093D7032093D6035093D903B4
:1011E0004093D8038091D6039091D7039F938F9318
:1011F0008091D8039091D9039F938F9381EE92E0D1
:101200009F938F931F920E9478148DB79EB7079675
:101210000FB6F8949EBF0FBE8DBFA4E0B0E00E9451
:10122000476C802D853008F0B8C20E94B00545E6B5
:101230006EED78E00E9458050E94B00599279F93B3
:101240008F938BE193E09F938F931F920E9478146A
:101250008091E6080F900F900F900F900F9080FDF7
:101260007BC20E94A93C809102018A3009F472C2BB
:10127000843109F46FC2289A80ED97E09093FC03C3
:101280008093FB0385E580937D0788E593E09F933A
:101290008F931F920E9478148091E6080F900F9010
:1012A0000F9082FF54C284E693E09F938F931F9226
:1012B0000E9478140F900F900F900E94222288E8CD
:1012C00093E19093AD038093AC0381E080937C071E
:1012D0000E94FB0582E893E09F938F931F920E94E8
:1012E000781480ED97E00E94F717EC010F900F90B3
:1012F0000F908091FF03882309F4A1C08091190306
:10130000882309F49CC01092FF0380917B078823F7
:1013100009F4D0C00E94C2050E944F3F20910201F3
:101320002A3009F4D0C0243109F4CDC0289A809124
:10133000DE04882309F4CDC08091DE0481508093BF
:10134000DE048091C205882369F081508093C20534
:10135000882341F41092C0051092BF051092BE057B
:101360001092BD058091AC039091AD0301979093CD
:10137000AD038093AC038091AC039091AD03892BB6
:1013800029F080914604882309F4D7C08091AC03EA
:101390009091AD03892B09F4D6C0809112039091EE
:1013A00013038F5F9F4F09F4E7C08091FF038823E9
:1013B00021F08091D404882311F40E9489110E94A5
:1013C000720ECE010E9400188823B9F164968091B4
:1013D0000F03882309F489C0815080930F03809103
:1013E0000001282F3327809127039091280382172B
:1013F00093070CF074C08091AD0480628093AD04BB
:1014000080911203909113038F5F9F4F09F4C8C01E
:101410000E94CC6484E08093FA038091D4048823F2
:1014200021F45AEAE52E55E0F52E0894E11CF11C52
:10143000F2E7EF16FBE0FF0651F00E94A9658091EC
:10144000FA03882309F055CF0E94106552CFEE248D
:10145000FF242091D8033091D9032F5F3F4F309361
:10146000D9032093D8038091D6039091D703019696
:101470009093D7038093D603832F9927D801082E02
:101480000E94546C8091D803D401082E0E94546CA1
:101490008091D703D501082E0E94546C8091D60309
:1014A000D601082E0E94546C84E190E00E94F71748
:1014B000EC01C3CF0E9468430E944F3F209102017C
:1014C0002A3009F030CF28988091DE04882309F073
:1014D00033CF80916F00806280936F0032CF809114
:1014E000AD048F7D8093AD0493CF809387071092D6
:1014F000B9041092B8041092B7041092B604109276
:10150000B5041092B40480911203909113038F5F7D
:101510009F4F09F064CF8091DE04882309F05FCFEC
:1015200088E99AE39093FC038093FB0380E09CE0BE
:10153000909313038093120352CF2A3079F1243110
:1015400069F1289A32CF0E94ED2A85E090E09093CD
:10155000AD038093AC0380915A0890915B0801968B
:1015600090935B0880935A08809112039091130323
:101570008F5F9F4F09F019CF8091D404882309F41D
:1015800014CF80E197E29093FC038093FB0380E803
:1015900090E0909313038093120307CF289805CF10
:1015A00080E797E19093FC038093FB0380E093E056
:1015B00090931303809312032BCF0E94E92E8AE9A4
:1015C00092E09F938F931F920E94781431E0932EA4
:1015D0000F900F900F90C0E5D0E08E010F5F1F4F6E
:1015E00022E0C22ED12CCC0EDD1E93E0A92EB12C10
:1015F000AC0EBD1E84E0682E712C6C0E7D1EB5E015
:101600004B2E512C4C0E5D1EA6E02A2E312C2C0E9A
:101610003D1EE2E09E1609F48BC0F3E09F1609F42C
:101620008AC023E0291508F483C080910201843127
:1016300068F085E08093F908109217098BE1809398
:10164000F5088EE48093140980931509DE010E9449
:10165000476C802D8C3008F068C0D8010E94476C20
:10166000802D8C3008F061C0D6010E94476C802D1F
:101670008C3008F05AC0D5010E94476C802D8C3008
:1016800008F053C0DE010E94476C802D8093DE0875
:10169000D8010E94476C802D8093DF08D6010E94FC
:1016A000476C802D8093E008D5010E94476C802D07
:1016B0008093E108D3010E94476C802D8093E2085B
:1016C000D2010E94476C802D8093E308D1010E94D3
:1016D000476C802D8093E408A7E5B0E00E94476C3A
:1016E000802D8093E50881E0981651F4A9EAB2E0D4
:1016F000BF93AF931F920E9478140F900F900F909A
:1017000045E66EED78E0892D0E9481059394B5E061
:10171000B91508F07ECF83E00E94750580E5A1E051
:10172000B0E0082E0E94546C1FCD0E94D02EE8CF4E
:101730000E94B62F7ACF0E94813077CF1092D903C2
:101740001092D8031092D7031092D6034BCD80E7A6
:1017500093E0ABCD289890CD83E393E09F938F9354
:101760001F920E94781488EE93E00E94F717EC0114
:101770000E94611C0F900F900F90CE010E940018E4
:101780008823D9F383E593E09F938F931F920E9460
:1017900078140F900F900F9064CD84E093E09F93A6
:1017A0008F931F920E9478140F900F900F903DCD51
:1017B0001F920F920FB60F9211248F939F93EF9366
:1017C000FF93809111038823A9F48091ED039091F8
:1017D000EE030196FC01E35DF94FE081ED3079F015
:1017E0008639910561F09093EE038093ED03E093C9
:1017F000C6000EC01092EE031092ED0309C01092C5
:10180000EE031092ED0381E080931103E093C60094
:10181000FF91EF919F918F910F900FBE0F901F90AE
:1018200018951F920F920FB60F9211242F933F938A
:101830004F935F938F939F93AF93BF93EF93FF93D8
:1018400090E08091C6008093E5035091F3035639F0
:1018500010F09093F4038091E5038D3091F0209186
:10186000F403822F99278130910509F46CC08230EE
:1018700091050CF48EC0029709F47FC01092F40316
:10188000A8C02091F403223061F79093F403852FD0
:1018900099278657984FFC01329740812091EF039A
:1018A0003091F003241B3109DC0111978C91281B26
:1018B0003109C9019F709093F0038093EF030024D6
:1018C000880F991F001C880F991F001C892F902DCD
:1018D000982F935C9093F1032F733070235C2093C7
:1018E000F2038081891709F46EC090E08091E203D1
:1018F0008F5F8093E2033091E403332309F069C0E2
:10190000992309F466C081E08093E403580F509353
:10191000E1035150E52FFF27E657F84F8DE0808314
:1019200080918C07823509F054C088E190E02CE06A
:101930000FB6F894A895809360000FBE20936000C6
:101940003093F90346C02F5F2093F403E52FFF2760
:10195000E657F84F8091E50380835F5F5093F30370
:101960002091E5038091EF039091F003820F911D88
:101970009093F0038093EF032CC0E52FFF27E657E9
:10198000F84F8091E5038083563938F31092F403C1
:10199000E7CF892B09F072CF8091E503833259F0AC
:1019A0008091E50380938A0781E08093F30380911F
:1019B000E5039927DDCF8091E403882389F781E04F
:1019C0008093F403EDCF8C91821709F08ECF91E0D4
:1019D00092CFFF91EF91BF91AF919F918F915F91C6
:1019E0004F913F912F910F900FBE0F901F90189520
:1019F000AC01A0E0B0E09D01A817B90748F4EDE202
:101A0000F6E08191280F311D1196A417B507C8F390
:101A10003F70FD01E35DF94FC9010024880F991F54
:101A2000001C880F991F001C892F902D835C8083D8
:101A30001196FD01E35DF94F2F733070822F835CA7
:101A40008083A25DB94F8DE08C9310921103809139
:101A50002D068093C6000895BF92CF92DF92EF9239
:101A6000FF920F931F93CF93DF93CDB7DEB72C85F3
:101A70009D857E85BB2483E280932D069F5990939C
:101A80002E0620932F0603E010E0772309F4ADC063
:101A9000CF84D88843E1E42EF12CEC0EFD1EA989F9
:101AA000BA897150109709F4A0C0109709F43CC08E
:101AB000F601EB0DF11DB3949081119789F4772312
:101AC000A1F1F70122E030E0E20EF31ED701C08061
:101AD000D180E20EF31E0D90BC91A02DBB2471505D
:101AE000109719F1F601EB0DF11DB3944081119798
:101AF00009F466C01097D1F0F601EB0DF11DB39417
:101B000060811197A1F4772391F0F7013296D70104
:101B1000CD90DC9032E0E32EF12CEE0EFF1EA08182
:101B2000B181BB24715003C090E040E060E0F80157
:101B3000E35DF94F892F86958695835C80830F5FDF
:101B40001F4FF801E35DF94F892F9927837090703B
:101B500082959295907F9827807F982755279A01A4
:101B6000329522952F7023273F702327822B835C89
:101B700080830F5F1F4FF801E35DF94F4F70507086
:101B8000440F551F440F551F862F99270024880F97
:101B9000991F001C880F991F001C892F902D842BE2
:101BA000835C80830F5F1F4FF801E35DF94F6F7314
:101BB000635C60830F5F1F4F109709F076CF15C0ED
:101BC000772309F4B3CFF701A2E0B0E0EA0EFB1EE1
:101BD000D701C080D18022E030E0E20EF31E0D90EC
:101BE000BC91A02DBB24715085CFC8010E94F80C78
:101BF000DF91CF911F910F91FF90EF90DF90CF90E9
:101C0000BF900895A3E07A2F4091E103465009F474
:101C10005FC0E72FFF27E657F84F80818D537F5F26
:101C2000E72FFF27E657F84F20812D537F5FE72FDF
:101C3000FF27E657F84F30813D537F5FE72FFF279F
:101C4000E657F84F60816D537F5F9927880F991F82
:101C5000880F991F522F52955F70582B822F99270A
:101C60008F70907082959295907F9827807F9827AB
:101C7000232F26952695282B832F992783709070E4
:101C80000024969587950794969587950794982FA5
:101C9000802D682B41504F3FD9F0EA2FFF27E657A0
:101CA000F84F5083AF5F41504F3F91F0EA2FFF272D
:101CB000E657F84F2083AF5F41504F3F49F0EA2F7E
:101CC000FF27E657F84F6083AF5F442309F0A1CFA9
:101CD0008DE897E09093E0038093DF03A350A093F7
:101CE000DE030895CF93DF93CDB7DEB722970FB60B
:101CF000F894DEBF0FBECDBF8091E403882309F4C2
:101D0000AFC20E94020E80918B07823609F471C027
:101D100080918C0799278436910509F457C0853640
:101D2000910584F58136910509F44EC182369105FD
:101D30000CF4C2C08236910509F49AC1833691052C
:101D4000C1F48091DA039091DB03892B09F04FC233
:101D5000A091DF03B091E0039C91992309F03DC26B
:101D60009C918AE0989FC00111249093DB0380939B
:101D7000DA031092E4031092E0031092DF03109252
:101D8000DE036EC28C36910509F410C18D369105C3
:101D90000CF0B3C08736910509F42BC18836910544
:101DA00041F78FEF80930F03E091DF03F091E003A1
:101DB000808190913F04892B80933F04882311F008
:101DC0001092E60381E08093EA03D3CFE091DF0332
:101DD000F091E00390818AE0989FC00111249093D4
:101DE0000D0380930C03892B21F281E08093E9039A
:101DF000C0CF80918C0799278037910509F4F2C0F4
:101E0000813791050CF485C08337910509F45BC1D6
:101E1000843791050CF03CC18137910509F078CFEA
:101E2000A091DF03B091E0038C918F3F09F40CC2C5
:101E30008C91882309F003C281E08C93A091DF0389
:101E4000B091E00345E66EED78E08C910E94580574
:101E5000809111038823E1F3E091DF03F091E00327
:101E60008081898380E58A8385E690E09F938F93C4
:101E70008EED98E09F938F9321E030E03F932F9376
:101E8000CE0102969F938F933F932F93CE01820FA3
:101E9000931F9F938F9383E08F9381E08F9381E5CE
:101EA0008F930E942C0DADB7BEB71F960FB6F89456
:101EB000BEBF0FBEADBF2CCF8B34910509F059CFFB
:101EC000E091DF03F091E003808191819093F00431
:101ED0008093EF042091ED043091EE04821B930B6C
:101EE000845E9D4F68E671E00E94F76B845B9040D2
:101EF0009093EC048093EB043CCF8437910509F474
:101F00007CC08637910509F034CF81E08093E803E7
:101F100030CF8D36910529F18E3691050CF093C0A6
:101F20008B34910509F0F4CEA091DF03B091E0036A
:101F30008D919C919093F0048093EF042091ED0497
:101F40003091EE04821B930B845E9D4F68E671E036
:101F50000E94F76B845B90409093EC048093EB04B9
:101F6000D7CE809111038823E1F3A091DF03B091D4
:101F7000E0039C91913009F43FC1198281E090E027
:101F80009F938F93CE0101969F938F9381E08F93C0
:101F90008F938DE48F930E942C0D8DB79EB707967B
:101FA0000FB6F8949EBF0FBE8DBFB2CE8FEF809359
:101FB0000F03E091DF03F091E00380818093400400
:101FC00081E08093EB03D5CEE091DF03F091E00355
:101FD000E081E03258F08FE1809310038FEF80931F
:101FE0000F03C7CE81E08093E70392CEE093100306
:101FF000F5CF81E08093EC03BCCE8091E103853185
:1020000008F4DAC0E091DF03F091E00380E1A5E697
:10201000B7E001900D928A95E1F780911103882332
:10202000E1F31F9280910E038F9384E58F930E94BA
:102030002C0D8AEF8093DC038FEF80930F030F90BA
:102040000F900F9096CE8E36910509F061CE80915B
:1020500011038823E1F38DE490E09F938F9380ED4B
:1020600095E09F938F9381E08F938F938EE492CF2F
:10207000A091DF03B091E0038BE0EDE7F7E00D9076
:1020800001928A95E1F78091860780936208A6CF36
:102090008437910509F03CCE8091E103853108F445
:1020A000BCC0A091DF03B091E00380E1E5E6F7E07A
:1020B0000D9001928A95E1F780EF8093DC038FEF1A
:1020C00080930F0325CE2091DF033091E003F901C7
:1020D00080818150853018F481818035E9F0198242
:1020E000809111038823E1F381E090E09F938F9327
:1020F000CE0101969F938F9381E08F938F9383E519
:102100008F930E942C0DEDB7FEB737960FB6F8945B
:10211000FEBF0FBEEDBFFCCD6EED78E085E62E5F15
:102120003F4FDB01F901982F01900D929A95E1F74D
:1021300022503040482FD9018C910E948105809116
:1021400014099927AA27BB27BC01CD0124EC39E04B
:1021500040E050E00E94B86BDC01CB018093A60305
:102160009093A703A093A803B093A90380911509A6
:102170009927AA27BB27BC01CD010E94B86BDC01BF
:10218000CB018093A2039093A303A093A403B093E5
:10219000A503E091DF03F091E00380810E947505C3
:1021A0000E94B005898380E00E94FB056EE670E026
:1021B00089810E94623194CFE091DF03F091E003C6
:1021C00080819181A281B381809365079093660796
:1021D000A0936707B093680720CF8AE0989FC0015B
:1021E00011240E94F71790932C0680932B06A09140
:1021F000DF03B091E003B4CD40ED55E08DE4FA018A
:10220000282F0D9001922A95E1F7A8EEB3E0FA018C
:10221000182E0E94606C9983B1CEA091DF03B0911B
:10222000E0038D919D910D90BC91A02D8093650749
:1022300090936607A0936707B09368073DCF8630F9
:1022400008F400CE85E0F9CD0E94B005E091DF03EF
:10225000F091E0038083A091DF03B091E003E8CD2B
:1022600022960FB6F894DEBF0FBECDBFDF91CF919F
:102270000895CF93C82F8A3029F08091C00085FF40
:10228000FCCF04C08DE00E943911F7CFC093C60087
:1022900080E090E0CF910895089588E18093C10097
:1022A0008091C00082608093C0008091C1008068EE
:1022B0008093C1008091C10080648093C1008AE254
:1022C0008093C40080910C0390910D030E94F71736
:1022D00090935A07809359078CED90E00E94F7176E
:1022E000909389078093880710925B078CE4809312
:1022F0005C0784E080935F078AE080935D0781E05C
:1023000080935E071092E0031092DF031092DE03C9
:102310000895EF92FF920F931F93809111038823EA
:1023200009F478C28091EA03882309F082C0809181
:10233000EB03882329F080911103882309F07FC1E2
:102340008091E803882329F080911103882309F004
:102350005BC18091EC03882329F0809111038823CD
:1023600009F036C180918807909189070E94001872
:10237000882329F080911103882309F0C8C0809137
:102380000C0390910D03892B09F084C18091E9031E
:10239000882329F080911103882309F00FC28091CE
:1023A000DA039091DB03892B09F07EC120911003A1
:1023B0002F3F59F180E190E09F938F93822F9927CF
:1023C00082959295907F9827807F9827845F9E4F73
:1023D0009F938F9381E090E09F938F9380E193E0B0
:1023E0009F938F9382E08F9381E08F9381E48F930B
:1023F0000E942C0D8FEF809310038DB79EB70B9624
:102400000FB6F8949EBF0FBE8DBF809162088823DF
:1024100029F080911103882309F05EC08091E703C1
:10242000882309F4F7C180911103882309F4F2C1CC
:1024300039C080911103882309F479CF0E942B229F
:1024400084E190E09F938F939091E60384E1989FBD
:10245000C0011124865D9C4F9F938F9381E090E093
:102460009F938F9386EE93E09F938F9382E08F9359
:1024700081E08F9388E48F930E942C0D8091E60376
:102480008F5F2DB73EB7255F3F4F0FB6F8943EBF25
:102490000FBE2DBF843008F4B8C11092E60310922D
:1024A000EA0345CF86E190E09F938F938CEA98E012
:1024B0009F938F9381E08F938F9380E58F930E94FA
:1024C0002C0D1092E7038DB79EB707960FB6F894C0
:1024D0009EBF0FBE8DBF9EC181E090E09F938F9302
:1024E00082E698E09F938F9381E08F938F9382E4AD
:1024F0008F930E942C0D109262082DB73EB7295F72
:102500003F4F0FB6F8943EBF0FBE2DBF87CF8091CF
:10251000F5089927880F991F880F991F7C010027BC
:10252000F7FC0095102F8091290590912A05A09124
:102530002B05B0912C05BC01CD01A80197010E948B
:102540002C6C30937607209375078091210590912C
:102550002205A0912305B0912405BC01CD01A8015D
:1025600097010E942C6C3093780720937707809115
:10257000C104809379078091C00480937A0788E032
:1025800090E09F938F9385E797E09F938F9381E0EF
:102590008F9383E08F9387E78F930E942C0D809118
:1025A0007B072DB73EB7295F3F4F0FB6F8943EBF6C
:1025B0000FBE2DBF853018F086E080937B0783E641
:1025C00090E00E94F7179093890780938807D7CEF1
:1025D0008BE090E09F938F938DE797E09F938F938D
:1025E00081E08F9380910E038F9387E48F930E94F5
:1025F0002C0D1092EC038DB79EB707960FB6F8948A
:102600009EBF0FBE8DBFAECE8AE090E09F938F93AA
:102610008BE597E09F938F9381E08F938F9386E56F
:102620008F930E942C0D1092E8032DB73EB7295FBF
:102630003F4F0FB6F8943EBF0FBE2DBF8ACE0E940B
:102640002B2280E590E09F938F938AE293E09F9303
:102650008F9321E030E03F932F9389E293E09F93A3
:102660008F933F932F9380E494E09F938F9383E025
:102670008F9381E08F938CE48F930E942C0D1092A6
:10268000EB038DB79EB70F960FB6F8949EBF0FBEA3
:102690008DBF56CE8091590790915A070E9400181D
:1026A000882309F077CE72CE80912B0690912C066C
:1026B0000E940018882309F479CE809111038823A1
:1026C00009F474CE8091F5089927880F991F880F17
:1026D000991F7C010027F7FC0095102F8091290598
:1026E00090912A05A0912B05B0912C05BC01CD013C
:1026F000A80197010E942C6C30931E0620931D06A2
:102700008091210590912205A0912305B091240587
:10271000BC01CD01A80197010E942C6C30932006CA
:1027200020931F062091A8093091A9094091AA0978
:102730005091AB09DA01C90103E0880F991FAA1F64
:10274000BB1F0A95D1F7820F931FA41FB51F820FDD
:10275000931FA41FB51F20918603309187034091DA
:10276000880350918903BC01CD010E942C6C3093E9
:102770002206209321068EE090E09F938F938DE1B7
:1027800096E09F938F9381E08F938F9383E48F9351
:102790000E942C0D8091DA039091DB030E94F717C1
:1027A00090932C0680932B062DB73EB7295F3F4FA1
:1027B0000FB6F8943EBF0FBE2DBFF8CD82E490E077
:1027C0009F938F9380E298E09F938F9381E08F9304
:1027D0008F9384E48F930E942C0D1092E9038DB7A0
:1027E0009EB707960FB6F8949EBF0FBE8DBF80911F
:1027F0000C0390910D03009709F4D1CD0E94F717B7
:1028000090935A0780935907CACD8093E60310929C
:10281000EA038DCD1F910F91FF90EF900895982FAF
:1028200080916308813031F0892F0E943911282F5F
:1028300033270CC080914104E82FFF27E65DFC4F51
:1028400090838F5F8093410421E030E0C9010895B7
:102850000F931F93CF93DF938C01EB01672B71F0E4
:10286000F80181918F010E940F14219739F0F8012E
:1028700081918F010E940F14219791F7DF91CF91E1
:102880001F910F9108950F931F93CF93DF938C01A6
:10289000EB01672B81F0F8010F5F1F4F84910E94BD
:1028A0000F14219741F0F8010F5F1F4F84910E9490
:1028B0000F14219781F7DF91CF911F910F91089508
:1028C000CF93C82F181634F480E20E940F14C15021
:1028D0001C16D4F3CF910895CF93C82F181634F453
:1028E00080E30E940F14C1501C16D4F3CF910895B9
:1028F0002F923F924F925F926F927F928F929F9210
:10290000AF92BF92CF92DF92EF92FF920F931F93FD
:10291000CF93DF93CDB7DEB7E0970FB6F894DEBF65
:102920000FBECDBF26968FAD26972896EEADFFAD94
:1029300028978824992454018093630848E4C42E7E
:10294000D12CCC0EDD1E7F01C701F701149111239C
:1029500031F0153221F00894E11CF11CF6CFB701DB
:10296000681B790B09F095C0112309F43DC2089446
:10297000E11CF11C1FA63FA4232C0FEF39A6F70181
:102980000894E11CF11C14911537C9F1812F806264
:102990008837A9F1103209F440C0133209F48DC010
:1029A0001A3209F479C01D3209F476C01B32C9F11C
:1029B0001E32C9F1103309F48AC0812F8153893046
:1029C00008F07EC060E070E0CB01880F991F880F8F
:1029D000991F880F991F860F971F680F791F610F26
:1029E000711D60537040F7010894E11CF11C1491B3
:1029F000812F80538A3040F3262E153739F630FE6A
:102A00003DC0F60184E090E0C80ED91E8080918020
:102A1000A280B380103209F0C0CF89A5882309F0C5
:102A2000AECF19A7ACCFF7010894E11CF11C1491AB
:102A30001A3209F451C060E070E014C0CB01880F75
:102A4000991F880F991F880F991F860F971F680F6E
:102A5000791F610F711D60537040F7010894E11CEC
:102A6000F11C1491812F80538A3040F3EFEF6F3FB8
:102A70007E0714F46FEF7FEF062F86CFF60182E01A
:102A800090E0C80ED91E808191814C01AA24BB24FC
:102A900081CF0E94431468CF1A3251F4F60182E0CC
:102AA00090E0C80ED91E208022200CF068CF21941F
:102AB00090E1392AEFED3E2262CF98E0392A5FCFCC
:102AC0001836C9F01C36D1F481E0382A58CF34FCCE
:102AD00056CFF0E23F2A53CFF60182E090E0C80ED5
:102AE000D91E608171819FEF6F3F790714F46FEFFA
:102AF0007FEF062F44CF24E0322A41CF133609F46A
:102B00004DC1143409F41FC1143609F41CC119361F
:102B100009F419C11F3409F40FC11F3609F40CC19F
:102B2000103709F4F9C0133709F4B2C0153509F4A8
:102B3000ECC0153709F4E9C0183509F444C018375A
:102B400009F441C0112309F44FC1CE0101969DA79C
:102B50008CA7198381E0482E19A6632C7724042DB5
:102B60005FA4541857FC2DC029A5222331F10F5F13
:102B7000050DC30180739070892B09F42FC12223A6
:102B800009F027C166FC1BC1C30180739070809758
:102B900009F410C1852D0E946C14842D992787FD9E
:102BA0009095BC018CA59DA50E94281464FECCCEF6
:102BB000822D801B0E946014C7CE66FED9CF0E5FA7
:102BC000D7CF5524D1CFE0E1EEA733FE07C0811463
:102BD0009104A104B10411F0F0E43F2A19A60FA753
:102BE00007FD02C02FED3222CE0189969DA78CA74A
:102BF00081149104A104B10419F49FA5992361F1F2
:102C0000EEA54E2E55246624772418AA8414950424
:102C1000A604B70410F0F1E0F8ABC501B401A301BC
:102C200092010E940A6CDC01CB01082F8A30F0F47B
:102C3000005DECA5FDA50293FDA7ECA7C501B401BD
:102C4000A30192010E940A6C49015A01F8A9FF23CD
:102C5000E1F62EA5283079F0632C7724CE01019679
:102C6000482EFCA54F1A28E2420E79CF095A183592
:102C700001F70F7DDECF632C772463FEEFCF0033A7
:102C800069F380E3ECA5FDA58293FDA7ECA7E6CF51
:102C9000F60182E090E0C80ED91E0190F081E02D8F
:102CA000FDA7ECA7EF2B81F4FE013196FDA7ECA761
:102CB00088E289838EE6818385E78B838CE68C832B
:102CC0008D8389E28E831F8207FD15C0802F99278F
:102CD00087FD9095AC0160E070E08CA59DA50E94F9
:102CE000D16A009731F0482EFCA54F1A04150CF05C
:102CF00033CF402E31CFECA5FDA501900020E9F7A0
:102D000031974E2E2CA5421A27CF153511F481E0AC
:102D1000382A9AE09EA762CFF60182E090E0C80EC2
:102D2000D91E808191814C01AA24BB2490E19EA7E9
:102D3000E0E43E2A18E752CF1F3411F4E1E03E2AC6
:102D4000F8E0FEA74BCF143411F491E0392A30FE9D
:102D500018C0F60184E090E0C80ED91E80809180F2
:102D6000A280B380B7FE0AC0B094A09490948094DF
:102D7000811C911CA11CB11C8DE289A79AE09EA721
:102D80002ECFF60182E090E0C80ED91E808191819D
:102D90004C01AA2497FCA094BA2CE4CFFE013196F2
:102DA000FDA7ECA7F60182E090E0C80ED91E808155
:102DB0008983D0CE822D801B0E946C14EBCE80E3E1
:102DC0008AA71BA762E070E0CE018A960E942814B1
:102DD000DBCE61E070E0CE018996F8CF822D801BBA
:102DE0000E94601429A5CBCEE0960FB6F894DEBF02
:102DF0000FBECDBFDF91CF911F910F91FF90EF904C
:102E0000DF90CF90BF90AF909F908F907F906F900A
:102E10005F904F903F902F9008951F920F920FB6A2
:102E20000F9211242F933F935F936F937F938F9310
:102E30009F93AF93BF93EF93FF938091FA038823FF
:102E400029F08091FA0381508093FA038091CB0599
:102E5000882319F081508093CB0580910204815022
:102E60008F3F09F493C0809302048091FB039091FB
:102E7000FC03892B01F18091FB039091FC030197E6
:102E80009093FC038093FB038091FB039091FC03E0
:102E9000209112033091130382239323892B89F00D
:102EA000809102018A3009F48BC0479A8091E6082C
:102EB00083FF8DC010C08FEF9FEF9093130380931B
:102EC0001203809102018A3009F478C047988091FA
:102ED000E60883FF7CC086B19927FC01E071F070A1
:102EE00084FF0AC08091FD039091FE0301969093A8
:102EF000FE038093FD036BC08091FD039091FE0360
:102F0000892B49F18091FD039091FE038A569140EF
:102F100010F58091FD039091FE0369E270E00E943C
:102F2000E36B8091FD039091FE03860F971F9093B2
:102F3000FE038093FD038091FD039091FE030B97A8
:102F400008F440C08091FD039091FE030A9790938E
:102F5000F0048093EF048091EF049091F0042091AD
:102F6000ED043091EE04821B930B845E9D4F68E666
:102F700071E00E94F76B845B90409093EC04809327
:102F8000EB041092FE031092FD0321C089E08093B0
:102F90000204809114038F5F81708093140388234F
:102FA00019F481E08093FF03809100049091010463
:102FB0000196909301048093000457CF5A9887CFCD
:102FC0005A9A85CFF093F004E093EF04C4CFFF91B9
:102FD000EF91BF91AF919F918F917F916F915F9191
:102FE0003F912F910F900FBE0F901F901895209139
:102FF000000430910104280F391FC901019608957A
:103000002091000430910104821B930B892F992792
:103010008695807490700895CF93DF930E94F71780
:10302000EC01CE010E9400188823D9F3DF91CF91E3
:1030300008951F93CF93DF930E94F717EC011FECC5
:1030400008C080911903882321F0909319031093ED
:103050007A00CE010E940018982F882391F3DF9107
:10306000CF911F9108959FB7F8945F983E9A469A22
:103070008091B0008F708093B0008091B000836029
:103080008093B0008091B1008B738093B1008091E8
:10309000B1008B608093B1001092B2008FEF8093EB
:1030A000B3008091B00080688093B0008091700080
:1030B0008A7F80937000809170008260809370009E
:1030C0009FBF08958AE090E00E94F71790930A044A
:1030D0008093090482E085BD83EA84BD17BC88E73C
:1030E00088BD86E086BD80916E00816080936E0011
:1030F00008951F920F920FB60F9211242F933F93B2
:103100004F935F936F937F938F939F93AF93BF93EF
:10311000EF93FF93809102018431C0F48091030406
:10312000882309F446C0209104043091050441E04D
:103130002F37340708F49CC08FEF8093B3002F5FC4
:1031400030403093050420930404A4C38091030409
:10315000882349F78091B00086FFADC08091B00010
:103160008F7B8093B000E0910804EE2309F0EFC05C
:1031700080910D09282F33278DED96E0289FA0011F
:10318000299F500D389F500D1124CA01209106042B
:1031900030910704821B930B9093050480930404E1
:1031A0001092070410920604469A81E0809303046B
:1031B000BACF8091B00086FFA8C08091B0008F7B0D
:1031C0008093B00089EA93E090930504809304040F
:1031D00080911503909116039C01220F331F280F35
:1031E000391F809192039927880F991F880F991F83
:1031F000280F391F37FD25C2C901959587959595EB
:10320000879590931603809315039093F80380930A
:10321000F7038091350980FFDDC080910609682F92
:103220007727882799272091290530912A054091F1
:103230002B0550912C0557FDE9C1A7E05595479501
:1032400037952795AA95D1F70E94B86B9B01AC01E1
:1032500097FDFAC1F6E05595479537952795FA956C
:10326000D1F78091F7039091F803820F931FDCC090
:103270002F3F310569F060F0A9014F5F50404F3793
:10328000510588F480E88093B3002058304059CF2E
:10329000809104048093B3001092050410920404FA
:1032A00010920304F7C28FEF8093B300509305048C
:1032B00040930404EFC28091B00080648093B0001A
:1032C0008CEB90E0909305048093040480910604B5
:1032D0009091070484549F4F9093070480930604B1
:1032E0008091F903882329F08091DE04853B08F062
:1032F000F2C0469A909108049F5F80910D0989174A
:1033000008F0E6C01092080450CF8091B0008064AD
:103310008093B00080910D09282F33278DED96E022
:10332000289FA001299F500D389F500D1124CA01DC
:103330002091060430910704821B930B909305049F
:10334000809304049C0181E080930304F0CE89EA19
:1033500093E090930504809304048E2F9927813085
:10336000910509F4BAC0029709F478C1FF27EE0F5E
:10337000FF1FE455F74F80819181880F991F20919D
:10338000040430910504820F931F909305048093E9
:103390000404209104043091050455E02D3D3507C7
:1033A00008F440C18CED95E09093050480930404EB
:1033B0009C012C5B304030930504209304048091E1
:1033C000060490910704820F931F90930704809343
:1033D0000604EBCE80910609682F77278827992766
:1033E0002091290530912A0540912B0550912C05FB
:1033F00057FD07C1E7E05595479537952795EA951D
:10340000D1F70E94B86B9B01AC0197FD22C176E019
:1034100055954795379527957A95D1F78091F7037C
:103420009091F803821B930B9093F8038093F7031A
:1034300080910709282F3327220F331F220F331FB4
:103440008091F7039091F803821793077CF08091A5
:103450000809282F3327220F331F220F331F809193
:10346000F7039091F8032817390724F43093F803F1
:103470002093F7032091F7033091F803809104041F
:1034800090910504280F391F205032408091F70396
:103490009091F80397FDD3C095958795959587955D
:1034A0009093F8038093F70345E02D3D340708F42B
:1034B000B2C08CED95E090930504809304042091B4
:1034C00004043091050430930704209306043BCF95
:1034D000909308046ACE46980DCF80911503909181
:1034E00016039C01220F331F280F391F809192036E
:1034F0009927880F991F880F991F280F391F37FDAB
:1035000099C1C901959587959595879590931603CF
:10351000809315039093F8038093F7038091350906
:1035200080FF30C180910609682F77278827992767
:103530002091290530912A0540912B0550912C05A9
:1035400057FD85C1E7E05595479537952795EA954D
:10355000D1F70E94B86B9B01AC0197FD73C1B6E037
:103560005595479537952795BA95D1F78091F703EB
:103570009091F803820F931F9093F8038093F703C1
:1035800080910709282F3327220F331F220F331F63
:103590008091F7039091F803821793077CF0809154
:1035A0000809282F3327220F331F220F331F809142
:1035B000F7039091F8032817390724F43093F803A0
:1035C0002093F7038091F7039091F803209104046E
:1035D00030910504820F931F805092409093050410
:1035E000809304048091F7039091F80397FD20C124
:1035F00095958795959587959093F8038093F70314
:10360000C8CE21583F4F4F4F5F4FF4CE21583F4F08
:103610004F4F5F4F12CE51E02737350758F487E7F9
:1036200091E049CF81E02737380708F0C2CE87E71D
:1036300091E0BACE309305042093040440CF039662
:103640002BCF2D5F3F4FD8CD215C3F4F4F4F5F4F6A
:1036500001CE215C3F4F4F4F5F4FD9CE8091170372
:10366000909118039C01220F331F280F391F80915E
:1036700091039927880F991F880F991F280F391FC9
:1036800037FDDBC0C90195958795959587959093F2
:103690001803809317039093F6038093F5038091AA
:1036A000350981FF9AC080910A09682F77278827FA
:1036B00099272091210530912205409123055091B1
:1036C000240557FDE2C0A7E0559547953795279506
:1036D000AA95D1F70E94B86B9B01AC0197FDD0C0B1
:1036E000F6E05595479537952795FA95D1F780914E
:1036F000F5039091F603820F931F9093F603809346
:10370000F50380910B09282F3327220F331F220F37
:10371000331F8091F5039091F603821793077CF095
:1037200080910C09282F3327220F331F220F331FBC
:103730008091F5039091F6032817390724F430930C
:10374000F6032093F5038091F5039091F603209101
:10375000040430910504820F931F8050924090938F
:103760000504809304048091F5039091F60397FD7E
:1037700067C095958795959587959093F603809367
:10378000F50307CE80910609682F772788279927A8
:103790002091290530912A0540912B0550912C0547
:1037A00057FD5FC0A7E05595479537952795AA9592
:1037B000D1F70E94B86B9B01AC0197FD4DC0F6E0BC
:1037C0005595479537952795FA95D1F78091F70349
:1037D0009091F803821B930BCFCE80910A09682F3A
:1037E000772788279927209121053091220540913C
:1037F00023055091240557FD3EC0E7E055954795B8
:1038000037952795EA95D1F70E94B86B9B01AC01DB
:1038100097FD2CC066E055954795379527956A9595
:10382000D1F78091F5039091F603821B930B65CF3E
:103830000396DECE2D5F3F4F64CE2D5F3F4F22CFEC
:10384000039697CF215C3F4F4F4F5F4F88CE215853
:103850003F4F4F4F5F4F76CE215C3F4F4F4F5F4FF3
:10386000AECF21583F4F4F4F5F4F9CCF215C3F4F12
:103870004F4F5F4FCFCF21583F4F4F4F5F4FBDCF7F
:10388000215C3F4F4F4F5F4F2BCF21583F4F4F4F42
:103890005F4F19CFFF91EF91BF91AF919F918F91A2
:1038A0007F916F915F914F913F912F910F900FBE3C
:1038B0000F901F90189510927C008FEC80937A00E7
:1038C0000895EF92FF920F931F93CF93DF9303E03E
:1038D00010E0D8010E94476C802DC82FDD27C5312C
:1038E000D10508F02A97C7BD1092120484E690E033
:1038F0000E94191880911D0390911E0380529340DD
:1039000010F4C0E0D0E0CA3FD105E0F48AEAE82E26
:1039100083E0F82EC7BD82E390E00E941918FF9261
:10392000EF921F920E94781480911D0390911E03C4
:103930000F900F900F908052934020F02196CA3F35
:10394000D10540F3D8010C2E0E94546CC09370082E
:103950008CE291E00E941918DF91CF911F910F9195
:10396000FF90EF900895EF92FF920F931F93CF93E4
:10397000DF9300E000930D0400930C0400930B040C
:1039800080ED97E00E94F717EC011CE821E0F22E91
:1039900095EFE92E033009F4ABC000E080912204DA
:1039A000909123048C5F93400CF091C080911C0394
:1039B000815080931C0380912004909121048C5F9E
:1039C00093400CF079C080911B03815080931B03BE
:1039D00080911E0490911F048C5F93400CF04AC0AC
:1039E00080911A03815080931A0388E080934904E0
:1039F0000E94DD2A80911C038A3008F055C0F092A5
:103A00000D048AE080931C0380911B038A3008F028
:103A100043C0F0920C048AE080931B0380911A0348
:103A20008A3098F5F0920B048AE080931A03809113
:103A30004904882379F0CE010E9400188823B9F345
:103A40008CEA93E09F938F931F920E9478140F90BB
:103A50000F900F90109219038FEC80937A00809151
:103A600019038823E1F31A3008F447C0115009F014
:103A700091CF48C080911E0490911F0487509440BC
:103A80008CF180911A038F5FAECF863F80F2F09267
:103A90000B04E0921A03CBCF863F08F4BFCFF0921D
:103AA0000C04E0921B03BACF863F08F4ADCFF0922E
:103AB0000D04E0921C03A8CF809120049091210472
:103AC000875094408CF080911B038F5F7FCF809153
:103AD0002204909123048750944044F080911C0369
:103AE0008F5F67CF0F5F81CF0F5F72CF01E063CF32
:103AF0001B3008F452CF19E050CF8AE090E00E94CA
:103B00001918B4CF86E490E00E941918DF91CF9184
:103B10001F910F91FF90EF9008951F920F920FB693
:103B20000F921124AF92BF92CF92DF92EF92FF9249
:103B30000F931F932F933F934F935F936F937F93B5
:103B40008F939F93AF93BF93EF93FF9320912B0499
:103B5000822F9927AA27BB272F5FFC01429740F4A9
:103B6000E25CFF4FEE0FFF1F0590F491E02D0994EA
:103B700010922B0482E080932A0480912A0480937F
:103B80007C0080912B04882309F443C48FEC80933C
:103B90007A003FC420932B048091780090917900A3
:103BA0002091300430913104820F931F909331049F
:103BB0008093300481E0DFCF20932B048091780044
:103BC0009091790020912E0430912F04820F931F41
:103BD00090932F0480932E0484E0CDCF20932B0468
:103BE00080917800909179002091370530913805C7
:103BF000821B930B90936F0880936E0880916E08E0
:103C000090916F08909339048093380482E0B3CF89
:103C100020932B04809135059091360520917800F2
:103C200030917900821B930B909365088093640810
:103C300080916408909165089093370480933604CE
:103C400087E099CF20932B048091780090917900A0
:103C500090932D0480932C0486E08DCF20932B0429
:103C6000209178003091790030932F0420932E0416
:103C700010922A0482CF20932B0420917800309157
:103C80007900309331042093300481E074CF109296
:103C90002B0481E08093190380910E0490910F040E
:103CA000019690930F0480930E0480917800909178
:103CB000790090931E0380931D0380911D039091C2
:103CC0001E035C01CC24DD2480913A0490913B04D6
:103CD000A0913C04B0913D04A80EB91ECA1EDB1E83
:103CE00080913E048F5F823108F4E8C280911F0307
:103CF00090912003A0912103B09122037C018D01BA
:103D000023E0EE0CFF1C001F111F2A95D1F7E81AC3
:103D1000F90A0A0B1B0BEA0CFB1C0C1D1D1D8091E4
:103D20001204992787FD9095A92FB92FBC01CD01C9
:103D300026EC34E240E050E00E94B86BDC01CB019D
:103D4000E81AF90A0A0B1B0BD801C7010496A11D3A
:103D5000B11DB7FD23C313E0B595A795979587953A
:103D60001A95D1F780931F0390932003A09321030A
:103D7000B093220380916808909169087C01002724
:103D8000F7FC0095102F80911F0390912003A091C4
:103D90002103B0912203E81AF90A0A0B1B0BE092E7
:103DA000D004F092D1040093D2041093D304209154
:103DB000130430911404409115045091160457FDDA
:103DC000FDC2A4E05595479537952795AA95D1F75B
:103DD0008091130490911404A0911504B0911604DD
:103DE000821B930BA40BB50B8093130490931404C4
:103DF000A0931504B09316048091130490911404B9
:103E0000A0911504B09116048E0D9F1DA01FB11F27
:103E10008093130490931404A0931504B093160494
:103E20008091100490911104BC0162957295707F8D
:103E30007627607F7627681B790B209113043091D9
:103E40001404409115045091160457FDB2C2E4E0E9
:103E50005595479537952795EA95D1F78091D004E8
:103E60009091D104821B930B880F991F880F991F83
:103E7000880F991F860F971F97FDA9C29595879563
:103E80009595879595958795959587959093110428
:103E900080931004D601C501D7FC95C2B595A795AE
:103EA0009795879580933A0490933B04A0933C04A4
:103EB000B0933D0489E080933E0482E05CCE209381
:103EC0002B04209178003091790080912E049091FC
:103ED0002F04280F391F809102018A3009F448C24B
:103EE000220F331F220F331F30932F0420932E04F1
:103EF000C90137FD73C295958795959587959595D9
:103F000087959093210480932004809134049091AC
:103F10003504820F931F97FD66C295958795909300
:103F200035048093340420913F0530914005821B75
:103F3000930B9093240380932303209126043091C4
:103F400027048091230390912403280F391F37FD04
:103F500047C235952795309327042093260483E0A4
:103F60000ACE20932B042091780030917900809123
:103F7000300490913104280F391F809102018A305A
:103F800009F407C2220F331F220F331F309331046D
:103F900020933004C90137FDFFC19595879595950C
:103FA000879595958795909323048093220480911B
:103FB000320490913304820F931F97FD0DC29595A3
:103FC000879590933304809332042091410530917A
:103FD0004205821B930B9093260380932503209127
:103FE0002804309129048091250390912603280FFD
:103FF000391F37FDEEC1359527953093290420935D
:10400000280481E0B8CD20932B0480917800909112
:1040100079002091370530913805821B930B9093DE
:104020006F0880936E0880916E0890916F082091C0
:10403000380430913904820F931F90931B048093AE
:104040001A0482E098CD20932B048091350590913D
:1040500036052091780030917900821B930B909364
:1040600065088093640880916408909165082091A8
:10407000360430913704820F931F90931D04809370
:104080001C0487E078CD20932B04809102018A30B4
:1040900009F471C1843109F4A8C18091780090912C
:1040A000790020912C0430912D04820F931F90935E
:1040B0001F0480931E0486E05ECD20932B04809124
:1040C00078009091790020912E0430912F04820F76
:1040D000931F90932F0480932E0410922A044DCDA9
:1040E00020932B04E2CD20932B04809178009091B3
:1040F0007900AA2797FDA095BA2FBC01CD010E9497
:104100003E6B7B018C0180912F0590913005A09131
:104110003105B09132059C01AD01C801B7010E9483
:10412000DE6ADC01CB01BC01CD010E94216BDC0108
:10413000CB019093190480931804809118049091F6
:10414000190402970CF4C6C080912F059091300598
:10415000A0913105B091320520E030E84BE354E402
:10416000BC01CD010E94486B8823DCF580912F05AE
:1041700090913005A0913105B09132052AE037EDDC
:1041800043EA5CE3BC01CD010E94DF6ADC01CB01A4
:1041900080932F0590933005A0933105B09332059D
:1041A0008091AE049091AF04845F9140D0F48091EF
:1041B0002F0590913005A0913105B09132052DEC7D
:1041C0003CEC4CEC5DE3BC01CD010E94DF6ADC01FC
:1041D000CB0180932F0590933005A0933105B093C8
:1041E000320581E0809317048091780090917900E6
:1041F0009093670880936608809118049091190441
:10420000AA2797FDA095BA2F2091F1043091F204CE
:104210004091F3045091F404820F931FA41FB51F23
:104220008093F1049093F204A093F304B093F40408
:104230002091F1043091F2044091F3045091F40480
:1042400057FDB2C00AE055954795379527950A95D1
:10425000D1F78091F1049091F204A091F304B09110
:10426000F404821B930BA40BB50B8093F104909381
:10427000F204A093F304B093F40483E07CCC209385
:104280002B0480912703909128039C01220F331F58
:10429000280F391F809178009091790063E070E0D9
:1042A0000E94E36B260F371F369527953695279585
:1042B000309328032093270385E05DCC80933E0450
:1042C000A0923A04B0923B04C0923C04D0923D04C8
:1042D00082E051CC80911804909119048F5F9F4F18
:1042E0000CF07FCF80912F0590913005A091310582
:1042F000B091320520E030E849E054E4BC01CD0142
:104300000E944B6B18160CF06CCF80912F0590918A
:104310003005A0913105B09132052AE037ED43EA2E
:104320005CE3BC01CD010E94DE6ADC01CB0180931D
:104330002F0590933005A0933105B09332058091FD
:10434000AE049091AF04845F914008F04ACF809111
:104350002F0590913005A0913105B09132052DECDB
:104360003CEC4CEC5DE3BC01CD010E94DE6A2FCF3A
:10437000220F331FB9CD8091780090917900209160
:104380002C0430912D04820F931F019696958795EA
:104390008ECE220F331FFACD0796FFCDD801C7016D
:1043A0000B96A11DB11DD7CC21503C4F4F4F5F4FF5
:1043B00049CF215F3F4F4F4F5F4F49CD215F3F4F67
:1043C0004F4F5F4FFECC0196A11DB11D67CD0F96DB
:1043D00055CD2F5F3F4F0FCE0196F1CD07968BCD78
:1043E0002F5F3F4FB6CD019698CD80917800909188
:1043F000790020912C0430912D04820F931F2FEF10
:1044000037E0281B390B30931F0420931E0486E0ED
:10441000B2CBFF91EF91BF91AF919F918F917F911F
:104420006F915F914F913F912F911F910F91FF904D
:10443000EF90DF90CF90BF90AF900F900FBE0F9096
:104440001F90189590E2EAE2F3E08FE49193815097
:1044500087FFFCCF08951F93CF93DF938091400493
:1044600020912903281710F42093400490913F04D1
:1044700090FF08C080914004882309F41EC1815038
:104480008093400491FF08C080914004821709F492
:10449000E4C18F5F80934004892F992780FF02C079
:1044A00081FD08C10E942222909140049A3008F0B8
:1044B000A2C081E180934104892F99279F938F9314
:1044C00083EE93E09F938F9381E08F930E94781403
:1044D0000F900F900F900F900F9080914004C82F75
:1044E000DD27C730D10509F4BBC1C830D1050CF0B8
:1044F0008CC0C330D10509F455C2C430D1050CF0CD
:10450000DFC0C130D10509F4BBC2C230D1050CF403
:1045100038C31092410483EA94E09F938F93C1E0E3
:10452000CF930E94781484E1809341040F900F9000
:104530000F908091290590912A05A0912B05B091AB
:104540002C05B7FD58C63AE0B595A7959795879580
:104550003A95D1F7BF93AF939F938F938DEA94E0F1
:104560009F938F93CF930E94781488E280934104A5
:104570008DB79EB707960FB6F8949EBF0FBE8DBF3E
:104580008091210590912205A0912305B0912405E9
:10459000B7FD2CC62AE0B595A795979587952A95DE
:1045A000D1F7BF93AF939F938F938CEB94E09F933E
:1045B0008F93CF930E9478148CE3809341042DB79E
:1045C0003EB7295F3F4F0FB6F8943EBF0FBE2DBFD9
:1045D0008091EF049091F0049F938F938BEC94E083
:1045E0009F938F93CF930E9478140F900F900F900A
:1045F0000F900F90D6C780E180934104892F9927AF
:104600009F938F9388EE93E05DCFCB30D10509F473
:104610005DC1CC30D1050CF00FC1C930D10509F412
:104620000BC52A970CF01CC31092410482E796E058
:104630009F938F9311E01F930E94781484E18093DD
:1046400041040F900F900F908091EB049091EC0437
:104650009F938F9381E896E09F938F931F930E947F
:10466000781488E2809341040F900F900F900F9080
:104670000F908091EF049091F0049F938F9380E9C5
:1046800096E09F938F931F930E9478148CE38093FE
:1046900041040F900F900F900F900F908091ED04B8
:1046A0009091EE049F938F938FE996E09F938F9361
:1046B0001F9399CF10924004F5CE20934004E2CE90
:1046C000C530D10509F403C426970CF08CC31092B1
:1046D00041048091DF08E82FFF27EE0FFF1FE4550C
:1046E000F74F808191819F938F938091DE08E82F0F
:1046F000FF27EE0FFF1FE455F74F808191819F93B5
:104700008F938AE195E09F938F9311E01F930E940E
:10471000781484E1809341048DB79EB707960FB655
:10472000F8949EBF0FBE8DBF8091E108E82FFF2750
:10473000EE0FFF1FE455F74F808191819F938F9378
:104740008091E008E82FFF27EE0FFF1FE455F74F99
:104750008081918188589F4F9F938F938AE295E043
:104760009F938F931F930E94781488E28093410453
:104770002DB73EB7295F3F4F0FB6F8943EBF0FBE2F
:104780002DBF8091E308E82FFF27EE0FFF1FE455B0
:10479000F74F8081918182599F4F9F938F93809192
:1047A000E208E82FFF27EE0FFF1FE455F74F808147
:1047B000918182599F4F9F938F938AE395E09F93B6
:1047C0008F931F930E9478148CE3809341046DB7FC
:1047D0007EB7695F7F4F0FB6F8947EBF0FBE6DBF87
:1047E0008091E508E82FFF27EE0FFF1FE455F74FF4
:1047F0008081918182599F4F9F938F938091E4088C
:10480000E82FFF27EE0FFF1FE455F74F80819181BE
:1048100082599F4F9F938F938AE495E09F938F9344
:104820001F930E9478148DB79EB707960FB6F89421
:104830009EBF0FBE8DBFB5C6CD30D10509F447C4AC
:10484000CD30D1050CF452C22E9709F4D9C4815051
:104850008093290310924004A4C6109240041CCEF9
:1048600084E18093410480912703909128039F93D2
:104870008F9384E496E09F938F9311E01F930E949F
:10488000781488E2809341040F900F900F900F905E
:104890000F908091DE0499279F938F9383E596E094
:1048A0009F938F931F930E9478148CE3809341040D
:1048B0000F900F900F900F900F908091AB08992759
:1048C00001979F938F9382E696E0F0CE1092410479
:1048D00080E197E09F938F9311E01F930E947814DB
:1048E00084E1809341040F900F900F908091810795
:1048F000992787FD90959F938F93809180079927A3
:1049000087FD90959F938F9380E297E09F938F937D
:104910001F930E94781488E2809341048DB79EB75C
:1049200007960FB6F8949EBF0FBE8DBF8091820789
:10493000992787FD90959F938F938091830799275F
:104940009F938F9380E397E09F938F931F930E9491
:1049500078148CE3809341042DB73EB7295F3F4F15
:104960000FB6F8943EBF0FBE2DBF809187079927E1
:104970009F938F9380918407992787FD90959F93AC
:104980008F9380E497E09F938F931F930E947814F6
:104990006DB77EB7695F7F4F0FB6F8947EBF0FBECD
:1049A0006DBFFFC5109241048091B0089091B1088D
:1049B0009F938F938091AE089091AF089F938F93B0
:1049C0008AED94E09F938F9311E01F930E947814D7
:1049D00084E1809341046DB77EB7695F7F4F0FB666
:1049E000F8947EBF0FBE6DBF8091B4089091B5085A
:1049F0009F938F938091B2089091B3089F938F9368
:104A00008AEE94E09F938F931F930E94781488E21C
:104A1000809341048DB79EB707960FB6F8949EBF5A
:104A20000FBE8DBF8091B8089091B9089F938F9366
:104A30008091B6089091B7089F938F938AEF94E086
:104A40009F938F931F930E9478148CE3809341046B
:104A50002DB73EB7295F3F4F0FB6F8943EBF0FBE4C
:104A60002DBF8091BC089091BD089F938F9380913A
:104A7000BA089091BB089F938F938AE095E083CF0B
:104A80008091E60880FD1CC084E1809341048EE89B
:104A900094E09F938F9311E01F930E94781488E213
:104AA000809341040F900F900F9085E994E09F93BD
:104AB0008F931F930E9478140F900F900F9071C5E1
:104AC000109241048091D0049091D104A091D2041D
:104AD000B091D304BC01CD0125E030E040E050E0CE
:104AE0000E942C6C3F932F9382E594E09F938F93C9
:104AF00011E01F930E94781484E1809341040F9089
:104B00000F900F900F900F908091CC049091CD0456
:104B1000A091CE04B091CF04BC01CD0125E030E0DE
:104B200040E050E00E942C6C3F932F9381E694E08C
:104B30009F938F931F930E94781488E2809341047F
:104B40000F900F900F900F900F9080911D039091F8
:104B50001E039F938F9380E794E09F938F931F93FF
:104B60000E9478148CE3809341040F900F900F9073
:104B70000F900F9087B599279F938F938FE794E0BD
:104B800095CD209709F063CE109241048DEE93E00D
:104B90009F938F9311E01F930E94781484E1809378
:104BA00041040F900F900F9085E690E09F938F93B4
:104BB0008CE490E09F938F93DF93CF9380910201D9
:104BC0006AE00E94D76B892F99279F938F938091DA
:104BD00002010E94D76B99279F938F938DEF93E0EB
:104BE0009F938F931F930E94781488E280934104CF
:104BF0002DB73EB7235F3F4F0FB6F8943EBF0FBEB1
:104C00002DBF81ED95E09F938F930E94B00599276A
:104C10009F938F9382E194E09F938F931F930E94C1
:104C200078148091AC039091AD036DB77EB7695F46
:104C30007F4F0FB6F8947EBF0FBE6DBF069708F486
:104C400088C490914604992309F47DC48CE3809331
:104C50004104892F99279F938F938DE294E026CD6D
:104C6000109241048EED96E09F938F9311E01F9375
:104C70000E94781484E1809341040F900F900F906C
:104C80008091920399279F938F9386EE96E09F934E
:104C90008F931F930E94781488E2809341040F90B1
:104CA0000F900F900F900F908091F7039091F80361
:104CB0009F938F9384EF96E09F938F931F930E940F
:104CC00078148CE3809341040F900F900F900F9015
:104CD0000F908091080999279F938F9380910709DE
:104CE00099279F938F9382E097E04DCE10924104D5
:104CF00080E597E09F938F9311E01F930E947814B3
:104D000084E1809341040F900F900F90809186086A
:104D100099279F938F938091850899279F938F93CD
:104D20008091840899279F938F9380918308992776
:104D30009F938F9380E697E09F938F931F930E949A
:104D4000781488E2809341048DB79EB70B960FB616
:104D5000F8949EBF0FBE8DBF80918A0899279F93BC
:104D60008F938091890899279F938F9380918808CA
:104D700099279F938F938091870899279F938F936B
:104D800085E797E09F938F931F930E9478148CE39D
:104D9000809341042DB73EB7255F3F4F0FB6F8947F
:104DA0003EBF0FBE2DBF80918E0899279F938F9392
:104DB00080918D0899279F938F9380918C089927D4
:104DC0009F938F9380918B0899279F938F938AE865
:104DD00097E09F938F931F930E9478146DB77EB7CF
:104DE000655F7F4FD9CD109241048AE096E09F9392
:104DF0008F9311E01F930E94781484E18093410403
:104E00000F900F900F9080913705909138059F93E8
:104E10008F9380911A0490911B049F938F9387E145
:104E200096E09F938F931F930E94781488E280935B
:104E300041046DB77EB7695F7F4F0FB6F8947EBFB0
:104E40000FBE6DBF80913505909136059F938F936E
:104E500080911C0490911D049F938F9386E296E0AD
:104E60009F938F931F930E9478148CE38093410447
:104E70008DB79EB707960FB6F8949EBF0FBE8DBF35
:104E800080912F0590913005A0913105B0913205A8
:104E9000BC01CD010E94216BDC01CB019F938F935C
:104EA00080915F09909160099F938F9385E396E0CD
:104EB0009F938F931F930E9478142DB73EB7295F5D
:104EC0003F4F0FB6F8943EBF0FBE2DBF6AC310927E
:104ED00041048AE595E09F938F93C1E0CF930E94B0
:104EE0007814809102010F900F900F908A3009F48E
:104EF000A5C28B3009F4DEC1843109F4DBC18D30E9
:104F000009F04FC384E18093410480911C039927E9
:104F10009F938F934091410550914205CA0157FDDF
:104F200039C3959587959595879595958795959589
:104F300087959F938F939A0157FD29C335952795A0
:104F400035952795359527958091220490912304D6
:104F5000821B930B9F938F938EEC95E09F938F937F
:104F6000CF930E94781488E2809341046DB77EB796
:104F7000675F7F4F0FB6F8947EBF0FBE6DBF809105
:104F80001B0399279F938F9340913F0550914005B4
:104F9000CA0157FD04C39595879595958795959575
:104FA0008795959587959F938F939A0157FDF4C2A6
:104FB000359527953595279535952795809120042A
:104FC00090912104821B930B9F938F9382EE95E027
:104FD0009F938F93CF930E9478148CE38093410426
:104FE0008DB79EB709960FB6F8949EBF0FBE8DBFC2
:104FF00080911A0399279F938F9320913D053091BB
:105000003E05C90137FDC1C2959587959F938F9342
:1050100080911E0490911F04281B390B3F932F93FE
:1050200086EF95E09F938F93CF930E9478142DB7CE
:105030003EB7275F3F4F45CF109241048091E50472
:105040009091E6049F938F938EEA96E09F938F93BF
:1050500011E01F930E94781484E1809341040F9023
:105060000F900F900F900F908091E3049091E404C3
:105070009F938F938AEB96E09F938F931F930E9449
:10508000781488E2809341040F900F900F900F9056
:105090000F908091E1049091E2049F938F9386ECAE
:1050A00096E09F938F931F930E9478148CE38093D4
:1050B00041040F900F900F900F900F908091DF049C
:1050C0009091E0049F938F9382ED96E0EFCA109247
:1050D00041048FE997E09F938F93C1E0CF930E94A3
:1050E000781484E1809341040F900F900F90809189
:1050F000A20899278D969F938F938091A108992755
:105100008D969F938F938091A00899278D969F935A
:105110008F9380919F0899278D969F938F938EEA06
:1051200097E09F938F93CF930E94781488E28093A7
:1051300041048DB79EB70B960FB6F8949EBF0FBE75
:105140008DBF8091A60899278D969F938F9380910C
:10515000A50899278D969F938F938091A4089927EE
:105160008D969F938F938091A30899278D969F93F7
:105170008F9382EC97E09F938F93CF930E94781444
:105180008CE3809341042DB73EB7255F3F4F0FB6A8
:10519000F8943EBF0FBE2DBF8091A70899278D962A
:1051A0009F938F9386ED97E09F938F93CF930E9469
:1051B00078140F900F900F900F900F908091A80887
:1051C000882309F02DC18091A908882309F01AC10C
:1051D0008091AA08882309F4E4C188E480934104FB
:1051E0008CEE97E09F938F93CF9364CC81509C4F2C
:1051F000AF4FBF4FCFC981509C4FAF4FBF4FA3C9D7
:10520000109241048FEE97E09F938F9311E01F93CC
:105210000E94781484E1809341040F900F900F90C6
:105220008091D8039091D9039F938F938DEF97E04E
:105230009F938F931F930E94781488E28093410478
:105240000F900F900F900F900F908091D603909138
:10525000D7039F938F938AE098E09F938F931F9338
:105260000E94781489E4809341040F900F900F906E
:105270000F900F9087E198E09F938F931F930E9468
:10528000781480913F040F900F900F9083FF89C195
:105290001092D9031092D803AEE0B0E080E0082E5F
:1052A0000E94546CAFE0B0E08091D803082E0E94B9
:1052B000546C77C184E18093410440914105509141
:1052C0004205CA0157FD57C19C0135952795359573
:1052D00027953595279535952795C90182959295FE
:1052E000907F9827807F9827BA01681B790BCB01A4
:1052F00077FD3FC1959587959F938F933F932F930C
:105300009A0157FD33C135952795359527953595E4
:1053100027958091220490912304821B930B9F93E5
:105320008F938BE995E09F938F93CF930E9478148E
:1053300088E2809341048DB79EB709960FB6F89422
:105340009EBF0FBE8DBF40913F0550914005CA01E1
:1053500057FD0AC19C0135952795359527953595BB
:10536000279535952795C90182959295907F982725
:10537000807F9827BA01681B790BCB0177FDF2C0BB
:10538000959587959F938F933F932F939A0157FD00
:10539000E6C03595279535952795359527958091C4
:1053A000200490912104821B930B9F938F938DEA8D
:1053B00095E09F938F93CF930E9478148CE3809312
:1053C00041048DB79EB709960FB6F8949EBF0FBEE5
:1053D0008DBF20913D0530913E05C90137FDCDC0FF
:1053E000959587959F938F9380911E0490911F04AC
:1053F000281B390B3F932F938FEB95E09F938F934F
:10540000CF9359CD84E48093410489EE97E09F9334
:105410008F93CF930E9478140F900F900F90D8CE57
:1054200080E48093410486EE97E09F938F93CF931F
:105430000E9478140F900F900F90C5CE84E1809356
:10544000410440914105509142059A0157FD9AC08F
:10545000359527953595279535952795C901880F59
:10546000991F880F991F880F991F481B590B5F932D
:105470004F933F932F938091220490912304821B9A
:10548000930B9F938F9388E695E09F938F93CF9391
:105490000E94781488E2809341042DB73EB7275FBD
:1054A0003F4F0FB6F8943EBF0FBE2DBF40913F0552
:1054B000509140059A0157FD62C035952795359565
:1054C000279535952795C901880F991F880F991F32
:1054D000880F991F481B590B5F934F933F932F934E
:1054E0008091200490912104821B930B9F938F93B2
:1054F0008AE795E09F938F93CF930E9478148CE373
:10550000809341046DB77EB7675F7F4F0FB6F89405
:105510007EBF0FBE6DBF80913D0590913E059F936C
:105520008F9380913D0590913E0520911E0430910E
:105530001F04821B930B9F938F938CE895E09F939E
:105540008F93CF936EC98CE38093410482E494E0FF
:10555000AECA8CE38093410480E294E0A8CA295F3C
:105560003F4F17CF01960CCF0F96F4CE295F3F4FD8
:10557000CACE0196BFCE0F96A7CE019631CF295F36
:105580003F4F9BCF295F3F4F63CF01963DCD295FB2
:105590003F4FD4CC0F96C5CC295F3F4F09CD0F9616
:1055A000FACC10923F04DF91CF911F910895109291
:1055B000B9008AE28093B800089585EA8093BC0020
:1055C000089584E98093BC0008951092B9008093F7
:1055D000BB0085E88093BC0008950E94E12A1092E8
:1055E00049048091BB001092480480E88093BC007D
:1055F0001092BD001092BA001092BB001092B90038
:105600001092B8000E94D72A0E94DD2A80E00E94F2
:10561000E52A08958093BB0085E88093BC00089537
:1056200085EC8093BC00089585E88093BC000895C4
:105630001F920F920FB60F9211242F933F934F9307
:105640005F936F937F938F939F93AF93BF93EF93EA
:10565000FF9380914904282F3327442755278F5FD4
:1056600080934904F90127313105C8F4E05BFF4F0D
:10567000EE0FFF1F0590F491E02D099480914704EF
:10568000E82FFF27ED58F74F9091BB0090838F5F75
:105690008C3008F49DC0109247040E94E12A1092B9
:1056A0004904E0C080E80E94E52ADCC088E90E9445
:1056B000E52AD8C00E94E12A8AE090E09093AD03E9
:1056C0008093AC030E94DD2ACDC084E10E94E52ACC
:1056D000C9C082E10E94E52AC5C080911C030E94D6
:1056E000E52AC0C080E10E94E52ABCC080911B036E
:1056F0000E94E52AB7C080911A030E94E52AB2C031
:1057000080914804E82FFF27ED56F64F8F5F809376
:10571000480480810E94E52AA5C090914804292F61
:10572000E92FFF27EE0FFF1FEE0FFF1FE053FA4F89
:10573000858518160CF054C09C3009F467C0990F89
:10574000892F8E5A0E94E52A8DC080914704E82F48
:10575000FF27E157F74F8091BB0080830E94142BF5
:1057600081C08091B900803409F46EC080914704F3
:10577000E82FFF27E156F74F10828F5F8C3068F1DA
:10578000109247040E94E12A1092490480914A0431
:105790008093460410924A0465C08091B90080331A
:1057A00009F440C00E94E12A8AE090E09093AD03A2
:1057B0008093AC03109249040E94DD2A53C00E94DA
:1057C000E12A8AE090E09093AD038093AC0367CF29
:1057D000809347040E94E12A62CF80934704D2CF8E
:1057E0009C3008F0A9CF922F9F5FE92FFF27EE0F83
:1057F000FF1FEE0FFF1FE053FA4F858518161CF0B0
:10580000292F9C3080F39093480496CF109248043F
:1058100083E08093490480914704880F8D5A0E9449
:10582000E52A20C080914A048823C9F49091480455
:1058300090934A04E92FFF27EE57F74F80818F5F3F
:1058400009F48FEF8083AECF80914704E82FFF27C4
:10585000E156F74F8C5F80830E94102B97CF909179
:105860004804E8CF8091BC0080688093BC00FF9121
:10587000EF91BF91AF919F918F917F916F915F91C8
:105880004F913F912F910F900FBE0F901F90189541
:1058900083EC8093810080916F00806280936F0021
:1058A00010923E0510923D051092400510923F0562
:1058B000109242051092410508951F920F920FB663
:1058C0000F921124EF92FF920F931F932F933F9308
:1058D0004F935F936F937F938F939F93AF93BF93F8
:1058E000CF93DF93EF93FF938091360982FD2CC015
:1058F000209186003091870080914C0490914D0456
:10590000281B390B809186009091870090934D045D
:1059100080934C04C9018D549440835F9A4108F0F0
:10592000B5C080914E048093AB0880914E04909155
:105930004F04049714F010928403C1E0D0E0D09398
:105940004F04C0934E0415C24091860050918700C9
:105950008091500490915104481B590B809186000E
:10596000909187009093510480935004CA018D5404
:105970009440835F9A4138F58091AA0480934B0448
:1059800080914B04843008F00EC18091AB048536C1
:1059900008F47BC18AE08093AB04809102018A30D5
:1059A00009F476C1843109F473C1289881E08093A9
:1059B000AA048091D404882309F0DBC180914B04B0
:1059C0008093AB08D6C10091AA040A3008F0E4C065
:1059D000CA018B5F9040845B914008F05BC1425DDF
:1059E0005140E02FFF27EE0FFF1FEE5AFB4F808143
:1059F0009181FA01E81BF90BCF0105960B9708F48A
:105A00005CC1E02FFF27EE0FFF1FEE5AFB4F808196
:105A100091819C01220F331F280F391F240F351F3E
:105A200037FDA4C1E901D595C795D595C795CA019C
:105A300001968C179D070CF071C121978091DE04AF
:105A40008E3B08F462C1E02FFF27EE0FFF1FDF013E
:105A5000AE5ABB4F8D919C919E01281B390BC901F9
:105A600063E070E00E94F76BCB01880F991F860FEF
:105A7000971FE859FB4F91838083E02FFF27EE0F9C
:105A8000FF1FEE5AFB4FD183C0830BC1C0914E0460
:105A9000D0914F04CA30D1050CF06BC1C9018B5FA6
:105AA0009040845B914008F060C0225D3140FE016F
:105AB000EC0FFD1FE455F74F80819181D901A81BA0
:105AC000B90BCD01B7FD0EC1069754F48091DE04E9
:105AD000883C08F046C18091DE04865F8093DE0436
:105AE000FE01EC0FFD1FE455F74F80819181AC0161
:105AF000440F551F480F591F420F531F57FD33C105
:105B00007A01F594E794F594E794C90101968E150E
:105B10009F050CF013C10894E108F1088091DE04A0
:105B2000833C08F403C18E010C0F1D1FF801E455DE
:105B3000F74F80819181F701E81BF90BCF0163E0FA
:105B400070E00E94F76BCB01880F991F860F971F9B
:105B50000E53174FD80111969C938E93FE01EC0FB4
:105B6000FD1FE455F74FF182E082FE013196F0937C
:105B70004F04E0934E04E530F10509F4B9C05D9897
:105B8000E630F10509F4BFC05C98379709F4B9C055
:105B90005B98EFC05C9A5B98043108F054C00F5FCB
:105BA0000093AA04E6C09091AB0880914B0498172B
:105BB00009F0EBCE4091AB044B3008F49BC010923F
:105BC00084031092AA043AC00091AA04E02FFF2790
:105BD000EE0FFF1F9F0122583B4FDF01A455B74F27
:105BE0008D919C91D9018D939C93DF01AE53B74F5A
:105BF0008D919C91EC56FB4F91838083E02FFF2782
:105C0000EE0FFF1F9F012455374FDF01AE5ABB4FE8
:105C10008D919C91D90111969C938E93DF01A85987
:105C2000BB4F8D919C91EE53F74F91838083E02F72
:105C3000EF5FEB3008F05EC0E093AA044F3120F62E
:105C40000091AA04DBCF043109F093C080910201D6
:105C50008A3009F47DC0843109F47AC028988EE135
:105C60008093AA042AE0C2ECD8E0AEE7B4E0ECEA04
:105C7000F8E08D919D9191838083329619821882EC
:105C80002296215027FFF5CF74C01092AB0485CE29
:105C9000289A8CCE809102018A3011F1843101F171
:105CA0002898053019F15D98063009F473CF5C9897
:105CB000073009F070CF5B9A72CF8091AB048A31C4
:105CC00008F448C08091DE04865F8093DE048091F2
:105CD000DE04893C08F495CE88EC8093DE0491CEF6
:105CE000289ADFCF909581959F4FEECE5D9ADFCFBA
:105CF0005D9A46CF4F3F09F459CE4F5F4093AB04B6
:105D000055CE5B9A36C05C9A40CFE02FFF27EE0F4E
:105D1000FF1FE859FB4F11821082AFCE4150504017
:105D2000C417D5070CF08ACE219688CEFE01EC0F61
:105D3000FD1FEE53F74F1182108210CF21503040DB
:105D4000E216F3060CF0EACE0894E11CF11CE6CE54
:105D5000289A85CF8B3008F4BACF8091DE048E5F0D
:105D6000B4CF88ECBBCE4D5F5F4FCACE2D5F3F4FA7
:105D700059CEFF91EF91DF91CF91BF91AF919F915C
:105D80008F917F916F915F914F913F912F911F91D3
:105D90000F91FF90EF900F900FBE0F901F901895EE
:105DA00081E08093E00882E08093DF0883E08093C5
:105DB000DE0884E08093E10885E08093E20886E0D5
:105DC0008093E30887E08093E40888E08093E50807
:105DD00008951F938AE68093E60851E050933609B0
:105DE0004EE14093E7088BEF8093E9088AE08093C7
:105DF000EA084093E8084093EC0885E08093ED08BA
:105E000080E48093EE081092EF0884E18093EB0821
:105E10008EE08093F008E0E1E093F1081CE010933D
:105E2000F208F8E0F093F30886EE8093F4084093CC
:105E3000F50880E88093F60830E53093F70896E996
:105E40009093F80883E08093F9083093FA089093D0
:105E5000FB0881E28093FC0883E28093FD08409375
:105E6000FE081092FF0860E2609300091092010999
:105E70001092020910920309109204091092190954
:105E800010921A0910921B0910921C0924E6209303
:105E9000050998E290930609509335091092070975
:105EA0008AEF8093080976E070930D092093090921
:105EB00090930A0910920B0980930C0982E3809356
:105EC0000E099AE590930F098093100910923409F6
:105ED00090931109309312095093130985E580932B
:105EE000140980931509E09316096093170920930C
:105EF00018098FE580931D0983EF80931F098AEAB3
:105F000080932109809322098FE080931E0980935A
:105F100020098CEF8093230920932409909325096D
:105F200090932609909327098BE480932809809306
:105F3000290980932A0910922B0970932C09F09358
:105F40002D0990932E0940932F0920933009209317
:105F5000310984E080933209AEEAB3E0E7E3F9E087
:105F60000D9001921A95E1F71F9108958AE68093AA
:105F7000E60871E0709336095EE15093E7088BEF15
:105F80008093E9089AE09093EA085093E8085093C8
:105F9000EC0885E08093ED0880E48093EE08109291
:105FA000EF088FE08093EB089093F00880E18093F6
:105FB000F10866E06093F208E8E0E093F30886EE0B
:105FC0008093F4085093F50880E88093F6082AE55A
:105FD0002093F70898E79093F80883E08093F908F6
:105FE0002093FA089093FB0881E28093FC0883E2F7
:105FF0008093FD085093FE081092FF0840E2409302
:1060000000091092010910920209109203091092DE
:1060100004091092190910921A0910921B09109282
:106020001C0934E63093050998E2909306097093B1
:106030003509109207098AEF8093080960930D09CA
:106040003093090990930A0910920B0980930C0967
:1060500082E380930E0920930F0980931009109218
:1060600034092093110980E5809312098CE3809311
:10607000130985E580931409809315094093160947
:10608000409317099BE4909318098FE580931D09AD
:1060900083EF80931F098AEA809321098093220964
:1060A00084E180931E09809320098CEF809323095B
:1060B000309324092093250920932609209327094A
:1060C000909328099093290990932A0910922B09FB
:1060D00060932C09E0932D0920932E0950932F09EA
:1060E000309330093093310984E0809332098CE099
:1060F000A5EBB3E0E7E3F9E00D9001928A95E1F7B3
:1061000008958AE68093E60871E0709336094EE1BF
:106110004093E7088BEF8093E9088AE08093EA08D0
:106120004093E8084093EC0885E08093ED0880E414
:106130008093EE081092EF088FE08093EB0868E000
:106140006093F00820E12093F10856E05093F208A4
:106150006093F30886EE8093F4084093F50880E896
:106160008093F60834E63093F70898E79093F808A0
:1061700083E08093F9083093FA089093FB0881E25A
:106180008093FC0883E28093FD0884E18093FE08FD
:106190001092FF0820930009109201091092020941
:1061A00010920309109204091092190910921A0909
:1061B00010921B0910921C093093050998E29093E4
:1061C000060970933509109207098AEF8093080930
:1061D00050930D093093090990930A0910920B0905
:1061E00080930C0992E390930E092AE520930F09FE
:1061F00090931009109234092093110980E580933F
:10620000120986E48093130985E58093140980932D
:10621000150980E280931609809317099093180955
:106220008FE580931D0983EF80931F098AEA80938D
:1062300021098093220940931E09409320098CEF85
:10624000809323093093240920932509209326095C
:10625000209327098BE48093280980932909809350
:106260002A0910922B0950932C0960932D09209331
:106270002E0940932F09309330093093310984E07F
:10628000809332098CE0ADEBB3E0E7E3F9E00D90E9
:1062900001928A95E1F708956817790744F4680F29
:1062A000791F77FD09C0CB01959587950895681BE7
:1062B000790B861B970B08956F5F7F4FCB019595E8
:1062C00087950895EF92FF920F931F93CF93C82F56
:1062D0008B018091D4048823A9F4C150CF3F91F061
:1062E0007B01E60EF71E1093FC030093FB038091E5
:1062F000FB039091FC03892BD1F7C7010E940C1876
:10630000C15088F7CF911F910F91FF90EF900895A2
:106310002F923F924F925F926F927F928F929F92B5
:10632000AF92BF92CF92DF92EF92FF920F931F93A3
:10633000CF93DF93CDB7DEB7ED970FB6F894DEBFFE
:106340000FBECDBF20913D0530913E0580911E04CA
:1063500090911F04281B390B3A8729873093A20993
:106360002093A109209128043091290437FDD4C736
:106370003595279535952795359527953AA729A7DA
:106380003C872B877901209126043091270437FD23
:10639000C0C73595279535952795359527953CA701
:1063A0002BA73E872D87F0926209E0926109309316
:1063B0005809209357098091900990919109AA2733
:1063C00097FDA095BA2F7C018D01EE0CFF1C001FDC
:1063D000111FE80EF91E0A1F1B1F80911A049091CD
:1063E0001B049C01442737FD4095542FDA01C90155
:1063F000880F991FAA1FBB1F880F991FAA1FBB1FB9
:10640000820F931FA41FB51F820F931FA41FB51FD8
:10641000E80EF91E0A1F1B1F17FD9CC7159507954F
:10642000F794E79415950795F794E794F0929109FE
:10643000E09290098091AC099091AD09AA2797FD4F
:10644000A095BA2F7C018D01EE0CFF1C001F111FBF
:10645000E80EF91E0A1F1B1F80911C0490911D0459
:106460009C01442737FD4095542FDA01C901880F5C
:10647000991FAA1FBB1F880F991FAA1FBB1F820F3E
:10648000931FA41FB51F820F931FA41FB51FE80EF3
:10649000F91E0A1F1B1F17FD54C715950795F79482
:1064A000E79415950795F794E794F092AD09E0927B
:1064B000AC0980915F0990916009AA2797FDA0958A
:1064C000BA2F9C01AD01220F331F441F551F280F07
:1064D000391F4A1F5B1F8091180490911904AA2745
:1064E00097FDA095BA2F280F391F4A1F5B1F57FD34
:1064F00016C75595479537952795559547953795DF
:1065000027953093600920935F0920911A043091F8
:106510001B04C901880F991F880F991F820F931FB1
:10652000820F931FAA2797FDA095BA2F20911905D6
:1065300030911A0540911B0550911C05820F931F45
:10654000A41FB51F8093190590931A05A0931B05EE
:10655000B0931C0520911C0430911D04C901880FC3
:10656000991F880F991F820F931F820F931FAA27CD
:1065700097FDA095BA2F20911505309116054091F1
:10658000170550911805820F931FA41FB51F809304
:10659000150590931605A0931705B09318058091E3
:1065A0006A0990916B0920911A0430911B04820FA3
:1065B000931F90936B0980936A098091A40990912D
:1065C000A50920911C0430911D04820F931F909304
:1065D000A5098093A4098091330590913405019613
:1065E00090933405809333058091110590911205A5
:1065F000A0911305B0911405BC01CD010E943E6B22
:106600005B016C018091660890916708AA2797FD4D
:10661000A095BA2FBC01CD010E943E6B7B018C017D
:1066200080912F0590913005A0913105B0913205F0
:106630009C01AD01C801B7010E94DE6ADC01CB01FB
:106640009C01AD01C601B5010E94DF6ADC01CB01EE
:10665000BC01CD010E94216BDC01CB0180931105AF
:1066600090931205A0931305B09314058FEC8093BB
:106670007A00109219032090010530900205409095
:1066800003055090040539E423163BE6330631E058
:10669000430630E053060CF414C188E49BE6A1E005
:1066A000B0E08D839E83AF83B887609009057090BA
:1066B0000A0580900B0590900C0539E463163BE6C3
:1066C000730631E0830630E093060CF4DCC488E402
:1066D0009BE6A1E0B0E089839A83AB83BC834985C4
:1066E0005A85CA01AA2797FDA095BA2F2091F904CF
:1066F0003091FA044091FB045091FC04280F391F9B
:106700004A1F5B1F2DA33EA34FA358A7A090A80923
:10671000B090A909C090AA09D090AB09A80EB91EE3
:10672000CA1EDB1E860175013091C7043BA33323CB
:1067300009F0DAC08091C604882309F0C2C44091F0
:10674000E6084CA346FF13C6EBA5FCA5CF01AA277C
:1067500097FDA095BA2FBC01CD0129813A814B81CB
:106760005C810E94B86B9B01AC0197FD2CC7BBE01C
:106770005595479537952795BA95D1F780918E0312
:10678000E82EFF2400271127C801B7010E94B86B2B
:1067900097FD14C7ACE09595879577956795AA9571
:1067A000D1F76F87788B898B9A8B60934D057093A7
:1067B0004E0580934F059093500529A53AA5C90130
:1067C000AA2797FDA095BA2FBC01CD012D813E814E
:1067D0004F8158850E94B86B9B01AC0197FD01C7A2
:1067E000FBE05595479537952795FA95D1F7C80160
:1067F000B7010E94B86B97FDEFC6DC01CB01ECE05E
:10680000B595A79597958795EA95D1F7809351050A
:1068100090935205A0935305B093540520914D05D4
:1068200030914E053093D9082093D8082091510516
:10683000309152053093DD082093DC082F8538898C
:1068400049895A89821B930BA40BB50B8AAF9BAF66
:10685000ACAFBDAF8093510590935205A093530503
:10686000B0935405A80EB91ECA1EDB1E8601750121
:1068700030918D033DA7332309F0A3C58EA79FA7B1
:10688000A8ABB9ABB7FD61C62EA53FA548A959A9CC
:1068900055954795379527958DA19EA1AFA1B8A590
:1068A000821B930BA40BB50B8DA39EA3AFA3B8A71C
:1068B0008093F9049093FA04A093FB04B093FC0432
:1068C0008CC598EB291694E939069EEF49069FEF8F
:1068D00059060CF0F1C328EB34E94EEF5FEF2D833E
:1068E0003E834F835887E1CE2DA13EA14FA158A5ED
:1068F0002093F9043093FA044093FB045093FC0472
:106900003091E6083CA31092DD081092DC0810924A
:10691000D9081092D8081092490510924A05109291
:106920004B0510924C0510924505109246051092A9
:1069300047051092480530918D033DA78091490588
:1069400090914A05A0914B05B0914C05BC01CD0139
:1069500024E630E040E050E00E942C6CDA01C901EE
:106960004091450550914605481B590B58A34F8F40
:106970008091450590914605A0914705B091480545
:10698000BC01CD0124E630E040E050E00E942C6CD8
:10699000DA01C9012091490530914A05821B930B08
:1069A0009AA389A38091860390918703A09188037D
:1069B000B0918903BC01CD0128E631E040E050E010
:1069C0000E94B86BE616F7060807190744F057014E
:1069D0006801A61AB70AC80AD90A8601750117FD07
:1069E000A3C4A092A809B092A909C092AA09D09202
:1069F000AB092BA53CA58F8D98A1280F391F7901D4
:106A00000027F7FC0095102F8091FD049091FE0463
:106A1000A091FF04B0910005E80EF91E0A1F1B1F8C
:106A2000570168018091CA049091CB04281B390B4F
:106A3000C901AA2797FDA095BA2F280E391E4A1E14
:106A40005B1E2091A2033091A3034091A4035091B7
:106A5000A503221533054405550574F4A8EAEA2E6A
:106A6000A1E6FA2E012D112DE21AF30A040B150BE3
:106A7000170128015701680188279927DC01821B2B
:106A8000930BA40BB50B281639064A065B060CF0CF
:106A9000E9C2F8E52F2EFEE93F2EFFEF4F2EFFEF64
:106AA0005F2E220E331E441E551E20920105309289
:106AB0000205409203055092040582017101209263
:106AC000FD043092FE044092FF045092000529A577
:106AD0003AA5A9A1BAA12A0F3B1FA901662757FD14
:106AE0006095762F8091050590910605A091070588
:106AF000B0910805480F591F6A1F7B1F5A016B018F
:106B00008091C8049091C904281B390BC901AA2798
:106B100097FDA095BA2F680E791E8A1E9B1E809144
:106B2000A6039091A703A091A803B091A9038EABEF
:106B30009FABA8AFB9AF86159705A805B90564F452
:106B400048EA51E660E070E0481B590B6A0B7B0B8A
:106B50003A014B015A016B018EA99FA9A8ADB9ADAD
:106B6000B095A095909581959F4FAF4FBF4F6816F8
:106B700079068A069B060CF064C2E8E56E2EEEE903
:106B80007E2EEFEF8E2EEFEF9E2E2EA93FA948AD61
:106B900059AD620E731E841E951E60920905709297
:106BA0000A0580920B0590920C05B401A301609236
:106BB00005057092060580920705909208058DA143
:106BC0009EA1AFA1B8A580930D0590930E05A0934B
:106BD0000F05B09310056092290570922A058092E6
:106BE0002B0590922C05209221053092220540928F
:106BF0002305509224054093250550932605609364
:106C0000270570932805E0921D05F0921E0500935C
:106C10001F0510932005809125039091260397FD71
:106C2000A4C37C01F594E794F594E794F594E79474
:106C3000FAA6E9A6809123039091240397FD93C3BC
:106C40008C011595079515950795159507951CA722
:106C50000BA780912204909123040F9734F458E1FC
:106C6000E52E5CEFF52EFAA6E9A68091220490911C
:106C70002304079734F440E3E42E48EFF42EFAA6F9
:106C8000E9A6209102012A3009F46BC28091220406
:106C900090912304815D97400CF007C280912204FB
:106CA00090912304805E974034F080EDE82E87E0D9
:106CB000F82EFAA6E9A680912004909121040F975E
:106CC00024F408E11CEF1CA70BA7809120049091ED
:106CD0002104079724F400E318EF1CA70BA72A3020
:106CE00009F455C28091200490912104815D974060
:106CF00024F008EE13E01CA70BA7809120049091CC
:106D00002104805E974024F000ED17E01CA70BA73C
:106D1000A0919903AA2309F497C06091250370916B
:106D200026038091550590915605681B790B20919B
:106D3000250330912603280F391F37FD3FC33595B2
:106D400027953093560520935505613871050CF44D
:106D50003AC260E870E070935C0560935B058A2F2F
:106D60009927869FF001879FF00D969FF00D1124C3
:106D7000CF01F7FD21C37C01F594E794F594E794E6
:106D8000F594E794F594E79429A53AA5E20EF31E4D
:106D9000FAA6E9A640912303509124038091570558
:106DA00090915805481B590B2091230330912403DF
:106DB000280F391F37FDFDC23595279530935805AB
:106DC00020935705413851050CF4F5C140E850E0D7
:106DD00050935A05409359058A2F9927849FD001D3
:106DE000859FB00D949FB00D1124AD019D01B7FD9D
:106DF000DDC2890115950795159507951595079598
:106E000015950795EBA5FCA50E0F1F1F1CA70BA73B
:106E1000869F9001879F300D969F300D1124C901E8
:106E20002091250330912603820F931F9093260310
:106E3000809325038091230390912403480F591FC9
:106E400050932403409323034D855E851416150645
:106E50000CF0C1C18091D8089091D90897FDA2C2C9
:106E6000AA2797FDA095BA2F6DA5262F3327442773
:106E70005527BC01CD010E94B86B97FD8EC2E6E09C
:106E80009595879577956795EA95D1F7AF8DB8A1D8
:106E9000A60FB71FB0935309A09352094B855C8589
:106EA000141615060CF0C1C18091DC089091DD0824
:106EB00097FD6FC2AA2797FDA095BA2F6DA5262F23
:106EC000332744275527BC01CD010E94B86B97FD9D
:106ED0005BC246E095958795779567954A95D1F77A
:106EE000A9A1BAA1A60FB71FB0934809A09347095B
:106EF0003CA137FDC1C11093460900934509F092AA
:106F00005509E09254098091E208E82FFF27EE0F1F
:106F1000FF1FE455F74F8081918182599F4FA091C7
:106F2000E504B091E604A817B9070CF0EEC0CD0156
:106F300001969093E6048093E504DC018091E308D8
:106F4000E82FFF27EE0FFF1FE455F74F8081918157
:106F500082599F4F6091E3047091E40468177907A8
:106F60000CF0C4C0CB0101969093E4048093E30439
:106F7000BC018091E408E82FFF27EE0FFF1FE455C6
:106F8000F74F8081918182599F4F4091E104509148
:106F9000E204481759070CF0D5C0CA010196909336
:106FA000E2048093E104AC018091E508E82FFF271B
:106FB000EE0FFF1FE455F74F8081918182599F4F5B
:106FC0002091DF043091E004281739070CF0ABC0A2
:106FD000C90101969093E0048093DF049C01B7FD02
:106FE00093C1AF3FB10539F034F08FEF90E090934B
:106FF000E6048093E50477FD76C16F3F710539F0B3
:1070000034F08FEF90E09093E4048093E30457FD15
:1070100070C14F3F510539F034F08FEF90E09093FD
:10702000E2048093E10437FD6AC12F3F310509F086
:107030000CF4EEC28FEF90E09093E0048093DF04B5
:10704000E7C26092090570920A0580920B05909242
:107050000C05A0920505B0920605C0920705D092D6
:107060000805ADCD2092010530920205409203053E
:1070700050920405A092FD04B092FE04C092FF0459
:10708000D092000524CD98EB691694E979069EEF1D
:1070900089069FEF99062CF528EB34E94EEF5FEF58
:1070A00029833A834B835C831ACB98EEE92E93E0D5
:1070B000F92EFAA6E9A6F2CD2D823E824F8258869D
:1070C000F4CA8DA19EA1AFA1B8A58093F9049093B5
:1070D000FA04A093FB04B093FC049091E6089CA3EF
:1070E00012CC69827A828B829C82F9CA80819181DA
:1070F00082599F4F861797070CF03BCF611571059A
:1071000009F437CFCB0101972FCF8081918182592C
:107110009F4F8A179B070CF011CF109709F40ECFE1
:10712000CD01019706CF8081918182599F4F8217AF
:1071300093070CF054CF2115310509F450CFC90144
:10714000019748CF8081918182599F4F841795077D
:107150000CF02ACF4115510509F426CFCA01019739
:107160001ECF8091220490912304835F934034F0DA
:1071700038EEE32E33E0F32EFAA6E9A6809122043E
:10718000909123048A5F93400CF495CD8ECD80912D
:10719000200490912104835F934024F008EE13E0D3
:1071A0001CA70BA780912004909121048A5F934033
:1071B0000CF4AECDA9CD3FEF403853070CF008CE0C
:1071C00040E85FEF05CE8FEF603878070CF0C3CD55
:1071D00060E87FEFC0CD8091D8089091D90897FDE5
:1071E0009BC1AA2797FDA095BA2FEDA52E2F332777
:1071F00044275527BC01CD010E94B86B97FDADC156
:1072000056E095958795779567955A95D1F72F8D87
:1072100038A1261B370B30935309209352094B8515
:107220005C85141615060CF43FCE8091DC08909115
:10723000DD0897FD6DC1AA2797FDA095BA2FEDA592
:107240002E2F332744275527BC01CD010E94B86B50
:1072500097FD88C136E095958795779567953A951E
:10726000D1F729A13AA1261B370B30934809209367
:1072700047093CA137FF3FCE4BA1442309F03BCE49
:107280008091C604882309F036CE8B859C85A1E0C9
:1072900081309A070CF044C12B853C854FEF20309C
:1072A00034070CF0A3C189A59AA5280F391F3C8784
:1072B0002B8720503F4F3093550920935409AD85BB
:1072C000BE85E1E0A130BE070CF465C12BA53CA54D
:1072D000A20FB31FBE87AD87A050B140B09346093F
:1072E000A093450910CE1092E4041092E30457FFD6
:1072F00090CE1092E2041092E10437FF96CE1092E5
:10730000E0041092DF0484C11092E6041092E504B8
:1073100072CE295F3F4F3DC8295F3F4F29C82D5F7F
:107320003F4F4F4F5F4FE5C8E60EF71E081F191F6E
:10733000E092A809F092A9090093AA091093AB0959
:1073400058CB23E030E040E050E0E20EF31E041F93
:10735000151FA3C883E090E0A0E0B0E0E80EF91E9E
:107360000A1F1B1F5BC807966BCC07965ACC2DA132
:107370003EA14FA158A52093F9043093FA044093FD
:10738000FB045093FC04BFCA615C7F4F8F4F9F4F3B
:10739000A0CD909581959F4F8DCD615C7F4F8F4F94
:1073A0009F4F6DCD909581959F4F5ACD215F3F4F57
:1073B00020CD2F5F3F4F00CD0F96DDCC2F5F3F4F8D
:1073C000BECC2DA13EA14FA158A52093F904309326
:1073D000FA044093FB045093FC0489859A85AA27FC
:1073E00097FDA095BA2F2AAD3BAD4CAD5DAD820F98
:1073F000931FA41FB51F8B8B9C8BAD8BBE8BBC01C9
:10740000CD0129813A814B815C810E94B86B9B013F
:10741000AC0197FDBBC06BE0559547953795279517
:107420006A95D1F760918F03862F9927AA27BB27EA
:107430008F8B988FA98FBA8FBC01CD010E94B86B3A
:1074400097FD9FC02CE095958795779567952A9530
:10745000D1F76B8F7C8F8D8F9E8F609345057093D6
:10746000460580934705909348056B897C898D89F3
:107470009E892D813E814F8158850E94B86B9B016A
:10748000AC0197FD79C08BE05595479537952795C9
:107490008A95D1F76F89788D898D9A8D0E94B86B06
:1074A00097FD65C0BCE09595879577956795BA95EA
:1074B000D1F76AAB7BAB8CAB9DAB60934905709306
:1074C0004A0580934B0590934C0529853A8537FDF5
:1074D0007FC0213431050CF431CA6B8D7C8D8D8DCC
:1074E0009E8D97FD2AC0613871058105910564F470
:1074F0006AA97BA98CA99DA997FD82C061387105F5
:10750000810591050CF41ACA81E08093E90416CA3A
:10751000909581959F4F8FCE909581959F4F61CE8D
:10752000E9A5FAA58E0F9F1F9C878B8780509140FD
:107530009093550980935409C2CE9095809570958B
:1075400061957F4F8F4F9F4FCECF0196A11DB11DEB
:107550008EA79FA7A8ABB9AB97C9615C7F4F8F4F30
:107560009F4F4ECE615C7F4F8F4F9F4F73CE6150C8
:10757000704F8F4F9F4F96CF2150384F4F4F5F4FD7
:1075800082CF6150704F8F4F9F4F5CCF2150384F4B
:107590004F4F5F4F40CF4D855E856FEF40305607B0
:1075A00054F58BA59CA5480F591F5E874D87405009
:1075B0005F4F5093460940934509A5CC6150704FE9
:1075C0008F4F9F4FE7C82150384F4F4F5F4FCFC865
:1075D000309521953F4F7DCF6150704F8F4F9F4F1A
:1075E0000CC92150384F4F4F5F4FFAC8F0925509E0
:1075F000E092540964CE109346090093450983CC68
:1076000090958095709561957F4F8F4F9F4F76CF66
:10761000ED960FB6F894DEBF0FBECDBFDF91CF91D0
:107620001F910F91FF90EF90DF90CF90BF90AF90A0
:107630009F908F907F906F905F904F903F902F9092
:107640000895809102018D3009F455C110927A009D
:1076500080912204909123049093550980935409BA
:1076600080912004909121049093460980934509CC
:1076700080911E0490911F049093A2098093A10908
:1076800080911A0490911B049C01442737FD40957A
:10769000542FDA01C901880F991FAA1FBB1F880F39
:1076A000991FAA1FBB1F820F931FA41FB51F820F14
:1076B000931FA41FB51F9093910980939009809107
:1076C0001C0490911D049C01442737FD4095542FC4
:1076D000DA01C901880F991FAA1FBB1F880F991FC4
:1076E000AA1FBB1F820F931FA41FB51F820F931FDA
:1076F000A41FB51F9093AD098093AC098091180425
:10770000909119049093600980935F098FEC8093A6
:107710007A008091E208E82FFF27EE0FFF1FE45563
:10772000F74F8081918182599F4FA091E504B091DC
:10773000E604A817B9070CF085C0CD010196909317
:10774000E6048093E504DC018091E308E82FFF273D
:10775000EE0FFF1FE455F74F8081918182599F4FB3
:107760006091E3047091E404681779070CF096C007
:10777000CB0101969093E4048093E304BC018091D3
:10778000E408E82FFF27EE0FFF1FE455F74F808135
:10779000918182599F4F4091E1045091E204481732
:1077A00059070CF06CC0CA0101969093E2048093D3
:1077B000E104AC018091E508E82FFF27EE0FFF1FE1
:1077C000E455F74F8081918182599F4F2091DF04CA
:1077D0003091E004281739070CF042C0C901019626
:1077E0009093E0048093DF049C01B7FD7FC0AF3F1E
:1077F000B10511F00CF061C077FD67C06F3F7105F6
:1078000039F034F08FEF90E09093E4048093E30438
:1078100057FD61C04F3F510539F034F08FEF90E0D4
:107820009093E2048093E10437FD5BC02F3F310564
:1078300009F00CF463C08FEF90E09093E004809324
:10784000DF045CC08081918182599F4F8A179B071A
:107850000CF07ACF109709F477CFCD0101976FCF55
:107860008081918182599F4F821793070CF0BDCF81
:107870002115310509F4B9CFC9010197B1CF808134
:10788000918182599F4F841795070CF093CF411532
:10789000510509F48FCFCA01019787CF808191816B
:1078A00082599F4F861797070CF069CF61157105B4
:1078B00009F465CFCB0101975DCF8FEF90E09093F6
:1078C000E6048093E50477FF99CF1092E4041092C8
:1078D000E30457FF9FCF1092E2041092E10437FFB8
:1078E000A5CF1092E0041092DF0408C01092E604C5
:1078F0001092E50481CF0E94B31CA8CE8091140998
:107900009927AA27BB27BC01CD0124EC39E040E030
:1079100050E00E94B86BDC01CB018093A6039093EA
:10792000A703A093A803B093A903809115099927F1
:10793000AA27BB27BC01CD010E94B86BDC01CB019B
:107940008093A2039093A303A093A403B093A503F1
:1079500008956F927F928F929F92AF92BF92CF9233
:10796000DF92EF92FF920F931F93CF9300E010E00E
:1079700078016801469A10933805009337051093F3
:1079800036050093350580E090E0A0E0B0E08093FC
:107990002F0590933005A0933105B09332051093D5
:1079A0004205009341051093400500933F05109355
:1079B0003E0500933D0510937209009371091092E2
:1079C0008F0310928E03109212040E94213B84E6D2
:1079D00090E00E9419180E94213B8091E60880FFE8
:1079E00010C080911D0390911E03875B934008F0A7
:1079F000FBC180911D0390911E038E5E924008F49E
:107A0000F3C1CFE18AE090E00E94191880911E0432
:107A100090911F04080F191F809122049091230454
:107A2000E80EF91E8091200490912104C80ED91E01
:107A3000C150C7FFE7CFA701405F5F4F56954795FD
:107A40005695479550934205409341059601205F16
:107A50003F4F3695279536952795309340052093CF
:107A60003F05C801409696958795929582958F70AF
:107A700089279F70892790933E0580933D059093B9
:107A800072098093710930933C0520933B05509314
:107A90003A054093390544E050E0DA010E94476C12
:107AA000802D853008F4A3C18091AC099091AD0977
:107AB00097FDD2C16CE070E00E94F76B70933605C1
:107AC00060933505809190099091910997FDD5C1FA
:107AD0006CE070E00E94F76B709338056093370597
:107AE0008091660890916708AA2797FDA095BA2F04
:107AF000BC01CD010E943E6BDC01CB0180932F05C0
:107B000090933005A0933105B0933205109255093A
:107B10001092540910924609109245091092A20938
:107B20001092A10984E690E00E94191880911A042D
:107B300090911B04AA2797FDA095BA2F9C01AD0137
:107B4000220F331F441F551F220F331F441F551F81
:107B5000280F391F4A1F5B1F280F391F4A1F5B1F41
:107B6000309391092093900980911C0490911D04F9
:107B7000AA2797FDA095BA2F7C018D01EE0CFF1C62
:107B8000001F111FEE0CFF1C001F111FE80EF91E35
:107B90000A1F1B1FE80EF91E0A1F1B1FF092AD09DA
:107BA000E092AC098091F508682E77248824992406
:107BB000C9019C01442737FD4095542FC401B301EE
:107BC0000E94B86B5B016C016093290570932A05D4
:107BD00080932B0590932C059701442737FD409502
:107BE000542FC401B3010E94B86BDC01CB01809318
:107BF000210590932205A0932305B0932405A0921C
:107C00000505B0920605C0920705D092080580933D
:107C1000FD049093FE04A093FF04B093000510921E
:107C2000F9041092FA041092FB041092FC04809163
:107C30001F0390912003A0912103B0912203909300
:107C40006908809368081092110410921004109231
:107C5000F1041092F2041092F3041092F404809153
:107C6000EF049091F0049093EE048093ED040E9451
:107C7000B06182E390E09093FC038093FB038091DA
:107C800014099927AA27BB27BC01CD0124EC39E0B0
:107C900040E050E00E94B86BDC01CB018856954C67
:107CA000AF4FBF4F8093A6039093A703A093A80361
:107CB000B093A903809115099927AA27BB27BC0176
:107CC000CD010E94B86BDC01CB018856954CAF4FBB
:107CD000BF4F8093A2039093A303A093A403B093F8
:107CE000A50310928B0310928A038091EF04909168
:107CF000F004AA2797FDA095BA2F20918603309112
:107D000087034091880350918903BC01CD010E94F3
:107D1000B86BDC01CB018093A8099093A909A093CB
:107D2000AA09B093AB091092E8041092E70481E02D
:107D3000809301010E94A5658091AD0484608093C9
:107D4000AD048FEF8093110A1092120A80E28093A3
:107D5000130A8091E208E82FFF27EE0FFF1FE4557A
:107D6000F74F8081918182599F4F9093E6048093D1
:107D7000E5048091E308E82FFF27EE0FFF1FE4558D
:107D8000F74F8081918182599F4F9093E4048093B3
:107D9000E3048091E408E82FFF27EE0FFF1FE4556E
:107DA000F74F8081918182599F4F9093E204809395
:107DB000E1048091E508E82FFF27EE0FFF1FE4554F
:107DC000F74F8081918182599F4F9093E004809377
:107DD000DF0484E68093DE048091F903882309F4AC
:107DE00050C0469A579A4DC00E94611C0ACEDA01D3
:107DF0000E94476C802D9927982F8827DA011196C9
:107E00000E94476C202D820F911D9093380580931E
:107E10003705DA0112960E94476C802D9927982F1A
:107E20008827DA0113960E94476C202D820F911D3E
:107E30009093360580933505DA0114960E94476CBD
:107E4000802D9927982F8827DA0115960E94476C74
:107E5000202D820F911D48CE909581959F4F6CE00B
:107E600070E00E94F76B7093360560933505809142
:107E700090099091910997FF2BCE909581959F4FF6
:107E800027CECF911F910F91FF90EF90DF90CF9071
:107E9000BF90AF909F908F907F906F90089590913A
:107EA000D404992381F58091AD048C7F8093AD0437
:107EB00010C0A92FBB27FD01EB59F84F8083FD01AE
:107EC000EB59F84F8081AD56B64F8C939F5F9C3035
:107ED00080F48091DC03882361F3A92FBB27FD0187
:107EE000EB59F84F8081AD56B64F8C939F5F9C3015
:107EF00080F38091DC03882359F08091DC0381506A
:107F00008093DC0305C08091AD0481608093AD0453
:107F100080919309992790933B0880933A08809128
:107F20009409992790933D0880933C088091960985
:107F3000992790933F0880933E088091950999274F
:107F4000909341088093400810924904109248048D
:107F50000E94DD2A08958091E9088B3F68F08B3FED
:107F600009F4D5C28C3F09F474C38D3F09F4F6C2FD
:107F70008E3F21F48091DF0480939E038091E80876
:107F80008B3F08F439C28B3F09F434C28C3F09F4AB
:107F900048C38D3F09F4D9C28E3F09F478C380915C
:107FA0009F03882309F02DC280939F038091EA08E4
:107FB0008B3F08F42DC28B3F09F428C28C3F09F493
:107FC00042C38D3F09F4C4C28E3F09F45AC3809165
:107FD0009D03882309F021C280939D038091EC08C2
:107FE0008B3F68F08B3F09F495C28C3F09F42EC398
:107FF0008D3F09F4B0C28E3F21F48091DF0480935D
:108000009C038091EE088B3F68F08B3F09F479C2A6
:108010008C3F09F4E2C28D3F09F4BEC28E3F21F4C9
:108020008091DF0480939A038091F6088B3F68F07B
:108030008B3F09F469C28C3F09F4FCC28D3F09F4FF
:1080400090C28E3F21F48091DF0480939B03809146
:10805000F7088B3F08F4E8C18B3F09F4E3C18C3F7C
:1080600009F4EEC28D3F09F494C28E3F09F412C3A5
:10807000809198038B3008F4DCC18F3F11F480931A
:1080800098038091F8088B3F68F08B3F09F427C272
:108090008C3F09F4D2C28D3F09F466C28E3F21F4B1
:1080A0008091DF04809397038091F9088B3F68F0FB
:1080B0008B3F09F417C28C3F09F489C28D3F09F444
:1080C0006EC28E3F21F48091DF04809399038091EA
:1080D000FA088B3F68F08B3F09F407C28C3F09F424
:1080E00079C28D3F09F452C28E3F21F48091DF04A2
:1080F000809396038091FB088B3F68F08B3F09F4D7
:10810000F7C18C3F09F4ABC28D3F09F43CC28E3FEE
:1081100021F48091DF0480939503209100092B3F87
:1081200008F48BC12B3F09F486C12C3F09F47CC2B3
:108130002D3F09F404C22E3F09F4A6C220919303F7
:10814000809101098B3F08F07FC18093C104809129
:1081500002098B3F68F08B3F09F4D0C18C3F09F4D2
:1081600066C28D3F09F4EEC18E3F21F48091DF0499
:108170008093C004809103098B3F68F08B3F09F422
:1081800084C18C3F09F471C28D3F09F4D2C18E3F86
:1081900021F48091DF048093BF04809104098B3F18
:1081A00068F08B3F09F474C18C3F09F461C28D3FC4
:1081B00009F4C2C18E3F21F48091DF048093BE0494
:1081C000809119098B3F68F08B3F09F464C18C3FA3
:1081D00009F454C28D3F09F4A3C18E3F21F480916C
:1081E000DF048093BD0480911A098B3F68F08B3FB8
:1081F00009F454C18C3F09F42FC28D3F09F493C197
:108200008E3F21F48091DF048093BC0480911B0990
:108210008B3F68F08B3F09F444C18C3F09F4ECC1FB
:108220008D3F09F4C5C18E3F21F48091DF04809316
:10823000BB0480911C098B3F68F08B3F09F434C16B
:108240008C3F09F4DCC18D3F09F4B5C18E3F21F4A8
:108250008091DF048093BA04809105098B3F68F018
:108260008B3F09F424C18C3F09F4CFC18D3F09F441
:1082700084C18E3F21F48091DF048093920380912A
:1082800009098B3F68F08B3F09F414C18C3F09F456
:10829000BFC18D3F09F474C18E3F21F48091DF048A
:1082A0008093910380910E098B3F68F08B3F09F416
:1082B00004C18C3F09F4AFC18D3F09F458C18E3F12
:1082C00021F48091DF0480939003809111098B3F0A
:1082D00068F08B3F09F4F4C08C3F09F49FC18D3FD7
:1082E00009F448C18E3F21F48091DF0480938F030D
:1082F000809112098B3F68F08B3F09F4E4C08C3FFA
:1083000009F46EC18D3F09F44DC18E3F21F4809177
:10831000DF0480938E03809113098B3F68F08B3FBD
:1083200009F4D4C08C3F09F464C18D3F09F43DC108
:108330008E3F21F48091DF0480938D038091180992
:108340008B3F68F08B3F09F4C4C08C3F09F45AC1DD
:108350008D3F09F433C18E3F21F48091DF04809377
:108360008C0380911E098B3F08F47FC08B3F09F47A
:108370007AC08C3F09F437C18D3F09F422C18E3F8A
:1083800009F48BC180916C09823008F473C08F3F6F
:1083900011F480936C09809120098B3F08F46EC022
:1083A0008B3F09F469C08C3F09F420C18D3F09F46B
:1083B0000BC18E3F09F474C180919F09823008F48B
:1083C00062C08F3F11F480939F09809133098B3FE6
:1083D00070F08B3F09F480C08C3F09F44CC18D3F95
:1083E00009F49BC08E3F09F05EC18091DF04809349
:1083F000AF0959C18091E50480939F03882309F454
:10840000D3CD843608F4D2CD84E6CECD8091E50478
:1084100080939D03882309F4DFCD843608F4DECDF4
:1084200084E6DACD8091E504809398038B3008F0E0
:1084300024CE8AE024CE2091E504209393038091FA
:1084400001098B3F08F481CE8B3F09F454C08C3F67
:1084500009F408C18D3F09F469C08E3F09F077CE59
:108460008091DF0472CE8091E50480936C098230A4
:1084700008F08DCF81E08DCF8091E50480939F0936
:10848000823008F09ECF81E09ECF8091E50483CEBC
:108490008091E50493CE8091E504A3CE8091E5041C
:1084A000B3CE8091E504C3CE8091E504D3CE809114
:1084B000E504E3CE8091E504F3CE8091E50403CF9B
:1084C0008091E50413CF8091E50423CF8091E504EA
:1084D00033CF8091E50443CF8091E50488CF80912C
:1084E000E504E0CD8091E504F0CD8091E50400CE77
:1084F0008091E50410CE8091E50427CE8091E504BB
:1085000037CE8091E5048ECD8091E5049ECD80919B
:10851000E50432CD8091E50472CD8091E10467CF0E
:108520008091E1045ECE8091E1046ECE8091E10401
:108530000CCE8091E1042FCE8091E1043FCE2091BA
:10854000E1047BCF8091E10413CE8091E10454CF0C
:108550008091E1045DCF8091E10451CD8091E104EF
:108560000BCD8091E10471CD8091E1049BCD809190
:10857000E104A9CE8091E104B9CE8091E1047DCEE1
:108580008091E1048DCE8091E104C5CD8091E1041C
:10859000AFCD8091E10448CF8091E10443CD80913B
:1085A000E10493CD8091E104B4CE8091E104C4CE86
:1085B0008091E1043CCE8091E1044CCE8091E104B5
:1085C000CECE8091E10451CF8091E10457CF8091CC
:1085D000E3047BCD8091E3048BCD8091E30422CD35
:1085E0008091E30496CE8091E3043FCF8091E30431
:1085F00045CF8091E304A0CE8091E30418CE809112
:10860000E30428CE8091E304AACE8091E30435CE22
:108610008091E30445CE8091E30455CE8091E3043C
:1086200065CE8091E304E8CE2091E30406CF8091EB
:10863000E3049ECD8091E30408CD8091E30432CD24
:108640008091E304F1CE8091E304E2CE8091E304D3
:10865000D6CC8091E30490CC8091E304D5CD809179
:10866000E30459CD8091E30470CD8091E30493CD70
:108670008091E304A3CD8091E304B9CE8091E3041B
:10868000B0CD8091DF04C4CE2091DF04D6CE80919E
:10869000DF04B2CE8091DF04C7CE8091DF04E5CE47
:1086A0008091DF04EBCE33272F5F3F4F8CE398E2BE
:1086B000B9010E94F76B7093A1036093A0038091AE
:1086C000F4088093A0098091F308809359090895D4
:1086D0002F923F924F925F926F927F928F929F92D2
:1086E000AF92BF92CF92DF92EF92FF920F931F93C0
:1086F000CF93DF93CDB7DEB7ED970FB6F894DEBF1B
:108700000FBECDBF8091AC04815009F485E0809309
:10871000AC040E948831209102012C3008F0BAC2CA
:10872000299AA090D504B090D604BA82A9828091EB
:10873000590999270A96A816B90614F49A838983C9
:108740008091DE04843608F0A7C28091790590916B
:108750007A05009709F081C41092D4048091AD0489
:108760008F7E8093AD042A3009F47FC4243109F44C
:108770007CC428988091AE049091AF04895E9340A8
:1087800008F47CC48091FD08282F33273A8329837D
:108790008091AD0480618093AD048091DE08A82FA4
:1087A000BB27AA0FBB1FFD01EE53F74F11821082AA
:1087B0008091DF08282F3327220F331FC9018E53E2
:1087C000974FFC0111821082A455B74F11961C924D
:1087D0001E922455374FD90111961C921E928091FA
:1087E000E108E82FFF27EE0FFF1FE455F74F118236
:1087F000108280918403815080938403809184034C
:108800008F3F21F08091AD0484FF3BC40E94AB3FB9
:108810008091880590918905AC01440F551F480F40
:10882000591F0091DE08A02FBB27AA0FBB1FFD0117
:10883000E455F74FE090F008CE2CDD248081918143
:108840008C9D50018D9DB00C9C9DB00C11244A0D47
:108850005B1D57FF02C00C945F5855954795559581
:108860004795AE53B74F8091F108682F77278D91C8
:108870009C91869F9001879F300D969F300D11240B
:10888000240F351F30938905209388058091BF05FB
:108890009091C0054091BB055091BC05840F951F78
:1088A000281B390B3093DC042093DB0480918A056C
:1088B00090918B05AC01440F551F480F591F109123
:1088C000DF08A12FBB27AA0FBB1FFD01E455F74FFF
:1088D000808191818C9D90018D9D300D9C9D300DEE
:1088E0001124420F531F57FF02C00C945B5855953B
:1088F000479555954795AE53B74F8D919C91869F5F
:108900009001879F300D969F300D1124240F351F45
:1089100030938B0520938A058091BD059091BE050B
:108920004091B9055091BA05840F951F281B390B4A
:108930003093DA042093D9048091E108E82FFF27CF
:10894000EE0FFF1FE455F74F80819181909581953F
:108950009F4F8330910514F40C942D4F0297909300
:10896000D8048093D7048091E008E82FFF27EE0F0A
:10897000FF1FE455F74FC080D18048E750E0C40E98
:10898000D51E809198039927AA2797FDA095BA2F05
:10899000BC01CD010E943E6BDC01CB0120E030E048
:1089A00040E251E4BC01CD010E94DF6ADC01CB0151
:1089B000BC01CD010E94216BDC01CB018093A60993
:1089C000F0909703809196039927AA2797FDA09589
:1089D000BA2FBC01CD010E943E6BDC01CB0120E02F
:1089E00030E040E251E4BC01CD010E94DF6ADC01CD
:1089F000CB01BC01CD010E94216BDC01CB01809336
:108A00004C0950919503509363098091870780FF2B
:108A100006C08091AF09813810F00C94904FD0922D
:108A2000D604C092D5048091D5049091D60497FFC6
:108A300002C00C945558F091E608FAA3F2FD02C06A
:108A40000C94774F109273094091DB045091DC0431
:108A5000CA0157FF02C00C94824F95958795959552
:108A6000879597FF02C00C948B4F2091B2043091F0
:108A7000B3042817390714F00C94354FCA0157FF77
:108A800002C00C94205C97FF02C00C94255CBC01D2
:108A900075956795759567956536710514F40C9411
:108AA000384F64E670E04091D9045091DA04CA016D
:108AB00057FD02C00C94414F039695958795959567
:108AC000879597FD02C00C94494F909581959F4FD3
:108AD0002091B0043091B1042817390714F40C9494
:108AE000524F215030408091AD0484FD02C00C945F
:108AF0006D4F1092B3041092B2041092B104109210
:108B0000B004E12FFF27EE0FFF1FE455F74F409110
:108B10000F09242F3327808191812817390734F4D6
:108B20008091340982FF02C00C940450E12FFF278A
:108B3000EE0FFF1FE455F74F842F9927209110095E
:108B4000821B9109208131812817390714F4109272
:108B5000C504E12FFF27EE0FFF1FE455F74F842FC9
:108B6000992722273327281B390B8081918182176F
:108B7000930734F48091340983FF02C00C94FF4FB3
:108B80008091C404882391F0E12FFF27EE0FFF1F8F
:108B9000E455F74F809110099927841B9109208192
:108BA00031818217930714F40C943050E02FFF2783
:108BB000EE0FFF1FE455F74F242F3327808191815B
:108BC0002817390734F48091340980FF02C00C94CF
:108BD000F94F5091C204552399F0E02FFF27EE0F73
:108BE000FF1FE455F74F842F992720911009821B0E
:108BF0009109208131812817390714F40C942B50E6
:108C0000E02FFF27EE0FFF1FE455F74F842F992722
:108C100022273327281B390B8081918182179307E4
:108C200034F48091340981FF02C00C94F44F809198
:108C3000C304882391F0E02FFF27EE0FFF1FE455B8
:108C4000F74F809110099927841B91092081318168
:108C50008217930714F40C9434508091C504882330
:108C600031F48091C404882311F40C94F14F91E005
:108C7000552331F48091C304882311F40C940F50D0
:108C800081E08093C7041092C6041092C50410922C
:108C9000C404FAC1299845CD8091DE048D3808F4CA
:108CA000A8CD8091AD048F7E8093AD049091FE0895
:108CB00082E3989FC001112490937A0580937905EF
:108CC000E981FA81B99714F00C9414508091AE04A4
:108CD0009091AF048F3F910519F010F00C944E580D
:108CE00010925D0510925E0510925F05109260056E
:108CF000109261051092620510926305109264054E
:108D00008A3F910511F40C94745D3091E008E32FD3
:108D1000FF27EE0FFF1FE455F74F808191818135CA
:108D200091050CF4E9C04091D404442309F0E4C057
:108D30008091E108E82FFF27EE0FFF1FE455F74F62
:108D4000808191818C34910514F40C94BB5C8091EA
:108D50007B058F5F893C10F40C94A55D2C3010F0DE
:108D60000C947B5F29981092D40410927B0510928A
:108D7000AF041092AE040091DE08E02FFF27EE0F43
:108D8000FF1FE455F74F808191818734910514F0DE
:108D90000C94355F1091DF08E12FFF27EE0FFF1FC6
:108DA000E455F74F808191810190F081E02DF7FF2C
:108DB00002C00C941F61E734F1050CF470C021E08F
:108DC000A12FBB27AA0FBB1FA455B74F8D919C9114
:108DD00011978734910544F0E02FFF27EE0FFF1F16
:108DE000E455F74F808191818D919C918734910555
:108DF00064F0E02FFF27EE0FFF1FE455F74F80814F
:108E00009181873491050CF022E0E12FFF27EE0FCE
:108E1000FF1FE455F74F808191818634910564F4FA
:108E2000E02FFF27EE0FFF1FE455F74F8081918160
:108E3000873491050CF023E0E12FFF27EE0FFF1F91
:108E4000E455F74F808191818A5B9F4F64F4E02F56
:108E5000FF27EE0FFF1FE455F74F80819181873484
:108E600091050CF024E0E12FFF27EE0FFF1FE455E2
:108E7000F74F808191818A5B9F4F64F4E02FFF2739
:108E8000EE0FFF1FE455F74F8081918186349105E5
:108E90000CF425E0822F0E9475051091DF08E12F68
:108EA000FF27EE0FFF1FE455F74F8081918101905E
:108EB000F081E02DF7FF02C00C9446607E9714F01D
:108EC0000C94215E8091DE08E82FFF27EE0FFF1F34
:108ED000E455F74F808191818A5B9F4F14F00C9489
:108EE000215E81E080937B0788EE93E09093FC0302
:108EF0008093FB033091E008E32FFF27EE0FFF1F65
:108F0000E455F74F808191818B5A9F4F0CF071CCC3
:108F1000D090E108ED2DFF27EE0FFF1FE455F74F2E
:108F200080819181855B9F4F14F00C9471598091E1
:108F30007C058F5F893C10F40C94AF5C88EC8093C7
:108F40007C0581E090E09093AF048093AE0481E0D3
:108F50008093D404109265051092660510926705FF
:108F6000109268051092F9041092FA041092FB0412
:108F70001092FC041092F5041092F6041092F7047B
:108F80001092F8048091F508E82EFF24002711279D
:108F900080919009909191099C01442737FD40955B
:108FA000542FC801B7010E94B86BDC01CB0180933C
:108FB000090590930A05A0930B05B0930C058091C9
:108FC000AC099091AD099C01442737FD4095542F81
:108FD000C801B7010E94B86BDC01CB018093010589
:108FE00090930205A0930305B09304058091290591
:108FF00090912A05A0912B05B0912C058093050531
:1090000090930605A0930705B0930805809121056C
:1090100090912205A0912305B09124058093FD0431
:109020009093FE04A093FF04B093000510925D0599
:1090300010925E0510925F05109260051092610516
:109040001092620510926305109264058091AD0440
:1090500088608093AD040C947359019790937A05BE
:10906000809379052A3009F081CB289A8091AE044B
:109070009091AF04895E934008F084CB1092D404A1
:10908000B8CBA090E608AAA20091C6040E8B0023DC
:1090900021F48091C704882369F080910E099927F3
:1090A00029813A818217930714F49A83898381E096
:1090B0008093E9048091AD0484FFCBC61092D8045C
:1090C0001092D7041092DC041092DB041092DA04A0
:1090D0001092D9049AE59093A60988E780937309C2
:1090E00090934C0989A3809363091092C60410924F
:1090F000C7041E8A2091660930916709409168096A
:10910000509169096091290570912A0580912B057C
:1091100090912C05698B7A8B8B8B9C8B260F371F3C
:10912000481F591F80916D0990916E09A0916F0998
:10913000B0917009A0902105B0902205C090230540
:10914000D0902405AFA2B8A6C9A6DAA68A0D9B1DA9
:10915000AC1DBD1DC0905B09D0905C09E0905D091D
:10916000F0905E09C8AAD9AAEAAAFBAAE090250550
:10917000F09026050091270510912805E88EF98EBC
:109180000A8F1B8FA8A8B9A8CAA8DBA8AE0CBF1C61
:10919000C01ED11EA8AAB9AACAAADBAAC0904D09AE
:1091A000D0904E09E0904F09F0905009CCA6DDA672
:1091B000EEA6FFA6E0901D05F0901E0500911F058C
:1091C00010912005EBA2FCA20DA31EA3ACA4BDA48C
:1091D000CEA4DFA4AE0CBF1CC01ED11EACA6BDA683
:1091E000CEA6DFA6B090C704BF8ABB2009F0D0C5C9
:1091F0000E89002309F0CCC580936D0990936E0908
:10920000A0936F09B09370092093660930936709A2
:1092100040936809509369098091660890916708A6
:10922000815092400CF07EC48091D404882309F0D0
:1092300079C480910E0490910F048F3F910509F03D
:1092400008F47FC5BF89BB2309F017C7EE89EE2359
:1092500009F013C7F091E904FD8BFF2309F00DC756
:10926000A0901709ABA6AA2009F407C7C8A8D9A8D7
:10927000EAA8FBA8C0925B09D0925C09E0925D0964
:10928000F0925E09ECA4FDA40EA51FA5E0924D0985
:10929000F0924E0900934F0910935009809166098E
:1092A00090916709A0916809B0916909B7FF02C060
:1092B0000C94B95F292E3A2E4B2E552447FC5A9414
:1092C00020926609309267094092680950926909B4
:1092D00080916D0990916E09A0916F09B09170090C
:1092E000B7FF02C00C94B35F892F9A2FAB2FBB2717
:1092F000A7FDBA958D839E83AF83B88780936D0950
:1093000090936E09A0936F09B09370098091F5084E
:10931000E82EFF24002711272091190530911A0506
:1093200040911B0550911C05C801B7010E94B86B04
:1093300097FF02C00C94D15F672E782E892E992456
:1093400087FC9A94209115053091160540911705D8
:1093500050911805C801B7010E94B86B97FF02C071
:109360000C94CB5FA72EB82EC92EDD24C7FCDA944F
:10937000D201C10186199709A809B90920911609D6
:10938000E22EFF2400271127BC01CD01A80197017F
:109390000E942C6C39014A0119012A018D819E819C
:1093A000AF81B8858A199B09AC09BD09BC01CD0103
:1093B000A80197010E942C6CD401C30197FE02C042
:1093C0000C94C55F892F9A2FAB2FBB27A7FDBA95A9
:1093D000BC01DA01C90157FF02C00C94BF5F892F9D
:1093E0009A2FAB2FBB27A7FDBA956C018091B204D1
:1093F0009091B30481349105D4F48091B00490919C
:10940000B104813491059CF48091E108E82FFF2795
:10941000EE0FFF1FE455F74F808191810190F0819D
:10942000E02DF7FF02C00C9430617A9734F0809100
:10943000110A8F3F11F40C94655F088D198D2A8DE8
:109440003B8D89899A89AB89BC89081B190B2A0B2A
:109450003B0B0AAF1BAF2CAF3DAF009369051093D8
:109460006A0520936B0530936C05EBA0FCA00DA161
:109470001EA12FA138A549A55AA5E21AF30A040B8B
:10948000150BE986FA860B871C87E0926D05F09232
:109490006E0500936F05109370058AAD9BADACAD62
:1094A000BDAD8093710590937205A0937305B09341
:1094B0007405E0927505F092760500937705109398
:1094C00078058091050590910605A0910705B0915A
:1094D0000805EAACFBAC0CAD1DAD8E199F09A00BC5
:1094E000B10B8093050590930605A0930705B093F3
:1094F00008058091FD049091FE04A091FF04B091B5
:10950000000509851A852B853C85801B910BA20BD4
:10951000B30B8093FD049093FE04A093FF04B093DB
:1095200000051BA5112371F12091E7043091E80497
:109530002138310594F080913D0590913E050196CA
:1095400090933E0580933D05809171099091720939
:109550000196909372098093710920583F4F94F4BB
:1095600080913D0590913E05019790933E05809333
:109570003D0580917109909172090197909372094C
:10958000809371091092E8041092E70401E0A02E84
:10959000B12C8AAD9BADACADBDADB7FF02C00C9494
:1095A000875F81509240A040B0401CF014E0A12E93
:1095B000B12C8091920590919305A0919405B09162
:1095C0009505E0906609F09067090091680910918F
:1095D00069098E199F09A00BB10B815E914BAF4FAA
:1095E000BF4F8F539C49A040B04010F40C94B75D1E
:1095F000F091120AFC8FF93114F40C944F5FB09281
:109600008D05A0928C058AAD9BADACADBDAD8150F2
:109610009041A040B04014F40C94C05D80918E0540
:10962000882311F40C94D75F7093C9046093C80425
:109630008AAD9BADACADBDADB7FF02C00C94166159
:109640009C01AD01B7FF02C00C941061B9E05595C3
:10965000479537952795BA95D1F780918C059091CC
:109660008D05820F931F90938D0580938C052AADF5
:109670003BAD4CAD5DAD57FF02C00C940A613901A2
:109680004A01A3E09594879477946794AA95D1F7BB
:1096900013012401F9E86F16F3E17F06F0E08F066D
:1096A000F0E09F0644F0F8E86F2EF3E17F2E812C66
:1096B000912C13012401D401C30197FE02C00C9424
:1096C0004461892F9A2FAB2FBB27A7FDBA95680F4E
:1096D000791F2AAD3BAD4CAD5DAD203080EF380732
:1096E0008FEF48078FEF580714F00C94D05D8091EE
:1096F0008F05882311F40C94A65F7093C9046093BE
:10970000C804DA01C90157FF02C00C9401619C0131
:10971000AD01B7FF02C00C94596169E055954795BA
:10972000379527956A95D1F780918C0590918D0595
:10973000820F931F90938D0580938C052AAD3BADCE
:109740004CAD5DAD57FF02C00C94536139014A0125
:1097500043E095948794779467944A95D1F798E776
:1097600069169CEE79069FEF89069FEF990644F4EF
:1097700038E7632E3CEE732E3FEF832E3FEF932EA0
:109780006092800570928105809282059092830597
:10979000D401C30197FE02C00C94FB60892F9A2F5D
:1097A000AB2FBB27A7FDBA956091C8047091C9047F
:1097B000680F791FABA52A2F332780918C059091D4
:1097C0008D052817390724F430938D0520938C05D7
:1097D000BC8DBB2379F02B2F332727FD309580914B
:1097E0008C0590918D052817390724F430938D0549
:1097F00020938C052AAD3BAD4CAD5DAD21383105D4
:109800004105510574F080914105909142052091E8
:109810008C0530918D05820F931F909342058093A4
:1098200041058AAD9BADACADBDAD80589F4FAF4FEC
:10983000BF4F74F4809141059091420520918C05B1
:1098400030918D05821B930B9093420580934105C7
:10985000B1E0AB2EB12C89859A85AB85BC85B7FF6D
:1098600002C00C949D5F81509240A040B0401CF01B
:10987000A4E0AA2EB12C20E030E040E050E080913E
:10988000960590919705A0919805B09199056090E3
:109890006D0970906E0980906F099090700986191B
:1098A0009709A809B909815E914BAF4FBF4F8F53FC
:1098B0009C49A040B04028F0FC8DF93114F40C9480
:1098C000395FB0928D05A0928C0589859A85AB850C
:1098D000BC8581509041A040B04014F40C94C45D0C
:1098E00080919005882311F40C94905FD092CB0462
:1098F000C092CA0489859A85AB85BC85B7FF02C032
:109900000C944A61B7FF02C00C94F560F9E0B5957C
:10991000A79597958795FA95D1F7A80EB91EB0929D
:109920008D05A0928C0529853A854B855C8557FF6E
:1099300002C00C94EF60E3E0559547953795279565
:10994000EA95D1F72938F3E13F07F0E04F07F0E05F
:109950005F0714F40C94856088E893E1A0E0B0E020
:109960008093840590938505A0938605B093870521
:109970008091840590918505A0918605B091870519
:10998000B7FF02C00C94D360892F9A2FAB2FBB274F
:10999000A7FDBA95C090CA04D090CB04C80ED91EBA
:1099A00029853A854B855C85203080EF38078FEF1D
:1099B00048078FEF580714F00C94DC5D80919105F7
:1099C000882311F40C947E5FD092CB04C092CA0419
:1099D000DA01C90157FF02C00C943B619C01AD0143
:1099E000B7FF02C00C943561B9E05595479537959E
:1099F0002795BA95D1F780918C0590918D05820FAE
:109A0000931F90938D0580938C0529853A854B850E
:109A10005C8557FF02C00C94DD60A3E05595479527
:109A200037952795AA95D1F728379CEE39079FEFF0
:109A300049079FEF590714F00C948F6088E79CEE5C
:109A4000AFEFBFEF8093840590938505A0938605C3
:109A5000B09387058091840590918505A091860536
:109A6000B0918705B7FF02C00C942A61892F9A2F05
:109A7000AB2FBB27A7FDBA95C090CA04D090CB04EA
:109A8000C80ED91EABA52A2F332780918C05909143
:109A90008D052817390724F430938D0520938C0504
:109AA000BC8DBB2379F02B2F332727FD3095809178
:109AB0008C0590918D052817390724F430938D0576
:109AC00020938C0529853A854B855C8521383105A5
:109AD0004105510574F080913F059091400520911A
:109AE0008C0530918D05820F931F909340058093D4
:109AF0003F0589859A85AB85BC8580589F4FAF4FC0
:109B0000BF4F0CF0D0C280913F059091400520914D
:109B10008C0530918D05821B930B909340058093AB
:109B20003F05C1C29090110A6FEF961611F40C9484
:109B300065588091F508A82EBB24CC24DD246989C2
:109B40007A898B899C89A60195010E942C6C7901E8
:109B50008A018091900990919109AA2797FDA0957B
:109B6000BA2FE81AF90A0A0B1B0B6FA178A589A571
:109B70009AA5A60195010E942C6C59016A01809159
:109B8000AC099091AD09AA2797FDA095BA2FA81A04
:109B9000B90ACA0ADB0A292C332427FC3094432C47
:109BA000532CC201B101A80197010E94B86B97FD27
:109BB0005FC23B014C01F9E09594879477946794D8
:109BC000FA95D1F7C201B101A60195010E94B86BC7
:109BD00097FF02C00C94785C5B016C01E9E0D594BE
:109BE000C794B794A794EA95D1F78091B204909165
:109BF000B304813491053CF48091B0049091B10498
:109C000081349105C4F0D401C30197FE02C00C94C5
:109C10006F5D3C014D019594879477946794D601CC
:109C2000C501D7FE02C00C946A5D5C016D01D5943C
:109C3000C794B794A7948091E108E82FFF27EE0F0F
:109C4000FF1FE455F74F808191810190F081E02D55
:109C5000F7FF02C00C94735C7A97A4F0C401B301BF
:109C600023E030E040E050E00E942C6C39014A01D2
:109C7000C601B50123E030E040E050E00E942C6CCA
:109C800059016A018091130A282F332727FD309547
:109C9000432F532F261537054805590514F439016C
:109CA0004A01992787FD9095909581959F4FAA2706
:109CB00097FDA095BA2F681679068A069B0614F4BC
:109CC0003C014D012A153B054C055D0514F4590175
:109CD0006A01A816B906CA06DB0614F45C016D0118
:109CE0008091090590910A05A0910B05B0910C0592
:109CF00086199709A809B9098093090590930A055F
:109D0000A0930B05B0930C0580910105909102057D
:109D1000A0910305B09104058A199B09AC09BD09FE
:109D20008093010590930205A0930305B093040569
:109D300080910E0490910F048F3F910511F008F06F
:109D400081CAA8A8B9A8CAA8DBA8A0925B09B0924A
:109D50005C09C0925D09D0925E09CCA4DDA4EEA49A
:109D6000FFA4C0924D09D0924E09E0924F09F092A3
:109D700050090091E9040D8BA090D704B090D8044D
:109D8000C501B7FEF0C1882799278A199B09EBC145
:109D90001092190510921A0510921B0510921C05BD
:109DA00010921505109216051092170510921805BD
:109DB0001092660910926709109268091092690959
:109DC00010926D0910926E0910926F09109270092D
:109DD0001CA61DA61EA61FA620E030E040E050E015
:109DE00028AB39AB4AAB5BAB8091090590910A0572
:109DF000A0910B05B0910C05809305059093060585
:109E0000A0930705B0930805809101059091020584
:109E1000A0910305B09104058093FD049093FE0486
:109E2000A093FF04B093000510920F0410920E044B
:109E30001092C9041092C8041092CB041092CA0464
:109E40003F89332309F0F5C94E89442309F0F1C94C
:109E5000E3C93091630939A34DC93FEF8E3F9307A2
:109E60000CF0D7C002960C94AF44B9016150704019
:109E70004091D9045091DA04CA0157FF02C00C94F2
:109E80005C45959587959595879597FF02C00C94AD
:109E900065452091B0043091B1042817390714F0BA
:109EA0000C947145CA0157FF02C00C942B5C97FFBC
:109EB00002C00C94285C9C01359527953595279513
:109EC0002536310514F40C94734524E630E0809176
:109ED000AD0484FF02C00C9479453093B104209303
:109EE000B0047093B3046093B2040C948145F09273
:109EF00073094091DB045091DC04CA0157FD02C094
:109F00000C942D450396959587959595879597FD86
:109F100002C00C943545909581959F4F0C94354522
:109F200080918007992787FD90954E2D5527849F16
:109F3000B001859F700D949F700D1124CB0120916D
:109F4000DB043091DC04820F931F9093DC04809338
:109F5000DB0480918107992787FD9095849FD0012C
:109F6000859FB00D949FB00D1124CD012091D9048F
:109F70003091DA04820F931F9093DA048093D9040E
:109F800080918207992787FD90952091D704309181
:109F9000D804820F931F9093D8048093D7048091A4
:109FA0008407282F332727FD30958091EB089927C8
:109FB000289FF001299FF00D389FF00D1124F09398
:109FC0008B03E0938A038091830799278C159D0565
:109FD00014F00C940F459093D6048093D5040C9400
:109FE0001345982F0C94384681E08093C3040C9459
:109FF0002D4681E08093C204582F0C94004681E0E6
:10A000008093C4040C94D64581E08093C5040C94DD
:10A01000A9451092D8041092D7040C94B34490939D
:10A02000C6048093C70430C88091D404882311F4F7
:10A030000C9466468091AE049091AF04FFEF8F3F81
:10A040009F0711F40C946A4601969093AF04809395
:10A05000AE040C946A461092C20450E00C94004680
:10A060001092C4040C94D6451092C3040C942D464F
:10A0700061507E4F8F4F9F4F9CCD60E070E06B0131
:10A080001092E9041D8AE0906609F090670900913A
:10A0900068091091690960906D0970906E0980904F
:10A0A0006F099090700980917309882309F0B6C7F1
:10A0B0001092CB041092CA041092C9041092C804E2
:10A0C000E0929205F0929305009394051093950504
:10A0D00060929605709297058092980590929905E6
:10A0E0001092190510921A0510921B0510921C056A
:10A0F000109215051092160510921705109218056A
:10A100001092110510921205109213051092140569
:10A1100010926609109267091092680910926909F5
:10A1200010926D0910926E0910926F0910927009C9
:10A1300010925B0910925C0910925D0910925E0901
:10A1400010924D0910924E0910924F091092500929
:10A1500010920F0410920E04A090D704B090D8046F
:10A16000C501B7FC10CE409774F068EE262E63E070
:10A17000362E3092AB032092AA031AA114FD03C01D
:10A1800081E080937F05D090F208ED2CFF2400271A
:10A190001127B501882777FD8095982F9501B7FC89
:10A1A00078C7442737FD4095542F0E94B86B9B0118
:10A1B000AC01C801B7010E94B86B97FD65C759E0B3
:10A1C00095958795779567955A95D1F79B018D2D34
:10A1D00099278A9DA0018B9D500D9A9D500D1124A9
:10A1E000CA0157FD43C79595879595958795280F83
:10A1F000391FC901AA2797FDA095BA2F809365053D
:10A2000090936605A0936705B0936805E090F90404
:10A21000F090FA040091FB041091FC04E81AF90A8A
:10A220000A0B1B0B51E5E51653ECF50650E005074C
:10A2300050E015070CF4E9C680E593ECA0E0B0E02F
:10A240008093F9049093FA04A093FB04B093FC0468
:10A250008091F9049091FA04A091FB04B091FC0460
:10A26000805B9C43AF4FBF4F64F480EB9CE3AFEF48
:10A27000BFEF8093F9049093FA04A093FB04B0938A
:10A28000FC04C090EF04D090F004C114D10409F490
:10A29000B5C57AA173FFB2C589899A89AB89BC8992
:10A2A000B7FF02C00C94425C09E0B595A79597955D
:10A2B00087950A95D1F79BAF8AAF97FF02C00C94A0
:10A2C0004E5C8FA198A5A9A5BAA5B7FF02C00C94B2
:10A2D000485C19E0B595A795979587951A95D1F79C
:10A2E000BC0197FF02C00C943D5CAAADBBADA617A4
:10A2F000B70714F47BAF6AAF6AAD7BAD77FF02C0DE
:10A300000C94395C2B01559447945594479455947B
:10A3100047940894411C511CECE1F2E0CE0EDF1E84
:10A3200076010027F7FC0095102FA4EEAA2EADEFC2
:10A33000BA2ECA0CDB1C6090A8097090A909809005
:10A34000AA099090AB092091860330918703409130
:10A350008803509189032D8F3E8F4F8F58A3C401DE
:10A36000B3010E942C6CE21AF30A040B150BC8010E
:10A37000B70128E631E040E050E00E942C6CDC019F
:10A38000CB018C01045B1040A090A109B090A20900
:10A39000C501B7FE02C00C94335C8138910514F0FE
:10A3A00000E010E02090AA033090AB0321143104A8
:10A3B000A9F44AAD5BAD4931510584F48091E704BD
:10A3C0009091E804800F911F9093E8048093E70434
:10A3D00080917F05882311F00C94455DC801880F9A
:10A3E000991F880F991F880F991FB2010E94F76B60
:10A3F0009B01442737FD4095542F260D371D481DDE
:10A40000591D2093A8093093A9094093AA09509394
:10A41000AB09F0909B036F2D7727AAADBBAD6A9F68
:10A42000C0016B9F900D7A9F900D112497FF02C081
:10A430000C94305C9595879595958795959587951E
:10A440009595879595958795681B790B7BAF6AAF36
:10A4500077FF02C00C94555C2114310411F00C9468
:10A460006A5C0091B2041091B3048091B0049091A1
:10A47000B104080F191F17FF02C00C94925D1595C7
:10A4800007951595079515950795005C1F4FCA010F
:10A49000B9012D8D3E8D4F8D58A10E942C6CDA0193
:10A4A000C9012091ED043091EE04442737FD409519
:10A4B000542F821B930BA40BB50B845E9D4FAF4FA3
:10A4C000BF4FBC01CD0128E631E040E050E00E94E2
:10A4D0002C6CDC01CB01845B90402AAD3BAD829FAC
:10A4E000F001839FF00D929FF00D1124CF01B80170
:10A4F0000E94F76B83E0F89EA00111245BAF4AAF86
:10A500004617570714F00C945D5CBA01CB01AA27DB
:10A5100097FDA095BA2F2091F9043091FA0440914B
:10A52000FB045091FC04820F931FA41FB51F80935E
:10A53000F9049093FA04A093FB04B093FC04809177
:10A540007E0581508F3F09F462C480937E055D894A
:10A55000552381F0109261051092620510926305F7
:10A560001092640510925D0510925E0510925F05D1
:10A57000109260056F89662309F044C580917309C4
:10A580009927AA27BB27BC01CD0129893A894B8984
:10A590005C890E94B86BDC01CB01BC01CD0128EFC6
:10A5A0003AE240E050E00E942C6C19017E8977234A
:10A5B00009F025C5809173099927AA27BB27BC01FB
:10A5C000CD012FA138A549A55AA50E94B86BDC0181
:10A5D000CB01BC01CD0128EF3AE240E050E00E94FF
:10A5E0002C6C3C832B83809047099090480989EC20
:10A5F000881691040CF4F8C4B8EC8B2E912C909230
:10A600004809809247090091520910915309093C69
:10A6100011050CF4E1C408EC10E010935309009309
:10A6200052098091540990915509AA2797FDA09548
:10A63000BA2F2091A609C22EDD24EE24FF24BC01EE
:10A64000CD01A70196010E94B86B9B01AC01C4012A
:10A65000AA2797FDA095BA2FF7E0880F991FAA1F88
:10A66000BB1FFA95D1F7280F391F4A1F5B1F57FDF3
:10A67000ECC4E6E05595479537952795EA95D1F7CF
:10A680004101820E931E2401809145099091460953
:10A69000AA2797FDA095BA2FBC01CD01A70196016D
:10A6A0000E94B86B9B01AC01C801AA2797FDA09539
:10A6B000BA2F77E0880F991FAA1FBB1F7A95D1F791
:10A6C000280F391F4A1F5B1F57FDBAC466E0559516
:10A6D0004795379527956A95D1F76B807C80620EF8
:10A6E000731E6301AA0CBB1CC501AA2797FDA09588
:10A6F000BA2F20914C09332744275527BC01CD019F
:10A700000E94B86B7B018C0197FD91C456E01595B2
:10A710000795F794E7945A95D1F739A1832F992794
:10A72000AA27BB2720910D0530910E0540910F05FA
:10A7300050911005BC01CD010E94B86BDC01CB012A
:10A74000BC01CD0120EF35E540E050E00E942C6CCB
:10A750005701A20EB31EC50141E0841640E49406E1
:10A7600024F0812C40E4942E240150E0851650EC16
:10A7700095060CF02CC4812C30EC932E9092550948
:10A780008092540961E0661660E4760624F0612C3C
:10A7900020E4722E630170E0671670EC77060CF00F
:10A7A00011C4612C00EC702E70924609609245092C
:10A7B000A1E0AA16A0E4BA0624F0A12C10E4B12E60
:10A7C000C501B0E0AB16B0ECBB060CF0F6C3A12C93
:10A7D000B0ECBB2EB092A209A092A1098091000119
:10A7E000482F552780912703909128034817590730
:10A7F00094F42091270330912803E981FA814E9F38
:10A80000C0014F9F900D5E9F900D1124B9010E94D1
:10A81000F76B7A836983C980DA80CC0CDD1CCC0CA1
:10A82000DD1CDA82C982DAA0D0FE51C00E89002375
:10A8300009F04DC01F89112309F049C080919E0580
:10A8400090919F0590934D0880934C08809110043F
:10A8500090911104909347088093460820914305F6
:10A86000309144052115310509F0F8C480911D038C
:10A8700090911E038959934010F00C94B25C809122
:10A880001D0390911E038436910510F00C94AD5D6C
:10A8900087B58B3010F40C94485E809112048F5F62
:10A8A000809312049AE0890290011124809170082B
:10A8B000821B87BD8CE291E09093FC038093FB03A5
:10A8C0008EE591E09093440580934305E8C4509051
:10A8D000A00940905909242D3327C901880F991FD9
:10A8E000880F991F8896E981FA81E817F90714F40F
:10A8F0009A838983852D9927880F991F880F991F1F
:10A9000080559040C980DA808C159D0514F49A8397
:10A910008983809146048823A1F08091AE049091B0
:10A92000AF040297C09768F4E980FA801E141F04F0
:10A9300044F481E090E09093AF048093AE043A83B6
:10A94000298309811A81109331080093300880917E
:10A95000650590916605A0916705B0916805880F1F
:10A96000991FAA1FBB1F880F991FAA1FBB1FA81AD8
:10A97000B90AB9AEA8AE013A11050CF40AC3C80170
:10A9800017FDA1C39595879528AD39AD821793071B
:10A9900014F499AF88AF909581959F4F48AD59AD0C
:10A9A0004817590714F499AF88AF252D3327220F84
:10A9B000331F220F331FC90149815A81841B950B14
:10A9C00068AD79AD8617970714F499AF88AF898180
:10A9D0009A81821B930BA8ADB9ADA817B90714F4DF
:10A9E00099AF88AF8091DB049091DC048401081B4F
:10A9F000190B1093650900936409A0907309AA20AC
:10AA000009F4C1C2281A390AC101AA2797FDA095E5
:10AA1000BA2F20915D0530915E0540915F05509100
:10AA20006005820F931FA41FB51F80935D0590934F
:10AA30005E05A0935F05B093600560915D05709120
:10AA40005E0580915F05909160056130BAEF7B07EC
:10AA5000B0E08B07B0E09B0774F080E09AEFA0E0D5
:10AA6000B0E080935D0590935E05A0935F05B09381
:10AA70006005BC01CD016030E6E07E07EFEF8E0798
:10AA8000EFEF9E0774F480E096E0AFEFBFEF8093A6
:10AA90005D0590935E05A0935F05B0936005BC01D2
:10AAA000CD01E090A003F090A1039701442737FD6A
:10AAB0004095542F0E942C6C6801C20ED31EB0909A
:10AAC0008C036B2D77278827992728AD39AD37FD63
:10AAD000C9C237FDC4C23595279509811A81200F57
:10AAE000311F442737FD4095542F0E94B86B97FDC6
:10AAF000B1C226E095958795779567952A95D1F708
:10AB00009B016C157D050CF46B01309521953F4F31
:10AB1000C216D3060CF469018091D9049091DA042D
:10AB20008301081B190B1093440900934309AA20C1
:10AB300009F423C22B813C81281B390BC901AA27A8
:10AB400097FDA095BA2F2091610530916205409143
:10AB5000630550916405820F931FA41FB51F809356
:10AB6000610590936205A0936305B09364056091BD
:10AB70006105709162058091630590916405613073
:10AB80003AEF730730E0830730E0930774F080E01A
:10AB90009AEFA0E0B0E08093610590936205A093E6
:10ABA0006305B0936405BC01CD01603046E07407D5
:10ABB0004FEF84074FEF940774F480E096E0AFEF17
:10ABC000BFEF8093610590936205A0936305B093F6
:10ABD0006405BC01CD019701442737FD4095542FF2
:10ABE0000E942C6C7801E20EF31E6B2D77278827CC
:10ABF000992728AD39AD37FD43C237FD3EC23595A3
:10AC00002795A981BA812A0F3B1F442737FD40951C
:10AC1000542F0E94B86B97FD2BC216E0959587952F
:10AC2000779567951A95D1F79B016E157F050CF402
:10AC30007B01309521953F4FE216F3060CF4790124
:10AC40008601222717FD2095322F0D871E872F871B
:10AC5000388B242D33273DAB2CAB452D55275FABCF
:10AC60004EABB3E9CB2EB9E0DB2E00ED15E02701AA
:10AC7000662457FC6094762C68AD79AD4B01AA240C
:10AC800097FCA094BA2CABE03A2EF4E7EF2EF9E053
:10AC9000FF2E07C0FBAFEAAFEAADD601EC930C94F0
:10ACA0008961F801258512160CF08FC049815A81FF
:10ACB000CA01AA2797FDA095BA2F332727FD309503
:10ACC000432F532FBC01CD010E94B86B97FD91C05B
:10ACD000E6E09595879577956795EA95D1F77BAFEF
:10ACE0006AAFF8018685282F332727FD3095432F3B
:10ACF000532F6D857E858F8598890E94B86B97FD4F
:10AD000073C056E095958795779567955A95D1F7D5
:10AD10002AAD3BAD260F371F3BAF2AAFF801878521
:10AD2000282F332727FD3095432F532FC301B2011E
:10AD30000E94B86B97FD51C046E095958795779531
:10AD400067954A95D1F72AAD3BAD260F371F3BAF2C
:10AD50002AAFF8018089282F332727FD3095432F0C
:10AD6000532FC501B4010E94B86BDC01CB01B7FDC4
:10AD700030C036E0B595A795979587953A95D1F768
:10AD8000F701608171812AAD3BAD820F931F0E9454
:10AD90004C31D7018D939C9397FD24C09595879551
:10ADA000959587959BAF8AAFECA9FDA98E179F0754
:10ADB0000CF470CF2EA93FA94AAD5BAD241735071F
:10ADC0000CF06ACF3BAF2AAF67CFD6011C920C9430
:10ADD0008961CF96A11DB11DCCCF615C7F4F8F4F94
:10ADE0009F4FAACF0396DACF615C7F4F8F4F9F4F63
:10ADF00088CF615C7F4F8F4F9F4F6ACFA090A10992
:10AE0000B090A20980917E05815008F09ECB88E128
:10AE100080937E058091F5089927880F991F880FE8
:10AE2000991F7C010027F7FC0095102F69897A890A
:10AE30008B899C89A80197010E942C6C3093230870
:10AE4000209322086FA178A589A59AA5A80197014A
:10AE50000E942C6C3093250820932408809190093F
:10AE60009091910997FDEAC4959587959595879559
:10AE700090932708809326088091AC099091AD09A2
:10AE800097FDDAC4959587959595879590932908B0
:10AE900080932808B0922B08A0922A088091D004B1
:10AEA0009091D104A091D204B091D304BC01CD0102
:10AEB00025E030E040E050E00E942C6C30932D08FB
:10AEC00020932C08809166089091670890932F0832
:10AED00080932E08D0923308C092320880912703C5
:10AEE0009091280390933508809334088091DE0474
:10AEF000992790933708809336088091A8099091FC
:10AF0000A909A091AA09B091AB09209186033091BB
:10AF100087034091880350918903BC01CD010E94B1
:10AF20002C6C30933908209338088091100490914C
:10AF30001104909347088093460880917B079927D6
:10AF400090934908809348088091F7039091F80303
:10AF500090934B0880934A088091BF059091C0055B
:10AF600090935F0880935E088091BD059091BE0527
:10AF70009093610880936008EACAC801AA2797FDE8
:10AF8000A095BA2FE0CDC801AA2797FDA095BA2FAA
:10AF900040CD68AD79AD6135710524F080E590E074
:10AFA00099AF88AFA8ADB9ADA05BBF4F0CF0FDCC99
:10AFB00000EB1FEF19AF08AFF8CC9093A209809374
:10AFC000A1090CCCD0924609C0924509F1CB509210
:10AFD000550940925409D6CBAFEF08331A070CF04D
:10AFE00020CB08E31FEF19CB98E389169FEF990652
:10AFF0000CF009CBA8E38A2EAFEF9A2E00CB1C826F
:10B000001B82F1CA22243324D1CAE092F904F092BF
:10B01000FA040093FB041093FC041AC9D092CB04E9
:10B02000C092CA047093C9046093C80449C82FE34E
:10B0300030E040E050E0E20EF31E041F151F66CB27
:10B04000215C3F4F4F4F5F4F41CB215C3F4F4F4FF4
:10B050005F4F0FCB615C7F4F8F4F9F4F4ACD2F5F6C
:10B060003F4F39CD309521953F4F33CD0396BBC827
:10B07000615C7F4F8F4F9F4FD0CD2F5F3F4FBFCD34
:10B08000309521953F4FB9CD61507E4F8F4F9F4FE7
:10B0900096C8222733272A193B0983C88091AD041B
:10B0A00082608093AD040C9485461092D604109271
:10B0B000D5040C941B454D5F5F4F0C9477444D5F56
:10B0C0005F4F0C942D4401965DCC8091F508E82EDD
:10B0D000FF240027112769897A898B899C89A80117
:10B0E00097010E942C6C39014A018091900990913E
:10B0F0009109AA2797FDA095BA2F681A790A8A0A9A
:10B100009B0A6FA178A589A59AA5A80197010E941D
:10B110002C6C59016A018091AC099091AD09AA2764
:10B1200097FDA095BA2FA81AB90ACA0ADB0AD4015A
:10B13000C30197FCF3C43C014D0154E095948794FE
:10B14000779467945A95D1F7D601C501D7FCF2C41C
:10B150005C016D0144E0D594C794B794A7944A95D7
:10B16000D1F78091B2049091B304813491050CF42D
:10B17000C5C3C401B30123E030E040E050E00E94C9
:10B180002C6C39014A01C601B50123E030E040E0F2
:10B1900050E00E942C6C59016A018091E108E82F6F
:10B1A000FF27EE0FFF1FE455F74F8081918101903B
:10B1B000F081E02DF7FDBAC47A97A4F0C401B30181
:10B1C00023E030E040E050E00E942C6C39014A015D
:10B1D000C601B50123E030E040E050E00E942C6C55
:10B1E00059016A0171E267167104810491042CF01F
:10B1F00030E2632E712C812C912C80EE68168FEF3B
:10B2000078068FEF88068FEF980644F420EE622EC2
:10B210002FEF722E2FEF822E2FEF922E91E2A91692
:10B22000B104C104D1042CF090E2A92EB12CC12CA0
:10B23000D12CA0EEAA16AFEFBA06AFEFCA06AFEF59
:10B24000DA0614F00C94704E80EEA82E8FEFB82E14
:10B250008FEFC82E8FEFD82E0C94704E8091D004B3
:10B260009091D104A091D204B091D304F4E0880F5E
:10B27000991FAA1FBB1FFA95D1F7809313049093CF
:10B280001404A0931504B0931604109211041092A4
:10B2900010042150304030934405209343054AA1C7
:10B2A00041FF3EC080919E03823308F051C38091DC
:10B2B000CB03815098F41092EA048091D0049091CD
:10B2C000D104A091D204B091D3048093CC04909384
:10B2D000CD04A093CE04B093CF0481E08093CB0340
:10B2E00041C010927C05ED2DFF27EE0FFF1FE455A6
:10B2F000F74F808191818C3491050CF499C2809133
:10B300007D058F5F893C08F41FC31092D40488EC3C
:10B3100080937D051092AF041092AE040C94F94313
:10B3200020919E0380918A0390918B03820F911D3F
:10B330002091EB083327829FB001839F700D929F6D
:10B34000700D1124CB01AA2797FDA095BA2F8093E9
:10B35000CC049093CD04A093CE04B093CF0481E0AD
:10B360008093EA04E0908603F090870300918803BD
:10B370001091890369897A898B899C89A801970131
:10B380000E942C6C59016A016FA178A589A59AA524
:10B39000A80197010E942C6CB901C5010E94A76AFF
:10B3A0006C01CD971CF0ECE3CE2ED12CC6010E948F
:10B3B0004D696C018091EA04882309F469C1809188
:10B3C000AD0499279C012071307084FD61C1B0905B
:10B3D0003609B0FC04C08091E60881FD5DC4098196
:10B3E0001A8130939B0520939A056090D004709049
:10B3F000D1048090D2049090D3048091CC04909199
:10B40000CD04A091CE04B091CF0486159705A80570
:10B41000B90514F0B0FC52C1E090D004F090D10412
:10B420008091CC049091CD04E81AF90A80919D0393
:10B4300099278E9D90018F9D300D9E9D300D11247A
:10B44000C90137FDDAC595958795959587959595A9
:10B45000879595958795081B190B209110043091BD
:10B46000110437FDC7C53595279535952795359531
:10B470002795293031050CF4CCC328E030E0229F19
:10B48000A001239F500D329F500D11249A0157FDAA
:10B49000AEC53595279535952795809110049091E7
:10B4A0001104280F391F80919F039927AA27BB27D2
:10B4B000442737FD4095542FBC01CD010E94B86B45
:10B4C00097FD90C5B7E09595879577956795BA955F
:10B4D000D1F79B015FEF613875070CF092C321E84B
:10B4E0003FEF021B130B6090F1047090F204809008
:10B4F000F3049090F40497FC64C5A7E095948794B6
:10B5000077946794AA95D1F780919C03282F3327CD
:10B5100044275527C401B3010E94B86B97FD4CC561
:10B52000F5E09595879577956795FA95D1F79B0105
:10B530007FEF213837070CF04BC321E83FEF021BA8
:10B54000130B85E990E0E80EF91E9BE2E91691E005
:10B55000F906E8F480919A0590919B05892BB9F43E
:10B5600080919E0590919F051816190684F480918C
:10B57000A0059091A105081719070CF49FC28091AE
:10B58000C9039091CA03801791070CF497C2809168
:10B59000430590914405892B21F000919E0510915F
:10B5A0009F0580919A039927AA27BB272091150A06
:10B5B000332727FD3095432F532FBC01CD010E9427
:10B5C000B86B97FD0AC5E7E09595879577956795E0
:10B5D000EA95D1F79B01AFEF61387A070CF0F0C222
:10B5E00021E83FEF021B130BC801AA2797FDA09586
:10B5F000BA2F5DE0880F991FAA1FBB1F5A95D1F77C
:10B600009601442737FD4095542FBC01CD010E947F
:10B610002C6C20936D0530936E0540936F0550930D
:10B62000700500916D0510916E0580919C059091BB
:10B630009D059C01220F331F280F391F200F311F3A
:10B6400037FDC8C4A9015595479555954795BA0149
:10B650008091E708282F3327220F331F220F331F33
:10B66000421753070CF0BCC2A901B9015090A009C0
:10B67000B0FE64C2E981FA81E417F5070CF05EC2FE
:10B68000AF01F0939D05E0939C055A83498318C050
:10B690006091EF08662309F43AC177276634710593
:10B6A0000CF00EC226E430E03093C8032093C703A9
:10B6B000E980FA80F0929D05E0929C055090A009E7
:10B6C0008091AD0481FFA7C08091AD0484FDA3C02B
:10B6D000E090A205F090A3050091A4051091A505A6
:10B6E000E114F10401051105B1F429813A817901D0
:10B6F0000027F7FC0095102FECE0EE0CFF1C001F5C
:10B70000111FEA95D1F7E092A205F092A3050093EC
:10B71000A4051093A50580911004909111048091C7
:10B7200010049091110497FDEEC3843691050CF03E
:10B7300072C069817A819B01442737FD4095542F5F
:10B74000C601AA2797FDA095BA2FBC01CD010E9482
:10B75000B86B97FD6CC49B01AC017DE05595479596
:10B76000379527957A95D1F720936D0530936E051F
:10B7700040936F05509370058091AE049091AF0493
:10B7800077E0803D970708F053C3D801C70169E00F
:10B79000B695A795979587956A95D1F7E81AF90A0E
:10B7A0000A0B1B0BDA01C90123E0880F991FAA1F9E
:10B7B000BB1F2A95D1F7E80EF91E0A1F1B1FE09246
:10B7C000A205F092A3050093A4051093A505D80146
:10B7D000C7011CE0B695A795979587951A95D1F75F
:10B7E00090939F0580939E054091ED08442309F4B2
:10B7F00014C355279C01BA010E94F76BC901861B2F
:10B80000970B9093A1058093A005260F371F3093C7
:10B81000CA032093C903A090A109B090A209809007
:10B82000540990905509609045097090460951C897
:10B8300010927D050C94F943039624CB039614CB08
:10B84000909581959F4F0C94434503960C944745E2
:10B8500003960C945B4F909581959F4F0C94574F96
:10B860004F960C941A52882799278A199B090C9491
:10B87000CD51695F7F4F0C948251709561957F4FD8
:10B880000C94755181509E4FAF4FBF4F0C94545143
:10B8900081509E4FAF4FBF4F0C9469519095819549
:10B8A0009F4F9BAF8AAF0C94615184EF91E09093CE
:10B8B000AB038093AA030C949F528AAD9BAD9095E5
:10B8C00081959F4F6817790714F00C948652BC013C
:10B8D0000C9486520894210831083092AB032092D0
:10B8E000AA030C949F52F095E195FF4F0C942C4EB7
:10B8F00061507E4F8F4F9F4F0C94EC4D8091B00460
:10B900009091B104813491050CF447CC32CC409134
:10B910009E0550919F0557FDB8C155954795559582
:10B9200047958091270390912803209100013327A8
:10B93000489F5001499FB00C589FB00C1124C5017D
:10B94000B9010E94F76BAACE80937D050C94F94350
:10B9500081E08093EA0488EC8093CB0303CD80934D
:10B960007C05C1CC87B5853F08F0F3C080911204F7
:10B9700081500C94505480819181855B9F4F0CF0D5
:10B98000F2C080917B058F5F80937B05893C10F42A
:10B990000C947C472C3008F07EC32998A4E0B0E0DA
:10B9A0008FEF082E0E94546C1092D40410927B05E5
:10B9B0001092AF041092AE040E94A93CA4E0B0E043
:10B9C000809137059091380597FD41C4892F990FD3
:10B9D000990B082E0E94546CA5E0B0E080913705C9
:10B9E00090913805082E0E94546CA6E0B0E080913A
:10B9F00035059091360597FD27C4892F990F990B2E
:10BA0000082E0E94546CA7E0B0E08091350590911B
:10BA10003605082E0E94546C08E010E080912F0536
:10BA200090913005A0913105B0913205BC01CD0156
:10BA30000E94216BDC01CB019C0197FDCDC3832FBC
:10BA4000992787FD9A95D801082E0E94546C09E029
:10BA500010E080912F0590913005A0913105B091B3
:10BA60003205BC01CD010E94216BDC01CB01D80164
:10BA7000082E0E94546C0E94B00568E770E00E9496
:10BA800062313091E0080C947C47C601AA2797FDEB
:10BA9000A095BA2FBC01CD012D8D3E8D4F8D58A1A3
:10BAA0000E94B86B3B014C010E942C6C3093EE0459
:10BAB0002093ED0410927F050C94EE518C0167CD1C
:10BAC0006739710534F186E990E09093C80380935B
:10BAD000C703EECD0196A11DB11D0C94154E019624
:10BAE000A11DB11D0C94094E81E080937F05109239
:10BAF0006505109266051092670510926805109210
:10BB0000F9041092FA041092FB041092FC040C94B5
:10BB100085467093C8036093C703CACD0F96A11DD5
:10BB2000B11D09CB095F1F4F0C943F52F095E19571
:10BB3000FF4F42CB0F96A11DB11D0ACB70939D05FF
:10BB400060939C055A834983BBCD80937B050C94FD
:10BB50007C4781E08093A705A2CB3F893093A6055F
:10BB60003093A7059CCB40937B050C947C47B09207
:10BB70008D05A0928C052091120A2C8F0C94034BFA
:10BB800010928E050C94694B2093840530938505A3
:10BB90004093860550938705109290050C94D04CE5
:10BBA0002092800530928105409282055092830553
:10BBB00010928F050C94DA4B109291050C94424D23
:10BBC0006F3F710509F00CF40DCD2FEF30E00ACD79
:10BBD0002F3F310509F00CF4B2CC2FEF30E0AFCCA1
:10BBE0005090A009252D3327220F331F220F331F1A
:10BBF00020553040241735070CF03ACDA901B90182
:10BC000037CD6F3F710509F00CF46BCC2FEF30E0AE
:10BC100068CC121613060CF432CC229FC001239F6D
:10BC2000900D329F900D112497FD6DC395958795CA
:10BC3000959587952091100430911104281B390B9C
:10BC400032CC0E94B00545E66EED78E00E945805C2
:10BC50008091E60880FF10C080911D0390911E0323
:10BC6000875B934038F480911D0390911E038E5E94
:10BC7000924010F40E94611C1092F9030E94A93CAA
:10BC800081E08093F903579AF6CE4D5F5F4F45CE22
:10BC900081E08093A60503CB8091AD0481FFD1C1E3
:10BCA0002091C7033091C803C9010F964091D50474
:10BCB0005091D604841795070CF0EFC18091A6052A
:10BCC000882309F0EAC18091A80581FFF8C28D7F21
:10BCD0006090D0047090D1048090D2049090D304EE
:10BCE0006092CC047092CD048092CE049092CF04E6
:10BCF00081608093A805421B530B9A012F5030405E
:10BD000037FDF4C280919A0590919B05280F391F49
:10BD100030939B0520939A0520919A0530919B05BD
:10BD2000C90137FF04C088279927821B930B8150D4
:10BD300092400CF481C18091EB089927829FF00119
:10BD4000839FF00D929FF00D1124CF0160E075E00C
:10BD50000E94F76BCB01AA2797FDA095BA2F2091DF
:10BD6000CC043091CD044091CE045091CF04820F89
:10BD7000931FA41FB51F8093CC049093CD04A09370
:10BD8000CE04B093CF0410929B0510929A05B1FE99
:10BD900006C08BE490E09093FC038093FB038091BA
:10BDA000EF08882309F048C100919E0510919F0576
:10BDB000A80117FD93C255954795559547958091D4
:10BDC000270390912803209100013327489F700199
:10BDD000499FF00C589FF00C1124C701B9010E9433
:10BDE000F76B663471050CF073C226E430E03093D3
:10BDF000C8032093C7038091430590914405892B84
:10BE000009F4FBCAD401C3016092CC047092CD0442
:10BE10008092CE049092CF04F8CA1092A10510929D
:10BE2000A0058FEF93E09093CA038093C903F3CCEE
:10BE3000AFE0803A9A0708F0E2C0D801C701FAE003
:10BE4000B695A79597958795FA95D1F7E81AF90AC7
:10BE50000A0B1B0BDA01C901880F991FAA1FBB1F10
:10BE6000880F991FAA1FBB1FA6CC1091DF080C9446
:10BE7000DF462093840530938505409386055093D3
:10BE8000870510928D0510928C05E8EE2E2EE3E0CA
:10BE90003E2E3092AB032092AA030C94424D609246
:10BEA00080057092810580928205909283051092A0
:10BEB0008D0510928C0588EE282E83E0382E309266
:10BEC000AB032092AA030C94DA4B7093C9046093DD
:10BED000C804D092CB04C092CA04CB0177FD6BC1D9
:10BEE000BC0175956795C601D7FC63C16C01D594FB
:10BEF000C7940C941D4A299A0C94B34681E0809310
:10BF000091050C94424D909581959F4F0ECCB09524
:10BF1000A095909581959F4FAF4FBF4F0C94D14AFC
:10BF200020938405309385054093860550938705BB
:10BF300081E0809390050C94D04CB095A09590959D
:10BF400081959F4FAF4FBF4F0C94334C209280058B
:10BF500030928105409282055092830581E0809362
:10BF60008F050C94DA4B81509F4FAF4FBF4F0C940D
:10BF7000744981509F4FAF4FBF4F0C945A49815025
:10BF80009F4FAF4FBF4F0C94EF4981509F4FAF4F22
:10BF9000BF4F0C94E24961507F4F8F4F9F4F0C94DD
:10BFA000B24961507F4F8F4F9F4F0C949C4981E065
:10BFB00080938E050C94694B615E7F4F8F4F9F4F2E
:10BFC000AFCA6FE770E080E090E0660E771E881ED3
:10BFD000991E93CA2D5F3F4F35CB61587F4F8F4FCE
:10BFE0009F4FF1CA61587F4F8F4F9F4F6BCA2D5F94
:10BFF0003F4F4FCA295F3F4F36CA0F9624CA80541D
:10C000009F4108F096C0D801C7017BE0B695A7957F
:10C01000979587957A95D1F7E81AF90A0A0B1B0BC1
:10C02000DA01C901820F931FA41FB51FC4CB615051
:10C03000704E8F4F9F4F8FCB00919E0510919F05A3
:10C04000DACE6090D0047090D1048090D2049090A9
:10C05000D304D401C30180599140A040B0408093E3
:10C06000CC049093CD04A093CE04B093CF04209140
:10C07000EF08222309F446C033273093C8032093E6
:10C08000C70300919E0510919F05BFC9F095E195EA
:10C09000FF4F0C945E47299A81CCC9010F9748172E
:10C0A00059070CF058C08091A705882309F053C0A8
:10C0B0008091A80580FF1EC18E7F6090D004709093
:10C0C000D1048090D2049090D3046092CC047092FA
:10C0D000CD048092CE049092CF0482608093A80514
:10C0E000421B530B9A01215F3F4F37FD0EC18091D8
:10C0F0009A0590919B05821B930B90939B058093CF
:10C100009A050ACE28E730E0B8CF20938405309313
:10C11000850540938605509387050C94B84C209371
:10C1200084053093850540938605509387050C94CC
:10C130002A4DD801C7016CE0B695A79597958795CC
:10C140006A95D1F7E81AF90A0A0B1B0BE20EF31EE7
:10C15000041F151F34CB2091A805822F99278370C7
:10C160009070892B81F12C7F2093A80510929B055C
:10C1700010929A056090D0047090D1048090D204FF
:10C180009090D3046092CC047092CD048092CE043F
:10C190009092CF04B1FEC0CD84EF91E09093FC0368
:10C1A0008093FB03B9CD81509F4FAF4FBF4F0C948D
:10C1B000C44C01969BCE019693CE295F3F4F4F4FC3
:10C1C0005F4F0C940D4D6090D0047090D10480901E
:10C1D000D2049090D304A0CD21503F4F30CC295FA2
:10C1E0003F4F4F4F5F4F0C949B4C81509E4FAF4F32
:10C1F000BF4F0C94864C81509F4FAF4FBF4F0C9454
:10C20000CE4BB095A095909581959F4FAF4FBF4F66
:10C210000C94874B295F3F4F4F4F5F4F0C943F4B20
:10C2200021503E4F4F4F5F4F0C94264BB095A09539
:10C23000909581959F4FAF4FBF4F0C94204BF09539
:10C24000E195FF4F0C94DB4681509F4FD6CB815038
:10C250009F4FBCCB81509F4FAF4FBF4F0C94364D7B
:10C26000F095E195FF4F0C94154A21503E4F4F4FEA
:10C270005F4F0C94F44CB095A095909581959F4F8D
:10C28000AF4FBF4F0C94EE4C81509F4FAF4FBF4FFD
:10C290000C94614BB095A095909581959F4FAF4FB1
:10C2A000BF4F0C94824C295F3F4F4F4F5F4F0C9410
:10C2B000A64B21503E4F4F4F5F4F0C948D4B6090DB
:10C2C000D0047090D1048090D2049090D30410CD0B
:10C2D0006739710534F026E930E089CD4D5F5F4F55
:10C2E0006ACD7093C8036093C70385CD30952195BF
:10C2F0003F4F08CD6090D0047090D1048090D2045C
:10C300009090D304EACE039691CC309521953F4F7F
:10C31000EECE3A94E2E0F0E0EE0EFF1E0C5F1F4F0F
:10C320000894C11CD11C37FC02C00C945156ED96E8
:10C330000FB6F894DEBF0FBECDBFDF91CF911F9136
:10C340000F91FF90EF90DF90CF90BF90AF909F90B4
:10C350008F907F906F905F904F903F902F900895B7
:10C360008091B5059091B605A091B705B091B8053B
:10C370008093AD059093AE05A093AF05B093B00543
:10C380008091B1059091B205A091B305B091B4052B
:10C390008093A9059093AA05A093AB05B093AC0533
:10C3A00008951092C0051092BF051092BE0510921C
:10C3B000BD05089584B1806A84B93D9A82E58CBD3B
:10C3C0001DBC459A81E08093B2098AEA8093B60940
:10C3D00083E88093B7099AE09093B8091092BA095C
:10C3E0001092B9091092BC091092BB091092140A5C
:10C3F0001092D8091092D9098CE48093DA0984E06C
:10C400008093DB099093DC090895EF92FF920F93DC
:10C410001F938091F5089927880F991F880F991FFE
:10C420007C010027F7FC0095102F80912905909141
:10C430002A05A0912B05B0912C05BC01CD01A801C6
:10C4400097010E942C6C3093BA092093B90980910E
:10C45000210590912205A0912305B0912405BC01EE
:10C46000CD01A80197010E942C6C3093BC09209348
:10C47000BB092091A8093091A9094091AA095091BE
:10C48000AB09DA01C901E3E0880F991FAA1FBB1F9E
:10C49000EA95D1F7820F931FA41FB51F820F931F38
:10C4A000A41FB51F20918603309187034091880314
:10C4B00050918903BC01CD010E942C6C3093C209BC
:10C4C0002093C109E0913305F091340580916A0908
:10C4D00090916B09BF010E94F76BCB019B01220F6A
:10C4E000331F220F331F280F391F280F391F37FD25
:10C4F0001CC135952795359527953093BE09209316
:10C50000BD098091A4099091A509BF010E94F76B14
:10C510009B01220F331F220F331F260F371F260FB9
:10C52000371F37FDFFC035952795359527953093F3
:10C53000C0092093BF091092340510923305109260
:10C540006B0910926A091092A5091092A4098091B2
:10C55000B80999278C30910509F4A1C08D30910557
:10C560000CF069C08A30910509F4A4C10B9709F455
:10C5700010C18091D809882309F4CBC02091DE092D
:10C580003091DF09C90181509E4F8F5F9340C8F4FD
:10C590004091E0095091E109CA0181509E4F8F5F9F
:10C5A000934078F48091E60885FF0BC03093C00576
:10C5B0002093BF055093BE054093BD058AEF80933D
:10C5C000C2058091E4099091E50921E0893692073E
:10C5D0000CF056C19C019093F0048093EF0480917D
:10C5E000ED049091EE04281B390BC901845E9D4F28
:10C5F00068E671E00E94F76B845B90409093EC04D6
:10C600008093EB042091E8093091E9098091FB03C4
:10C610009091FC038217930740F480917B07882355
:10C6200021F43093FC032093FB038091DD098736CE
:10C6300009F0ADC12AC18E30910509F476C18E3062
:10C6400091050CF475C00F9709F093CF80910D09F7
:10C650008093C909809135098093CA09809192031A
:10C660008093CB09809106098093CC0980910709BA
:10C670008093CD09809108098093CE098091910320
:10C680008093CF0980910A098093D00980910B098A
:10C690008093D10980910C098093D2096ACF80914F
:10C6A0007B07863018F010927B0785E08093C909DC
:10C6B000809132098093CA0980912C0890912D08AD
:10C6C0009093CC098093CB098091CC049091CD04B8
:10C6D000A091CE04B091CF04BC01CD0125E030E0A3
:10C6E00040E050E00E942C6C3093CE092093CD099D
:10C6F000809128098093CF09809129098093D009DE
:10C7000080912A098093D1098091D809882309F062
:10C7100035CF1092C0051092BF051092BE05109241
:10C72000BD0535C12D5F3F4FFECE2D5F3F4FE1CEA2
:10C73000809123098093C909809124098093CA09B3
:10C74000809125098093CB09809126098093CC099B
:10C75000809127098093CD0980912B098093CE0980
:10C7600080912C098093CF0980912D098093D00965
:10C77000809130098093D10980912E098093D2094C
:10C7800080912F098093D309809131098093D40936
:10C79000F0CEF8948091E008E82FFF27EE0FFF1FFE
:10C7A000E455F74F0190F081E02DE038F1050CF0F1
:10C7B000D1C02FEFE138F20714F4E1E8FFEFE09386
:10C7C000C9098091E108E82FFF27EE0FFF1FE4550C
:10C7D000F74F0190F081E02DE038F1050CF4CDC069
:10C7E000EFE7F0E0E093CA098091DF08E82FFF2728
:10C7F000EE0FFF1FE455F74F0190F081E02DE03878
:10C80000F1050CF4B2C0EFE7F0E0E093CB098091C2
:10C81000DE08E82FFF27EE0FFF1FE455F74F0190CA
:10C82000F081E02DE038F1050CF497C0EFE7F0E07F
:10C830007894E093CC098091E5048093CD098091B0
:10C84000E3048093CE098091E1048093CF09809125
:10C85000DF048093D0098091DE048093D109809118
:10C86000DD048093D209809130089091310897FDC2
:10C870008CC095958795959587958093D30979CEAA
:10C880002091EF043091F004AACE8091EA098093C0
:10C89000110A8091EB098093130A8091EC0980932F
:10C8A000120A8091ED098093140A8091EE09809319
:10C8B000150A6DC08091C1048093C9098091C0049C
:10C8C0008093CA098091BF048093CB098091BE04F4
:10C8D0008093CC098091BD048093CD098091BC04E4
:10C8E0008093CE098091BB048093CF098091BA04D4
:10C8F0008093D0098091AD048093D1098091AD04DB
:10C90000837F8093AD0480912703909128038093C7
:10C91000D209809100018093D309A2E0B0E00E9487
:10C92000476C802D8093D40924CE8091D9098093BF
:10C93000C9098091DA098093CA098091DB09809343
:10C94000CB098091DC098093CC098091020180930E
:10C95000CD090FCEEFE7F0E032CF8FEFE138F807E7
:10C960000CF066CFE1E8FFEF63CF6FEFE138F60739
:10C970000CF04BCFE1E8FFEF48CF4FEFE138F40781
:10C980000CF030CFE1E8FFEF2DCF039672CF1F916F
:10C990000F91FF90EF9008958091B209882309F4D8
:10C9A0003BC0459886EB99E09093B4098093B30916
:10C9B0008091C105E82FFF27E453FC4F982F9F5F1C
:10C9C00080818093B809973008F027C09093C10503
:10C9D0001092B2090E94056281E08093B5090000BF
:10C9E0000000000000000000000000000000000047
:10C9F0000000000000000000000000000000000037
:10CA00000000000000000000000000000000809115
:10CA1000B6098093D5098EBD08951092C105D8CF6F
:10CA20002091B209222309F045C00DB407FE42C08F
:10CA300084E08093FA03459A3EB58091C305992717
:10CA40008130910509F437C0823091050CF451C052
:10CA5000029709F439C02091B509203208F030C09E
:10CA600045980000000000000000000000000000E9
:10CA700000000000000000000000000000000000B6
:10CA800000000000000000000000000000000000A6
:10CA90000000E091B309F091B409E20FF11D80812B
:10CAA0008EBD8091D5099081890F8093D5092F5F24
:10CAB0002093B5090895353551F12093C305CBCFA7
:10CAC00081E08093B209F3CF8091D709E82FFF2747
:10CAD000E950F64F30838F5F8093D7098A3100F198
:10CAE0008091C405381711F12093D8091092C3051D
:10CAF000B2CF892B09F0AFCF2093D7093093C4056B
:10CB0000313809F0A8CF81E08093C305A4CF80918C
:10CB1000C405830F8093C40582E08093C3059BCF37
:10CB20008091C405830F8093C40595CF8AE1E7EF18
:10CB3000F9E0ADEDB9E001900D928A95E1F781E061
:10CB40008093D8091092C30586CF87B18C6087B9CE
:10CB5000089508958091C9008F778093C9008091CE
:10CB6000C9008F7B8093C9008091C9008F7D80931D
:10CB7000C9005A9A52981092CD0084E190E08093B7
:10CB8000CC008091C80082608093C80080E18093CF
:10CB9000C9008091CA008F778093CA008091CA0033
:10CBA0008F7B8093CA008091CA008F7D8093CA00DA
:10CBB0008091CA008F7E8093CA008091CA00877FCF
:10CBC0008093CA008091C9008B7F8093C9008091B7
:10CBD000CA0084608093CA008091CA0082608093FA
:10CBE000CA008091C80087FF0CC08091CE00809160
:10CBF000C800882334F48091CE008091C800882337
:10CC0000A4F38091C90080688093C90008951F93A0
:10CC1000CF93DF9380E197E20E94F717EC0110E0D9
:10CC20008091C9008F778093C9008091C9008F7E61
:10CC30008093C9005A988FE198E09F938F931F9338
:10CC40000E9478140F900F900F90CE010E94001850
:10CC5000882309F066C04A9BF8CF8AE590E00E94DD
:10CC6000F717EC0185E598E09F938F931F920E9440
:10CC70007814529A0F900F900F90CE010E940018D6
:10CC80008823D9F383E690E05A9A019797FFFCCF67
:10CC90008FE891E05A98019797FFFCCF89E090E0E8
:10CCA0005A9A019797FFFCCF89E090E05A98019734
:10CCB00097FFFCCF8FE891E05A9A019797FFFCCF3E
:10CCC0008FE891E05A98019797FFFCCF89E090E0B8
:10CCD0005A9A019797FFFCCF89E090E05A98019704
:10CCE00097FFFCCF8FE891E05A9A019797FFFCCF0E
:10CCF0008FE891E05A98019797FFFCCF89E090E088
:10CD00005A9A019797FFFCCF89E090E05A980197D3
:10CD100097FFFCCF8FE891E05A9A019797FFFCCFDD
:10CD20000AC08BE598E09F938F931F930E9478141D
:10CD30000F900F900F9052985A980E94AA65DF9119
:10CD4000CF911F9108951F920F920FB60F92112449
:10CD5000CF92DF92EF92FF920F931F932F933F9307
:10CD60004F935F936F937F938F939F93AF93BF93F3
:10CD7000CF93DF93EF93FF932091CE008091D50363
:10CD8000813009F44BC08091CB058823C9F040E085
:10CD900050E08091CC058823C9F4452B09F44AC0A2
:10CDA00081E08093CC058091CD058F5F8093CD0588
:10CDB00043E08091CD058031E8F44093CB0507C274
:10CDC00041E050E08091CC05882339F3813009F4AB
:10CDD0004AC08230B9F1833009F44AC081E08093BF
:10CDE000D5031092CD051092CF0544E48091CD0576
:10CDF000803118F38091CF05882331F48091D503D9
:10CE0000882311F4809384031092CD051092CF05EE
:10CE10001092CC0584E48093CB05D9C11092D50340
:10CE200084E48093CB051092CD051092CC0510922E
:10CE3000CE05CDC144E48093CD058093CC0580938D
:10CE4000CE05D4CF452B51F643E02093CE059091EB
:10CE5000CD05923009F4C7C083E08093CC059F5F75
:10CE60009093CD05C3CF452B09F0B8CF82E099CF81
:10CE7000452B09F0B3CF482F82E08093CC058091F9
:10CE8000CD058F5F8093CD059091CE05892F869536
:10CE90008695C82FDD27CF70D0702196892F9927CE
:10CEA000982F88273327822B932B937080509240A2
:10CEB00063E070E00E94F76B6B01CB30D10508F0A6
:10CEC0008BC07E01EC0EFD1EF701E455F74F80810B
:10CED00091819B01281B390BC90137FD34C106978D
:10CEE0006CF4C530D10550F48091DE04883C08F024
:10CEF00032C18091DE04865F8093DE04C630D105A6
:10CF000009F482C0C230D10509F478C0C430D1051B
:10CF100009F413C18091DE04843B08F469C0C53074
:10CF2000D10508F065C087010E53174FF701E4558E
:10CF3000F74F808191819601281B390BC90163E06D
:10CF400070E00E94F76BCB01880F991F860F971F27
:10CF5000F80191838083C530D10538F42CEA38E09C
:10CF6000E20EF31EF701D182C082C530D10509F46B
:10CF7000DFC0C730D10509F4D6C0269709F036CFF7
:10CF800020911C0A30911D0A2237310509F411C184
:10CF90005FEF2F38350709F4FFC02F583F4F09F4D2
:10CFA000E5C08091200A9091210A9093B90880935E
:10CFB000B8088091220A9091230A8237910509F4DA
:10CFC000D3C042988091240A9091250A8237910516
:10CFD00009F4D9C043980ACF629708F407CF81E0DB
:10CFE0008093D50303CF27FDB2C01092CF0534CF75
:10CFF000F701EE53F74F11821082ADCFC4E0D0E0BD
:10D0000078E0E72EF12C86CF35E6C316D10444F044
:10D010001092170A1092160A1092190A1092180A02
:10D020005AE0C516D1044CF48091160A9091170A63
:10D0300001969093170A8093160A2091160A309150
:10D04000170A2730310509F4A0C08AE0C816D104B8
:10D050004CF4F901E20FF31FE85DF54F8FE89FEF05
:10D06000918380839CE9C9169FEFD906B4F4F90136
:10D07000E20FF31FE85DF54F82E790E09183808334
:10D080002630310550F48091180A9091190A809544
:10D0900090959093190A8093180A2630310509F06B
:10D0A00031CF2091180A3091190A2115310539F034
:10D0B0008091340A9091350A8F589F4F59F0232B55
:10D0C00009F020CF8091340A9091350A823791057A
:10D0D00009F018CF20912A0A30912B0A30931D0AAB
:10D0E00020931C0A80912C0A90912D0A90931F0A7C
:10D0F00080931E0A80912E0A90912F0A9093210A04
:10D100008093200A8091300A9091310A9093230AEB
:10D110008093220A8091320A9091330A9093250AD3
:10D120008093240AEFCED092BD08C092BC0825CFD0
:10D13000D092BB08C092BA081CCFC2E0D0E064E035
:10D14000E62EF12CE7CE909581959F4FC8CE81E0D9
:10D150008093CF0581CE88EC8093DE0480916F00B0
:10D160008F7D80936F00CACE429A2CCF80911E0A89
:10D1700090911F0A8237910509F013CF9093B70859
:10D180008093B6080ECF439A31CE1092170A1092B0
:10D19000160A20E030E059CF80911E0A90911F0AB4
:10D1A0008F589F4F09F0F9CE1092B7081092B60829
:10D1B000F4CE80911E0A90911F0AFFEF8F389F07CF
:10D1C00009F0E6CE9093B7088093B608E1CEFF91C0
:10D1D000EF91DF91CF91BF91AF919F918F917F910F
:10D1E0006F915F914F913F912F911F910F91FF9000
:10D1F000EF90DF90CF900F900FBE0F901F9018957B
:10D20000CF93FC0197FD21C0C1E028E631E0CF01BA
:10D21000B9010E94F76BFC018B35910554F08B55D9
:10D2200090408A35910538F484EB90E08E1B9F0B7B
:10D23000FC0141E013C0CF01855B90408A35910528
:10D2400048F4E45BF0404FEF09C0CFEFF095E19573
:10D25000FF4FDBCF2E1B3F0BF9014FEFEE0FFF1FF0
:10D26000E054F64F259134918C2F992787FD9095A6
:10D27000829FB001839F700D929F700D1124842FA7
:10D28000992787FD9095689FA001699F500D789F11
:10D29000500D1124CA01CF9108952AE530E0281BD2
:10D2A000390BC9010E94006908951F93CF93DF9342
:10D2B000EB016115710519F4009709F494C097FD0D
:10D2C0003EC011E0209729F48AE51802B00111242C
:10D2D0008AC0AA2797FDA095BA2F26E0880F991F2C
:10D2E000AA1FBB1F2A95D1F79E01442737FD409501
:10D2F000542FBC01CD010E942C6CF90137FD2CC0CC
:10D3000081E0EA35F807ACF08CE1E73AF807CCF0B9
:10D310002AE530E01C161D061CF5812F992787FD94
:10D320009095829FB001839F700D929F700D112484
:10D330005AC0EA59F74F8491282F3327EBCF1FEFBC
:10D34000C1CF89E0ED38F8078CF485E0EA3BF807B7
:10D3500084F028E530E0DECFF095E195FF4FD0CFA7
:10D36000D7FD0EC0B901645B70403DC029E530E0D7
:10D37000D1CF84E0E731F80754F027E530E0CACF99
:10D38000111684F764EB70E0621B730B2CC083E012
:10D39000EE32F8071CF026E530E0BCCF82E0E93938
:10D3A000F8071CF025E530E0B5CF82E0E233F8075E
:10D3B0001CF024E530E0AECF81E0E73EF8071CF03A
:10D3C00023E530E0A7CF81E0ED3AF8071CF022E535
:10D3D00030E0A0CFEF57F1401CF021E530E09ACFCC
:10D3E00020E530E097CFCB01DF91CF911F910895D9
:10D3F000EF92FF920F931F93CF93DF937B018C01EA
:10D4000020E030E040E050E0FA01E9016FE00BC0BD
:10D41000C21BD30BE40BF50B2F5F3F4F4F4F5F4FFA
:10D42000615067FD31C0220F331F441F551FCC0FC1
:10D43000DD1FEE1FFF1FCC0FDD1FEE1FFF1FD801EA
:10D44000C7017EE1B695A795979587957A95D1F70F
:10D45000C80FD91FEA1FFB1FEE0CFF1C001F111F76
:10D46000EE0CFF1C001F111F2F5F3F4F4F4F5F4FF0
:10D47000C217D307E407F50758F621503040404063
:10D480005040615067FFCFCF569547953795279508
:10D49000CA01B901DF91CF911F910F91FF90EF90D9
:10D4A0000895002422273327442751E0BB27EE2785
:10D4B000FF27A0E1660F771F881F991F001C221FFE
:10D4C000331F441F660F771F881F991F001C221FE0
:10D4D000331F441F2AF4050E2B1F3E1F4F1F04C08D
:10D4E000051A2B0B3E0B4F0B550FBB1FEE1F587F22
:10D4F000556047FD5250AA95E9F6E695B7955795C0
:10D50000E695B7955795852F9B2F089522273327AA
:10D5100041E0552768E0880F991F221F331F880FAD
:10D52000991F221F331F1AF4240F351F02C0241B1A
:10D53000350B440F551F487F456037FD42506A95B3
:10D5400051F75695479556954795842F0895AA27E4
:10D5500097FF04C0809590958A1F9A1F77FF04C09B
:10D56000609570956A1F7A1F669F9001779FA00152
:10D57000679F300D411D5A1F300D411D5A1F889F56
:10D58000F001999F2E0F3F1F401D511D899F300DA7
:10D59000411D5A1F300D411D5A1FCA01B9011124E6
:10D5A00080CFFC014150504030F001900616D1F779
:10D5B0003197CF0108958827992708955058192E3B
:10D5C000A6D001D08CC0BA176207730784079507ED
:10D5D000B1F188F40EF410940B2EBA2FA02D062E64
:10D5E000622F202D072E732F302D082E842F402DD3
:10D5F000092E952F502DFF275523B9F0591B49F0BF
:10D60000573E98F0469537952795A795F040539546
:10D61000C9F776F0BA0F621F731F841F30F4879525
:10D6200077956795B795F040939517FA0F2E089563
:10D63000BF1BBB27BA0B620B730B840BF6CFDEF656
:10D6400092C097FB70D09F3738F0FEE9F91B982FF6
:10D65000872F762F6B2F05C083C09695879577957A
:10D660006795F150D0F73EF490958095709561954F
:10D670007F4F8F4F9F4F0895E89403C097FB0EF4A0
:10D68000F3DFB62F672F782F892F9EE9002427C05C
:10D690000ED05EF004C00BD026F001C008D019F007
:10D6A00020F48FEF089580E0089581E0089597FBBE
:10D6B000092E052600F868942DD0E89407FC07C0D1
:10D6C000621773078407950721F008F40094079404
:10D6D000989408959A95BB0F661F771F881F112491
:10D6E0009923A1F08823B2F79F3F59F0BB0F48F46C
:10D6F00021F4002011F460FF04C06F5F7F4F8F4F53
:10D700009F4F881F9795879597F9089529C0052EF3
:10D71000092607FA440F551F5F3F79F0AA27A5177E
:10D7200008F051E04795880F991F9F3F31F0BB27C4
:10D73000B91708F091E0879508959F919F91112462
:10D7400014C097FB880F991F9F3F31F0BB27B91773
:10D7500008F091E0879508959F919F91112405C04D
:10D76000662777278827992708959FEF80EC0895EB
:10D77000629FD001739FF001829FE00DF11D649FB5
:10D78000E00DF11D929FF00D839FF00D749FF00D41
:10D79000659FF00D9927729FB00DE11DF91F639FE2
:10D7A000B00DE11DF91FBD01CF0111240895991B92
:10D7B00079E004C0991F961708F0961B881F7A9588
:10D7C000C9F780950895AA1BBB1B51E107C0AA1F8A
:10D7D000BB1FA617B70710F0A61BB70B881F991F12
:10D7E0005A95A9F780959095BC01CD01089597FBB6
:10D7F000092E07260AD077FD04D0E5DF06D00020E9
:10D800001AF4709561957F4F0895F6F7909581957C
:10D810009F4F0895A1E21A2EAA1BBB1BFD010DC04C
:10D82000AA1FBB1FEE1FFF1FA217B307E407F507D0
:10D8300020F0A21BB30BE40BF50B661F771F881FAC
:10D84000991F1A9469F760957095809590959B0142
:10D85000AC01BD01CF01089597FB092E05260ED01E
:10D8600057FD04D0D7DF0AD0001C38F450954095FE
:10D87000309521953F4F4F4F5F4F0895F6F79095A4
:10D880008095709561957F4F8F4F9F4F0895F999BF
:10D89000FECFB2BDA1BDF89A119600B40895F7DF8E
:10D8A00001921A94E1F70895F999FECFB2BDA1BD96
:10D8B00000BC11960FB6F894FA9AF99A0FBE089523
:0AD8C0000190F2DF1A94E1F70895D9
:10D8CA005E010A0151756164726F0000416E676CF6
:10D8DA00654E69636B20202020202020416E676CF2
:10D8EA0065526F6C6C202020202020204163634EFB
:10D8FA0069636B202020202020202020416363526E
:10D90A006F6C6C2020202020202020204779726F05
:10D91A0047696572202020202020202048696768F6
:10D92A00742056616C756520202020204163635A5B
:10D93A002020202020202020202020204761732022
:10D94A00202020202020202020202020436F6D70BE
:10D95A006173732056616C7565202020566F6C7454
:10D96A00616765202020202020202020456D7066D8
:10D97A00616E672020202020202020204779726FA6
:10D98A00204B6F6D70617373202020204D6F746F70
:10D99A00722046726F6E7420202020204D6F746FA3
:10D9AA007220526561722020202020204D6F746FF2
:10D9BA0072204C6566742020202020204D6F746FE1
:10D9CA00722052696768742020202020202020209D
:10D9DA00202020202020202020202020202020203D
:10D9EA00202020202020202020202020566172691B
:10D9FA006F4D657465722020202020204D4B334DD9
:10DA0A0061672043616C5374617465205365727653
:10DA1A006F2020202020202020202020486F6F7691
:10DA2A00657267617320202020202020202020207A
:10DA3A0020202020202020202020202020202020DC
:10DA4A0020202020202020202020202020202020CC
:10DA5A0020202020202020202020202020202020BC
:10DA6A0020202020202020202020202020202020AC
:10DA7A00202020202020202020202020202020209C
:10DA8A002020202020202020202020204932432D21
:10DA9A004572726F72202020202020202020202012
:10DAAA002020202020202020202020204750535FA3
:10DABA004E69636B20202020202020204750535F8E
:10DACA00526F6C6C2020202020202020C800016486
:10DADA00FF01FFFF01FC01FC0101737373FF0300E7
:10DAEA007D0000C409C40964000E48616C6C6F2093
:10DAFA0057656C7400000000000000000000000080
:10DB0A00000000000000000000000000000000000B
:10DB1A0000000000000000000000000000000000FB
:10DB2A0000000000000000000000000000000000EB
:10DB3A0000000000000000000000010203040506C6
:10DB4A000708090A01040B050000ECFF6440415A6A
:10DB5A004664640A02969696960840403A10FB304C
:10DB6A00380190D0030090D00300F4016400537090
:10DB7A006F727400004E6F726D616C0000426567CF
:10DB8A00696E6E657200007800FF03640A0B0D0B64
:06DB9A000C0E0F01010159
:00000001FF
